:1000000000400020B17B0000F17B0000F37B00008A
:1000100000000000000000000000000000000000E0
:10002000000000000000000000000000F57B000060
:100030000000000000000000F77B0000F97B0000DA
:10004000FB7B0000695900005D7F0000FB7B000026
:10005000FB7B000000000000FB7B0000FB7B00003E
:100060002938000031830000FB7B0000FB7B00008F
:10007000FB7B0000FB7B0000FB7B0000FB7B0000A8
:10008000FB7B0000E17F0000FB7B0000FB7B0000AE
:10009000FB7B0000FB7B0000FB7B0000FB7B000088
:1000A000FB7B0000FB7B0000000000000000000064
:1000B0000000000000000000000000000000000040
:1000C00010B5064C2378002B07D1054B002B02D02E
:1000D000044800E000BF0123237010BD6C02002023
:1000E00000000000E4EF0000044B10B5002B03D02B
:1000F0000349044800E000BF10BDC04600000000F6
:1001000070020020E4EF0000164B002B00D1144BCE
:100110009D46402292029A1A924600218B460F4633
:100120001348144A121A0BF037FF0F4B002B00D064
:1001300098470E4B002B00D0984700200021040068
:100140000D000D48002802D00C4800E000BF0BF065
:10015000E3FE2000290007F053FF0BF0B7FEC04676
:100160000000080000400020000000000000000027
:100170006C020020D02F00200000000000000000D2
:1001800002000120104011D1042A0ED91368180969
:1001900080B2002809D001388000031D11180979A8
:1001A000002902D001309842F8D170470020FCE7C6
:1001B0000378002B03D05AB2002A01DB01307047CC
:1001C0003F229343C03B59424B41C01803789343AD
:1001D000802BF4D10130F9E710B500240378002B0F
:1001E00001D1200010BDFFF7E3FF0134F6E770B541
:1001F000002204000D00411C092003F03DFE0028F0
:1002000006D001236200134343600023A34200DBB6
:1002100070BD9A00A958821891600133F6E770B555
:10022000012803DC1C2001F0E9F970BD01230D68F1
:1002300011201D42F7D04868184206D1042804D97D
:100240000F2302681340042B01D00E20EBE703F0CC
:1002500071FC6D100400002D03DDFFF7BDFFA84207
:1002600006DA1220DFE72000FFF7A2FF0400013DBD
:10027000012DF8D120787F2809DDDF280BDCF82359
:100280003F22DB00800118406378134018430123AC
:1002900040001843C9E7EF280BDCFC226378120109
:1002A0009B0113403F220007000C0343A07810403D
:1002B000ECE7F72812DCFC22637892021B03134060
:1002C000E0228004520310403F221843E378134099
:1002D000FC220343A07812018001E8E7012040429C
:1002E000D5E7F8B54D680F00EB0706D4042D04D907
:1002F0000F232E683340092B03D00B2001F07EF929
:10030000F8BD6B683609B6B25C10731EA3420FD8F5
:100310000321200009F0FCFC6421642803DC0100B7
:10032000032800DA03212800891903F0D7FD05000E
:100330002B6800201B099BB2013B9C42E0D23A682B
:10034000A31C9B005A510123013464001C436C60C0
:10035000D6E7F0B585B0012803DC1C2001F04EF98A
:1003600012E001274B683A000093022806D08B6800
:100370003B4203D05F10002F00DC17000125009BDB
:100380002B4203D00120404205B0F0BD009B042B5E
:10039000F8D91B680C680F261900314004292DD1AB
:1003A0002C4205D1042C03D923681E40042E01D011
:1003B0000E20D3E70098FFF7E3FEB842E2DB009897
:1003C00003F0B8FB0600200003F0B4FB0378010043
:1003D000002BD7D0781E30180CF094F9041ED1D021
:1003E0003378002B01D0A64202D36800012521E01A
:1003F0003000FFF7DDFE01350600F1E709293ED1A7
:10040000009B5B685B1001939F42BBDC2C422ED1AA
:10041000042C2CD923683340042B28D1200003F06E
:1004200089FB039602907E1C009AB300D058844248
:1004300002D178002843A7E728420ED104280CD91E
:100440000368039A1340042B07D103F073FB0100E8
:1004500002980CF021F90028EBD0019B37009E4256
:10046000E1DD8FE71F00019B9F4200DD8AE77B1CD7
:1004700000999A008A58A242F4D17800B6E703297D
:1004800000D07FE71A0992B25B0F92000B40D31A9B
:1004900001939F4200DD75E72C4229D1042C27D916
:1004A00022681640032E19D1100980B2520F800025
:1004B0003240251D801A019B2E181B1A0193009BA8
:1004C000781E0433019A904200DD5BE72A00191878
:1004D000B2420FD316D10130400087E7042E07D176
:1004E000200003F027FB05002000FFF749FEE2E7AC
:1004F0000F2033E70C78A4461478A44502D10131CB
:100500000132E5E70130DDE7F0B50C0085B00128E8
:1005100004DC1C2001F072F805B0F0BD012708686A
:10052000384206D1042804D90F2102680A40042A5F
:1005300001D00E20EEE762681740FAD1042AF8D9FC
:1005400013680B40042BF4D103F0F4FA0500606843
:1005500003F0F0FA02900CF0A9F8039003002800D1
:10056000002B19D1FFF738FE0190019B0122591C85
:10057000092003F081FC334E306000280ED10020AA
:10058000CAE7039B0299C0180CF0BCF80196019BC6
:100590005E1C0028F5D1E8E70197F8E70122019BEE
:1005A0005B0013434360039B002B18D12800FFF727
:1005B000FFFD019B0400BB4201DC3068ACE7611B1E
:1005C000280003F0D7FC0028D9D0BB1C32689B0060
:1005D00098502000FFF7ECFD01372500E9E7019B6B
:1005E000012B02D12368836096E7681C02990CF006
:1005F00089F801240700019B002F13D0A342DCDB04
:10060000791B280003F0B6FC0028B8D0326801340A
:10061000A3009850039B0299FD1828000CF072F873
:100620000700E8E7A342C8DB28000CF03FF8010010
:10063000280003F09FFC0028A1D001343368A400F7
:10064000E050BAE7E00F002010B503F057FA43007E
:100650000120184310BD0000C30711D404280FD98E
:100660000F2302681340032B0AD119400133591A92
:10067000C0234907DB051940024B1A4011430160B2
:100680007047C046FFFFFF9FF7B507000E001C2014
:10069000012F06DD4C68012322001A40009203D18D
:1006A0000D2000F0ABFF53E0022F02D08A681A42FF
:1006B000F6D0012335681D4200D0A9E0042D00D8F2
:1006C000A6E01C41002C00DC1C000F20296808401B
:1006D000092828D16B685B100093022F05D0B368FE
:1006E000009A5B109A4200DD0093009B01221D1BC3
:1006F0000135EB43DB171D40691C092003F0BCFBEF
:10070000071E09D001236D001D4303003268083322
:1007100045600099A14201DA3800FEBD0134A10014
:10072000515802C3F5E7042845D1280003F002FA26
:10073000FFF752FD0190022F04D0B3685B1098427E
:1007400000DD0193019BA34204DA002003F006FCC4
:100750000700E1E7280003F0EDF90700009BA34242
:1007600021DB2800009703F0E5F905003800FFF7CA
:100770001FFD019B01340700A342F7DA009BC41A56
:10078000200003F0EBFB071EC6D003F0D3F9019065
:10079000306803F0CFF92200009B591B41180198E3
:1007A0000BF0DEFBB8E73800FFF702FD009B070007
:1007B00001330093D2E703282AD10B099BB2490FDA
:1007C0009B000140591A022F04D0B2685210914286
:1007D00000DD1100A14205DA00220320110003F020
:1007E0004BFBB5E703200E1B331DD9170140C91879
:1007F0008910002203F040FB071E00D18CE7013670
:1008000031000334FFF728FF381D29193200C7E7EC
:10081000212046E7F7B5002804DC1C2000F0EEFE9E
:10082000040014E00D6801272E003E4011D03D4128
:10083000FF2D01D91320F1E700223900032003F036
:100840001BFB041E03D00021FFF706FF25712000CB
:10085000FEBD042DEED90F232A681340042B1BD1B3
:100860002800FFF78DFCC31C07000320D9170140A7
:10087000C9188910320003F0FFFA041EE7D03900CE
:10088000FFF7EAFE280003F055F9231D01003A00A6
:1008900018000BF065FBDAE7092B1FD103206B680A
:1008A00032005B1001930333D9170140C918891036
:1008B00003F0E2FA041ECAD00199FFF7CDFE019BB6
:1008C0009E42C4DAB300EB189B683B4204D05B1035
:1008D000FF2BAFD8A21913710136F0E7032BA9D172
:1008E0002C00B4E710B57F2902DC0170013010BD87
:1008F0001A4B99420CDC40238A115B42134303706C
:100900003F230B4080214942194341700230EEE7FA
:10091000134B994210DC20230A135B4213433F24FC
:10092000802203708B1152422340214013430A431B
:10093000437082700330DAE70A4B9942D7DCF02328
:100940000370603B4370113B8A11FF3B1A43827076
:100950003F2211401943C1700430C8E7FF0700006F
:10096000FFFF0000FF0F0100F0B50D0085B000286B
:1009700003DC1C2000F042FE0DE0096801220800A3
:1009800010400AD002AC11412000FFF7ABFF011B61
:10099000200003F0EFFA04001AE004293FD90F23E6
:1009A0000C682340092B3AD14B685B100193032359
:1009B0009C46019B9A420EDD03F0D0FA041E07D03C
:1009C0002E68012503F0B6F82F00019B9D421DDD26
:1009D000200005B0F0BD01329300CC580123234024
:1009E00001D10D20C6E764107F2C0DDD0D4E0223D2
:1009F000B44209DD0C4E6346B44205DD00270B4EC0
:100A0000E30FA6427B419B00C018D2E70135AB0043
:100A1000F1583942E5D04910FFF764FFD5E72120AE
:100A2000A8E7C046FF070000FFFF0000FF0F01001E
:100A300070B5002805DC1C2000F0E0FD0500280052
:100A400070BD0C68E30701D40D20F5E76410E343A3
:100A5000DB171C40E11C89100022032003F00CFA74
:100A6000051EECD02100FFF7F7FDE8E710B5040004
:100A70000120084010D104290DD90F230A68134022
:100A8000042B08D1080003F055F8010020000BF0FA
:100A900003FE4342584110BD0020FCE7F7B50F00AC
:100AA000012803DC1C2000F0A9FDFEBD01264D68D5
:100AB0002E4006D1042D04D90F222B681A40092A92
:100AC00001D00B20EFE76A681B099BB25410A342C8
:100AD00000D85C1E39681E48FFF7C8FF012301904B
:100AE000002813D139681B48FFF7C0FF002811D038
:100AF000002C0DD00123621C013C9C4092005351FC
:100B000023436B6004E00136B200AB50B442FADA22
:100B10000020CAE73B680D20DA07C4D55B10002B24
:100B200011DD9C420FDB9B00A200291DEB188918E8
:100B30000433994209D10123013C9C40AA181C436B
:100B400053606C60E4E71220ADE758681860EFE787
:100B50003BD600003FD60000002310B50C000B7000
:100B6000C30705D50D49421020000BF059FD08E0E0
:100B70000B49002802D0042804D10A4920000BF0B8
:100B80006FFD10BD0428FCD90F2302681340042B0D
:100B9000F7D102F0CFFF04490200E5E7E4E00000EE
:100BA00044D600004AD600004FD60000F0B593B0FE
:100BB000060002911C20012E1DDD029B01251B68F1
:100BC0001C002C4000D0ADE0042B00D8E6E01A68F1
:100BD0000F231A40092A4AD10394039A02999200DA
:100BE0008A5817002F4005D1042A03D910681840ED
:100BF000092806D0222000F001FD0190019813B0D1
:100C0000F0BD52685210A418039A01320392964222
:100C1000E3D1611C012203F02FF90190002802D1D9
:100C200000230193EAE7019B6400190025435D60FE
:100C30000831029ABB00D05802684368120992B288
:100C40005B109A4200D8531E0022934209DCDA431B
:100C5000D21713409B00C918039B01379F42E8DB62
:100C6000CCE794000519AD6801320D51EDE727007E
:100C7000032A59D10193029ABB00D3582B42B9D110
:100C8000042BB7D9186801990140032939D1020909
:100C900092B2430F92000B40D31A1C190137BE4287
:100CA000E9D10320E31CD9170140C918891000229B
:100CB00003F0E2F801900028B2D000252100FFF7F0
:100CC000CBFC019B1E1D029AAB00D45801231C4291
:100CD0001FD1042C1DD90F2123681940032918D1D5
:100CE000180980B25B0F80000B40C01A00238342BA
:100CF00013DBC343DB17184001353618BD42E2DB76
:100D00007CE7042900D075E71800FFF739FA2418AA
:100D1000C4E72000FFF734FAE8E7E2181279F2544A
:100D20000133E4E700273C000F25029ABB00D358AB
:100D30000122134234D1042B32D918680100294012
:100D4000042935D11800FFF71BFA24180137BE42D9
:100D5000EBD1200003F002F90190002800D15FE7F9
:100D6000029FB600BB19041D029301233D681D427A
:100D700029D1042D27D90F262B681E40042E37D1E8
:100D80002800FFF7FDF90600280002F0D3FE01005D
:100D9000200032000BF0E4F8A41922E02700C3E79A
:100DA000180005A9FFF7D8FE05A80BF07FFCCCE7DB
:100DB000032900D01EE7020992B2430F92000B40B4
:100DC000D31A1C19C2E705A92800FFF7C5FE05A81C
:100DD0000BF06CFC05A90500020020000BF0C0F828
:100DE0006419029B0437BB42BFD10023237005E77F
:100DF000032EF6D11A0992B25B0F92001E40961B89
:100E0000291DC5E7F0B50D0097B0002806DC1C20B1
:100E100000F0F4FB0700380017B0F0BD0C680121AA
:100E200023000B40009306D1042C04D922680F3311
:100E30001A40092A01D00B20EAE762685210039297
:100E4000002A03DC009803F089F8E3E7504A019296
:100E500001280BD06868084208D1042806D9026826
:100E60001340042B02D102F065FE019001980BF0B3
:100E70001DFC06000F27039B0834013B05935E43CE
:100E8000039B02909B00E3180493012320681842FF
:100E900073D1042871D901680B003B409C46042B98
:100EA00003D1FFF76DF9861909E0032B6CD1624677
:100EB0000B099BB2490F9B0011405A1A9619049BCB
:100EC0000434A342E1D1300003F048F8071EA2D059
:100ED0002B680793029B002B03D0686802F02AFE60
:100EE0000190380002F026FE0400009B079A9B0048
:100EF000D3189E68300002F01DFE01233340050028
:100F00000693002B01D1042E04D809A93000FFF765
:100F100023FE09AD28000BF0C9FB069B0490002BB3
:100F20000ED1042E0CD90F2133681940032907D1A3
:100F30001A0992B25B0F92000B40D31A351D04932D
:100F40002000049A29000BF00BF8049BE418029B84
:100F5000002B0AD0059B009A934206DD2000029ADE
:100F600001990AF0FDFF029BE418009B01330093F6
:100F7000009A039B9342B8D14DE709A9FFF7ECFD16
:100F800009A80BF093FB8EE702F0D4FDF9E7C04609
:100F900006DB000010B50024A04207DD0B68013419
:100FA0001C4003D05C10E343DB171C40611C012292
:100FB000092002F061FF002803D0012364001C43D4
:100FC000446010BD0A6870B510000125284034D176
:100FD000042A32D90F24136849681C40092C17D100
:100FE00054681B099BB22C41A34200D85C1E84426A
:100FF00005DC02200133984206DB00200FE085006B
:101000005519A9600130F2E7840011510130F2E76F
:10101000032C12D1294203D1132000F0EFFA70BD46
:101020004910FF29F8D81B099BB204329B00D31842
:101030009342E2D911700132FAE70B2000F0DEFA98
:10104000DBE70000F8B5012700254E680C003740AB
:10105000AF420ED13D00042E0BD90F2233681A4047
:10106000092A10D172681B099BB25510AB4200D8F7
:101070005D1E2168CB0716D54C10002C01DDA54262
:101080001CDA122030E0042A04D13000FFF778F88F
:101090000500EEE7032AECD11D09ADB25B0FAD00F0
:1010A0001340ED1AE5E72748FFF7E0FC002813D0CE
:1010B0000BF052FA290008F011FF4C1C002F3ED112
:1010C000042E3CD90F2332681340092B10D1013470
:1010D000A400A4592000F8BD21681B48FFF7C6FCF6
:1010E0002C000028EAD1113000F088FA0400F1E762
:1010F000042B1CD1300002F01DFD0500012C0EDC7C
:10110000FFF756F8461B300002F028FF041EE1D01E
:1011100002F010FD320029000AF022FFDAE72B78F6
:10112000013C002BADD02800FFF742F8E5E7032B88
:1011300005D13419E37801245B001C43CAE70B2076
:10114000D2E7C04634D600003FD60000F7B54D6860
:101150000F002A0001210A402FD1042D2DD90F2480
:101160002B68BE681C40092C14D169681B099BB20E
:101170004C100192A34200D85C1E39682A48FFF740
:1011800075FC00282DD00F232A681340092B1DD190
:10119000012317E0032C10D10E4203D1132000F0DD
:1011A0002DFAFEBD72100192FF2AF7D81A0992B2E9
:1011B0005B0F92001C40141BDFE70B20EFE70133AD
:1011C0009A00AE509C42FADA0020EAE7032BFBD1EA
:1011D0002B0001335A1BA242F6DC6A461279DA7000
:1011E000F7E73968CB0706D54910002901DD8C42A5
:1011F00009DA1220D3E70D48FFF738FC2100002858
:1012000001D11130CBE70F232A681340092B03D1FA
:10121000013189004E51D7E7032BD5D16B461B799D
:101220006D18EB70D0E7C0463BD600003FD60000FB
:1012300070B501240868204207D1042805D90F257C
:1012400001680D40092D02D14468200070BD032DB6
:1012500008D10A0992B24B0F92002B40D31A5B00BF
:101260001C43F2E7042DF0D102F064FCFEF7B4FF5A
:1012700040000443E9E7000010B5034A0D2103488C
:1012800004F046FC10BDC046CCD50000C4D500001B
:1012900000207047042070470120704710B50020DF
:1012A00002F05CFE10BD0020704700207047002057
:1012B00070470020704700207047002070470020D2
:1012C000704700207047000010B5034A0C21034806
:1012D00004F01EFC10BDC046D4D6000034D7000078
:1012E00070470378002B03D05AB2002A01DB01308B
:1012F00070473F229343C03B59424B41C01803788B
:101300009343802BF4D10130F9E70000F8B50127B1
:10131000060014000800394227D104293FD90F23C1
:101320000A681A40042A3AD13C4213D1042C11D93C
:1013300022681340042B0DD102F0FCFB05002000B5
:1013400002F0F8FB010028000BF0A6F900282EDBC4
:101350001FD127E0E30722D502F0ECFB0A2200218F
:101360000BF06CFA0500601010E0174015D1042A4C
:1013700015D90F2312681340042B10D120004D10F3
:1013800002F0D8FB0A2239000BF058FA85420EDB36
:1013900008DD002E09DC00200CE04D10E3E70F22F1
:1013A000054B1A700136022EF5D8042002E0042005
:1013B00076173040F8BDC046AC020020F8B50600F4
:1013C0000024294BE500ED182B79032B06D00134BE
:1013D000FF2CF6D1013CFF3C2000F8BD30000BF0A3
:1013E00065F9E3B202003100180004F0CDFB0028DB
:1013F000F2D12A6851688842E9D08300D3189B68EB
:101400000130F02BF7D101238000083012181A4266
:10141000DDD1042ADBD90F21136819400429D6D164
:101420001B0998B201230130800010181842CED158
:101430000428CCD90F2203681340042BC7D102F033
:1014400079FB03270500092128000BF017F9002874
:10145000BDD0013F451C002FF5D1310028000BF015
:1014600051F98542B8D0B2E7A425002010B5012477
:10147000044002D04410200010BD042810D90F23CE
:1014800002681340042B07D102F054FB21000A220A
:101490000BF0D4F90400EEE7032B01D10430F5E79B
:1014A0000D22014B1A70E6E7AC020020012210B5B4
:1014B000024018D1042802D903681A0992B2012304
:1014C0000B4012D1042902D90B681B099BB20024DE
:1014D000934206D104309B000431C318984206D3CE
:1014E0000124200010BD0022E9E70023EFE7047883
:1014F0000A78002C01D1002AF2D001300131944247
:10150000ECD00024EDE70000F7B50700009101934F
:101510003049314B002A02D002220A70013A0026DB
:101520001A601B68CE54BE4200DBF7BD009AB300C0
:10153000D058294B274D1C68C8239B0065191C1BDC
:101540000123184206D0254A4310210028000BF041
:1015500035F809E0224A002802D004281BD1214A8C
:10156000210028000BF02AF81A4C20000BF09EF8FE
:10157000194A019B1060002B0BD07B1EB34208DD83
:10158000194B984205D8431C136020222254002294
:10159000E2540136C7E7042819D90F2301680B402C
:1015A000042B04D102F0C6FA104A0300CDE7092B40
:1015B00003D143680E4A5B10C7E7032B08D10A0921
:1015C00092B2490F92000B40D31A0A4ABDE7012399
:1015D000094ABAE7AD020020D0050020E4E000008F
:1015E00044D600004AD600001F0300000FE70000A9
:1015F000A4D90000B3D90000BED90000014B187077
:1016000000207047AC02002070B501F0E5FF094CE6
:101610000100251D1F2228000BF060F828000BF0A8
:1016200045F804230430800800011843206020009E
:1016300070BDC04688020020C368F0B59D00836875
:1016400089B05D190300183306930369069A9F0059
:10165000069B0290DF19436901939B00D318039303
:10166000D14B1B78002B26D17F222B68CF491C122F
:1016700013409B005B58043501929F46029B5878AB
:1016800004F09EFE0023029A137027E0C64B1B78DD
:10169000002B10D12B68019A1C121340C34A9B00E7
:1016A0009B580435E9E7069B3A1DD11ABE4BD82951
:1016B00028DD1A221A70029BBB4C9B68217801938B
:1016C000EA1A029B92109B7812021A43029B5878E6
:1016D00004F07EFE0023029A23701370029B069A88
:1016E0009B680193ED1A029BAD10DD60069BFE1A0C
:1016F000029BB6101E61039B9B1A029A9B105361BA
:1017000009B0F0BD39001B7817000C60002BD2D156
:101710002B68019A1C121340A44A9B009B58043565
:10172000ABE7069B3A1DD11A9F4BD82902DD1A223E
:101730001A70C0E738001B7817002A68291D02605C
:10174000002B01D00D00B6E76B68019A1C12134004
:10175000964A9B009B5808358FE7069B3A1DD11A85
:10176000914BD82902DD1A221A70A4E73900A4008F
:101770001B782C1917000C60002B9CD12B68019A48
:101780001C121340894A9B009B58043575E7069B41
:101790003A1DD11A844BD82902DD1A221A708AE721
:1017A00039001700824AA400A2581B780A60002B57
:1017B00000D080E72B68019A1C1213407B4A9B00E3
:1017C0009B58043559E7043F794B3A68A400E2502E
:1017D000754B1B78002B00D06DE72B68019A1C120B
:1017E0001340724A9B009B58043546E7704BA40097
:1017F000E058FFF73BFE6C4B06001B78002B09D12D
:10180000043F3868FFF732FE0123861976001E4335
:10181000674BE650644B1B78002B00D04BE72B68DE
:10182000019A1C121340614A9B009B58043524E71F
:10183000069B391DCA1A5C4BD82A02DD1A221A707F
:1018400039E70698039C0122A04202D222000C3AFA
:10185000126838001B780F000260002B00D02AE7C6
:101860002B68019A1C121340504A9B009B58043568
:1018700003E7069A3B1D991A4B4AD82902DD1A2321
:10188000137018E706990398814219D202000C3AA6
:101890001068484A4010A418241A039AA400A258B9
:1018A0003A601F00404B1B78002B00D003E72B68E9
:1018B000019A1C1213403D4A9B009B580435DCE6FC
:1018C000182111700022EBE7069B039A934219D26C
:1018D00013000C3B1868374B043FE418130040100A
:1018E000241A3A68A400E2502F4B1B78002B00D03A
:1018F000E1E62B68019A1C1213402C4A9B009B586E
:101900000435BAE61822284B1A70EDE7069B039AB5
:10191000934228D2274B043FE61814000C3C23685E
:101920005B10F31A9B009858FFF7A0FD04903868ED
:10193000FFF79CFD2468049B6410341B1E180123D0
:1019400076001E43039BA400E650174B1B78002B28
:1019500000D0B0E62B68019A1C121340134A9B007A
:101960009B58043589E618220F4B1A70EDE7069B49
:101970003A1DD11A0C4BD82902DD1A221A709AE6A8
:1019800039001700039AA400A2581B780A60002BA4
:1019900000D090E62B68019A1C121340034A9B006A
:1019A0009B58043569E6C046AC020020A4D700006D
:1019B0009C2D0020FDFFFF3F043F039B3A68A400DD
:1019C000E250D64B1B78002B00D074E62B68019AAE
:1019D0001C121340D24A9B009B5804354DE6039BD2
:1019E000A4001C192368043F38685E10FFF73EFD11
:1019F0000123361876001E43C84B26601B78002B47
:101A000000D058E62B68019A1C121340C44A9B0070
:101A10009B58043531E6069BA4003F1BBF4CBB42DC
:101A20000CD82378002B00D045E62B68019A1C12B5
:101A30001340BB4A9B009B5804351EE6B94802F090
:101A400069F82378002B00D035E62B68019A1C1228
:101A50001340B34A9B009B5804350EE6A300ED18D3
:101A6000002C00DA3AE6AD4B1B78002B00D022E6C2
:101A70002B68019A1C121340A94A9B009B580435FD
:101A8000FBE5043F3B68042B04D1A300ED18002CB8
:101A900000DA23E6A14B1B78002B00D00BE62B6865
:101AA000019A1C1213409E4A9B009B580435E4E5A2
:101AB000043F3B68042B04D0A300ED18002C00DA8F
:101AC0000CE6964B1B78002B00D0F4E52B68019AAE
:101AD0001C121340924A9B009B580435CDE501230C
:101AE0003E1F306818420AD018410138002809DB2F
:101AF00001234000A40018432D193060EEE5FFF7E4
:101B0000B5FCF2E7854B1B78002B01D03700D2E5FE
:101B10002B68019A1C121340814A9B009B58370086
:101B20000435AAE5FF20610040000140FE38FF387F
:101B30000143396002993B008968241204916D1AAF
:101B40000299AD1089782D020D43854005437D60D3
:101B500006991700039A521A9210824002439A6023
:101B6000029B029A9C70E4B26F4BE400E3589360CE
:101B70006A4A1278002A03D008331D0003979AE5B9
:101B80001D00019A9B680C351C121340644A9B008F
:101B90009B58039771E53B1F1C68039A069B934271
:101BA00032D10A20E30711D4042C18D90F2322685C
:101BB0001340042B16D1200001F0BCFF0AF076FD83
:101BC000C8239B00984200D918000630643004F006
:101BD0000FF800280FD1043D069B03937EE50720F4
:101BE000042CF3D02000431E9841FA234042FF33D7
:101BF00018400730EAE7029B2100587804F0FAFB0E
:101C00000023029A1370E7E7039B039A0C3B1B68BF
:101C100002995B109B00D31A0C3B1C601F1D130024
:101C2000083B1B685A108A70D2B23F49D2005B0051
:101C300055589B0A029A9B009560ED18039B069AE3
:101C4000043B1B685B109B00D3180393334B1B783A
:101C5000002B00D02FE52B68019A1C121340304A4C
:101C60009B009B58043508E53B1F1868FFF7FEFBF7
:101C7000A40006003F1B1E2827DC00280DDC274B94
:101C80001B78002B00D016E52B68019A1C1213401C
:101C9000234A9B009B580435EFE401F083FC033E8C
:101CA000361801F07FFC214B801B9842F9D81B4B62
:101CB0001B78002B00D0FEE42B68019A1C12134005
:101CC000174A9B009B580435D7E40123029A1370EE
:101CD00001F068FC029B0A3886195E60FEE43B1F37
:101CE0001868FFF7C3FBA40006003F1B00280DDCAB
:101CF0000A4B1B78002B00D0DDE42B68019A1C12E4
:101D00001340074A9B009B580435B6E4084B9842A1
:101D100010DD1D22014B1A70CDE4C046AC0200203C
:101D2000A4D70000D0D90000A42500203F420F0016
:101D300080EE36000123029A137001F033FCFA237F
:101D40009B005E430A3E3018029B5860C6E4A30025
:101D5000FF1A002320001A003900FFF7D5FBD74EE9
:101D6000D74C3168200002F005F9D64B3168186075
:101D7000200004F0FFF93168200004F042FBD24B50
:101D80001B78002B00D096E42B68019A1C1213409C
:101D9000CE4A9B009B5804356FE4CB4BA4001B78C4
:101DA0003F1B002B00D086E42B68019A1C121340C5
:101DB000C64A9B009B5804355FE4029803F07CFF01
:101DC000C14B1B78002B00D075E42B68019A1C12C4
:101DD0001340BE4A9B009B5804354EE43B1F1B68D2
:101DE000002B58D13B0001260C3B186806402FD031
:101DF00046103A0001217300083A0B431360002E8D
:101E000000DC95E0012173000B433A1F13603B0097
:101E1000083B1B680B419B1B04933B000C3B186861
:101E200008423BD0049BA4005B188B400B43039AF1
:101E3000A350A54B1B78002B00D03CE42B68019AE3
:101E40001C121340A14A9B009B580435FFF715FC58
:101E500004281BD90F2302681340092B02D14368C1
:101E60005E10C6E7042B08D101F064FE0378002B56
:101E7000BFD0FFF736FA0136F8E7032B06D1160973
:101E8000B6B2520FB6001340F61AB2E719228E4BC3
:101E90001A70FFF710FC5B105E1EB0E7042842D9F1
:101EA0000F2302681340092B05D1049BA4000233C1
:101EB0009B001B58BBE7042B2BD1039BA4001B19D1
:101EC000079301F037FE0600049C0134012C10DC5E
:101ED0003000FFF706FA831B1800049302F03EF867
:101EE000041E0ED001F026FE049A31000AF038F8E4
:101EF00007E03178013C002906D112220C00724B18
:101F00001A70079B1C6094E73000FFF7EAF906009F
:101F1000DCE7032B07D10122049BA400C3181B7923
:101F20005B00134383E71922674B1A70FFF7C3FB6B
:101F300004357EE7A300069AFB189B1AD82B08DD10
:101F40001A22614B1A70FFF7B6FB01221C003A609F
:101F50000437631E002CF8DC5B4B1B78002B01D090
:101F6000FFF7A9FB2B68019A1C121340574A9B00EC
:101F70009B580435FFF781FB069A3B1D9B1A524E76
:101F8000D82B03DD1A233370FFF795FB069B039ACA
:101F9000A40093422AD23B1F1868FFF767FA011E7C
:101FA00021DD039B0C3B1A68521082421BDB900719
:101FB000801A474B4018C018039B8000C2583B1B37
:101FC0001A60414B3F1B1B780437002B01D0FFF7F1
:101FD00072FB2B68019A1C1213403C4A9B009B58D1
:101FE0000435FFF74AFB20233370EAE71823FBE7A9
:101FF000344BA4001A683B1B1F001A60324B043795
:102000001B78002B01D0FFF756FB2B68019A1C129E
:1020100013402E4A9B009B580435FFF72EFB3A1FB6
:102020001368042B02D13A00A4002D19264B1B780B
:10203000002B02D01700FFF73EFB2B6801991C1202
:102040000B4022499B005B5817000435FFF715FB36
:10205000043F3B68042B04D00023A4003B602D19EF
:102060000437194B1B78002B01D0FFF724FB2B689A
:10207000019A1C121340154A9B009B580435FFF728
:10208000FCFAA3009C46F81A002C23DC1C22002634
:102090000D4B1A706346FF1A0B4B06601B78043712
:1020A000002B01D0FFF707FB2B68019A1C1213408D
:1020B000064A9B009B580435FFF7DFFAD005002045
:1020C000AD02002008000020AC020020A4D70000D0
:1020D000FCFFFF3F002103685B1001268A00825845
:1020E000164003D10D22D54B1A70D3E752109342FC
:1020F00000DD130001318C42EFDC5E0001231E4342
:10210000C8E7A3009C46F81A002C17DC1C22002606
:10211000CA4B1A706346FF1AC84B06601B78043717
:10212000002B01D0FFF7C7FA2B68019A1C1213404D
:10213000C34A9B009B580435FFF79FFA00210368B0
:102140005B1001268A008258164003D10D22BB4B3A
:102150001A70DFE75210934200DA130001318C420B
:10216000EFDC5E0001231E43D4E73B000122083B65
:102170001968A40011421DD03B1F1B68134219D0DF
:10218000114113410022994200DA04323B1B1A60CC
:10219000AA4B3F1B1B780437002B01D0FFF78BFAAB
:1021A0002B68019A1C121340A54A9B009B580435CA
:1021B000FFF763FA02203B1F1A684042FFF7A6F8B8
:1021C0003E1B3060E4E73B000120083B1968A40097
:1021D00001421ED03B1F1A6802421AD00141501022
:1021E000CB0FD217884253413A1B9B001360934B8D
:1021F0003F1B1B780437002B01D0FFF75CFA2B68DC
:10220000019A1C1213408E4A9B009B580435FFF71D
:1022100034FA01203B1F1A684042FFF777F83E1B53
:102220003060E4E73B00083B18683B1F1968A600D4
:10223000BE1B0423814202D0042802D8002333604D
:1022400016E001231842F9D10F2302681A40042A2C
:10225000F4D1033A1142F1D10429EFD90A681340AD
:10226000042BEBD1FFF722F9431E98418000306028
:10227000724BA4001B783F1B0437002B01D0FFF7E3
:102280001AFA2B68019A1C1213406D4A9B009B5846
:102290000435FFF7F2F93B00083B18683B1F19684B
:1022A000A600BE1B0023814202D0042802D80423CA
:1022B000336016E001231842F9D10F2302681A4057
:1022C000042AF4D1033A1142F1D10429EFD90A6862
:1022D0001340042BEBD1FFF7E9F84342584180004B
:1022E0003060564BA4001B783F1B0437002B01D0F5
:1022F000FFF7E1F92B68019A1C121340504A9B002A
:102300009B580435FFF7B9F93B000122083B1968D7
:10231000A40011421ED03B1F1B6813421AD05B1051
:102320004A10D80FC9179A4241413B1B89001960D6
:10233000424B3F1B1B780437002B01D0FFF7BBF942
:102340002B68019A1C1213403D4A9B009B58043590
:10235000FFF793F93B1F1A680120FEF7D7FF3E1BDA
:102360003060E5E73B000122083B1968A4001142F8
:102370001DD03B1F1B68134219D01141134100228D
:10238000994200DD04323B1B1A602C4B3F1B1B782B
:102390000437002B01D0FFF78EF92B68019A1C122D
:1023A0001340274A9B009B580435FFF766F93B1FF3
:1023B0001A680220FEF7AAFF3E1B3060E5E73B1FCC
:1023C0001B68A400043B5A1E93413A1B17009B0054
:1023D00013601A4B04371B78002B01D0FFF76BF901
:1023E0002B68019A1C121340154A9B009B58043518
:1023F000FFF743F93B00083B1868FFF737F83B1F2E
:1024000006001868FFF732F80121A4003B1B1F00EB
:10241000321852000A431A60084B04371B78002B0D
:1024200001D0FFF748F92B68019A1C121340044AA7
:102430009B009B580435FFF720F9C046AC020020F2
:10244000A4D700003B00083B1868FFF70FF83B1FBC
:1024500006001868FFF70AF80121A4003B1B1F00C3
:10246000321A52000A431A60E44B04371B78002BDF
:1024700001D0FFF720F92B68019A1C121340E04AA3
:102480009B009B580435FFF7F8F83B00083B1868A1
:10249000FEF7ECFF3B1F06001868FEF7E7FF02009F
:1024A0000121A4003B1B1F00724352000A431A6023
:1024B000D24B04371B78002B01D0FFF7FCF82B68B8
:1024C000019A1C121340CE4A9B009B580435FFF71B
:1024D000D4F83B1F1868FEF7C9FF061E17D11F234B
:1024E000C64A1370A4003B1B1F001E60C34B043779
:1024F0001B78002B01D0FFF7DEF82B68019A1C1225
:102500001340BF4A9B009B580435FFF7B6F83B00C9
:10251000083B1868FEF7AAFF310007F0F9FB01231A
:1025200046001E43DEE73B1F1868FEF79FFF061EAE
:1025300017D11F23B14A1370A4003B1B1F001E605C
:10254000AE4B04371B78002B01D0FFF7B4F82B6893
:10255000019A1C121340AA4A9B009B580435FFF7AE
:102560008CF83B00083B1868FEF780FF310007F04D
:10257000B5FC01234E001E43DEE73B1F1868FEF743
:1025800075FFC11743184B400121A4003A1B1700E7
:102590005B000B431360994B04371B78002B01D071
:1025A000FFF789F82B68019A1C121340944A9B008C
:1025B0009B580435FFF761F8A300FE1A3068012C20
:1025C00025D1FEF753FF01230790049309F0C4FFC0
:1025D0000799002900DC012107F080FC049BA4007E
:1025E000C918012349001943844B3F1B1B783160F4
:1025F0000437002B01D0FFF75EF82B68019A1C12FC
:1026000013407F4A9B009B580435FFF736F8FEF7CE
:102610002DFF04907068FEF729FF049B0130C31A58
:102620000793D3E7A300FE1A31002000049301F0C2
:1026300027FE049B3060FF1A704B04371B78002B79
:1026400001D0FFF738F82B68019A1C1213406C4A2E
:102650009B009B580435FFF710F83B00083B1868B7
:10266000FEF704FF3B1F06001868FEF7FFFE02009E
:102670000121A4003B1B1F00324052000A431A6094
:102680005E4B04371B78002B01D0FFF714F82B6842
:10269000019A1C1213405A4A9B009B580435FEF7BE
:1026A000ECFF3B00083B1868FEF7E0FE06003B1F0E
:1026B0001868FEF7DBFE32000121A4003B1B1F005F
:1026C000024352000A431A604C4B04371B78002B1C
:1026D00001D0FEF7F0FF2B68019A1C121340484A04
:1026E0009B009B580435FEF7C8FF3B00083B186869
:1026F000FEF7BCFE06003B1F1868FEF7B7FE32006F
:102700000121A4003B1B1F00424052000A431A60F3
:102710003A4B04371B78002B01D0FEF7CCFF2B6817
:10272000019A1C121340364A9B009B580435FEF751
:10273000A4FF3B1F1868FEF799FEC3430121A400C4
:102740003A1B17005B000B4313602C4B04371B78BC
:10275000002B01D0FEF7AFFF2B68019A1C1213402B
:10276000274A9B009B580435FEF787FF3B00083B38
:102770001868FEF77BFE06003B1F1868FEF776FE22
:10278000320082400121A4003B1B1F0052000A437B
:102790001A601A4B04371B78002B01D0FEF78BFF11
:1027A0002B68019A1C121340154A9B009B58043554
:1027B000FEF763FF3B00083B1868FEF757FE060074
:1027C0003B1F1868FEF752FE320002410121A400AF
:1027D0003B1B1F0052000A431A60084B04371B784A
:1027E000002B01D0FEF767FF2B68019A1C121340E3
:1027F000034A9B009B580435FEF73FFFAC020020C4
:10280000A4D700003B000C3B1868FEF72FFE3B00EE
:10281000083B06001868FEF729FEF1170200C317EF
:10282000300007F0ADFB3B1F049005911868FEF7E0
:102830001DFE02000498059907F056FB0123A40031
:102840003E1B370040001843E54B30601B780437CF
:10285000002B01D0FEF72FFF2B68019A1C121340AA
:10286000E04A9B009B580435FEF707FFA300FE1AC1
:10287000310020000493FEF78DFB049B3060FF1AAB
:10288000D74B04371B78002B01D0FEF714FF2B68C1
:10289000019A1C121340D34A9B009B580435FEF743
:1028A000ECFEA300FF1A39002000FEF78BFBCC4B97
:1028B0001B78002B01D0FEF7FEFE2B68019A1C123C
:1028C0001340C84A9B009B580435FEF7D6FEA30070
:1028D000FE1A310020000493FEF7B4FB049B306025
:1028E000FF1ABF4B04371B78002B01D0FEF7E3FE25
:1028F0002B68019A1C121340BA4A9B009B5804355E
:10290000FEF7BBFEA300FF1A39002000FEF71EFCF5
:10291000B34B1B78002B01D0FEF7CDFE2B68019A3C
:102920001C121340AF4A9B009B580435FEF7A5FECE
:10293000A300FE1A310020000493FEF779FC049BEB
:102940003060FF1AA64B04371B78002B01D0FEF72E
:10295000B2FE2B68019A1C121340A24A9B009B589E
:102960000435FEF78AFE3B1F186801F0E3F83A00D1
:102970000121083A12680300A4000A4229D1042A5E
:102980000CD910680F221040013808280FD807F022
:102990002BF9052026220E0E0E0E24009249180057
:1029A00009F07AFE434258413B1B800018608C4B73
:1029B0003F1B1B780437002B01D0FEF77CFE2B68F1
:1029C000019A1C121340874A9B009B580435FEF75E
:1029D00054FE8649E3E78649E1E78649DFE7864911
:1029E000DDE7069B3E1DF31A7D4CD82B03DD1A2331
:1029F0002370FEF760FE00F0DFFD01223B00400087
:102A00001043186023783700002B01D0FEF753FEE7
:102A10002B68019A1C121340724A9B009B58043584
:102A2000FEF72BFE069B3E1DF31A6D4CD82B03DDE3
:102A30001A232370FEF73FFE00F0B4FD6F4A4000FA
:102A4000104001223B001043186023783700002B10
:102A500001D0FEF730FE2B68019A1C121340614A28
:102A60009B009B580435FEF708FE069A3B1D9B1AF7
:102A70005B4CD82B03DD1A232370FEF71CFE00F0FD
:102A80009BFD5F4B1A68831A904201D25D4A9B18E6
:102A900001213A005B000B43136023780437002BBD
:102AA00001D0FEF708FE2B68019A1C1213404D4A14
:102AB0009B009B580435FEF7E0FD00F07DFD504B78
:102AC000A4001860464B3F1B1B78002B01D0FEF77B
:102AD000F2FD2B68019A1C121340424A9B009B583E
:102AE0000435FEF7CAFD00F075FDA300002810D1E3
:102AF000FF1A3B4B1B78002B01D0FEF7DCFD2B6847
:102B0000019A1C121340374A9B009B580435FEF76C
:102B1000B4FD3E00FF1A012320001A003900FEF721
:102B2000F3FC394C2068643003F062F8002803D1CC
:102B3000043D3700FEF7D2FD029B21685A783348E6
:102B400003F071FC0123029A137000F02BFD304B4F
:102B500022681B68063253431818FFF7F5F800F097
:102B600039FDA300002810D1FF1A1D4B1B78002B44
:102B700001D0FEF7A0FD2B68019A1C121340194AE0
:102B80009B009B580435FEF778FD3E00FF1A20009D
:102B9000012300223900FEF7B7FC1B4C206864308B
:102BA00003F026F80028C3D0184803F0CDF9C9E790
:102BB000A4003E1BFEF728FD3700094B30601B7850
:102BC0000437002B01D0FEF776FD2B68019A1C120A
:102BD0001340044A9B009B580435FEF74EFDC04647
:102BE000AC020020A4D70000E0D90000E8D9000022
:102BF000EFD90000F6D90000FBD90000FEFFFF7FEF
:102C0000D805002037894100D0050020AD02002002
:102C100004000020FB4BA4001B783F1B002B01D0BD
:102C2000FEF749FD2B68019A1C121340F64A9B00DF
:102C30009B580435FEF721FDA4003E1B300000F038
:102C4000F6FC3700EF4B30601B780437002B01D0C7
:102C5000FEF731FD2B68019A1C121340EA4A9B00D3
:102C60009B580435FEF709FDA4003E1B300000F020
:102C7000E0FC3700E34B30601B780437002B01D0B9
:102C8000FEF719FD2B68019A1C121340DE4A9B00C7
:102C90009B580435FEF7F1FCA300FE1A310020001A
:102CA000049300F0C9FC049B3060FF1AD54B043735
:102CB0001B78002B01D0FEF7FEFC2B68019A1C123A
:102CC0001340D14A9B009B580435FEF7D6FCA40064
:102CD0003F1B380000F0E6FCCA4B1B78002B01D0EC
:102CE000FEF7E9FC2B68019A1C121340C64A9B00B0
:102CF0009B580435FEF7C1FCA300FE1A31002000EA
:102D0000049300F0F7FC049B3060FF1ABD4B0437BE
:102D10001B78002B01D0FEF7CEFC2B68019A1C1209
:102D20001340B94A9B009B580435FEF7A6FCA4004B
:102D30003F1B380000F020FDB24B1B78002B01D068
:102D4000FEF7B9FC2B68019A1C121340AE4A9B0097
:102D50009B580435FEF791FC0121200000F0F4FCA3
:102D6000A84B1B78002B01D0FEF7A5FC2B68019A1D
:102D70001C121340A44A9B009B580435FEF77DFCAF
:102D80000021200000F0E0FC9E4B1B78002B01D0BE
:102D9000FEF791FC2B68019A1C1213409A4A9B0083
:102DA0009B580435FEF769FCA4003E1B300000F080
:102DB00005FD3700934B30601B780437002B01D0A2
:102DC000FEF779FC2B68019A1C1213408E4A9B0077
:102DD0009B580435FEF751FCA4003E1B300000F068
:102DE00001FD3700874B30601B780437002B01D082
:102DF000FEF761FC2B68019A1C121340824A9B006B
:102E00009B580435FEF739FCA4003F1B380000F046
:102E1000C3FC7C4B1B78002B01D0FEF74CFC2B68CD
:102E2000019A1C121340784A9B009B580435FEF708
:102E300024FCA4003F1B380003F004FF714B1B78F7
:102E4000002B01D0FEF737FC2B68019A1C121340AF
:102E50006D4A9B009B580435FEF70FFCA4003E1BF7
:102E6000300003F0C9FF3700664B30601B78043731
:102E7000002B01D0FEF71FFC2B68019A1C12134097
:102E8000614A9B009B580435FEF7F7FBA4003F1BEB
:102E9000380003F053FE5B4B1B78002B01D0FEF78C
:102EA0000AFC2B68019A1C121340574A9B009B583E
:102EB0000435FEF7E2FBA4003E1B300003F058FE91
:102EC0003700504B30601B780437002B01D0FEF7E1
:102ED000F2FB2B68019A1C1213404B4A9B009B5833
:102EE0000435FEF7CAFBA300FF1A3900200001F0E9
:102EF00029FD444B1B78002B01D0FEF7DCFB2B682F
:102F0000019A1C121340404A9B009B580435FEF75F
:102F1000B4FBA300FF1A3900200001F027FB394B56
:102F20001B78002B01D0FEF7C6FB2B68019A1C1200
:102F30001340354A9B009B580435FEF79EFBA300C7
:102F4000FF1A3900200001F035FC2E4B1B78002BB6
:102F500001D0FEF7B0FB2B68019A1C1213402A4ADD
:102F60009B009B580435FEF788FBA300FF1A39002D
:102F7000200001F047FC234B1B78002B01D0FEF70B
:102F80009AFB2B68019A1C1213401F4A9B009B5806
:102F90000435FEF772FBA300FE1A310020000493F3
:102FA00003F09AFF049B3060FF1A164B04371B781E
:102FB000002B01D0FEF77FFB2B68019A1C121340F7
:102FC000114A9B009B580435FEF757FBA300FE1ADD
:102FD00031002000049303F087FF049B3060FF1A48
:102FE000084B04371B78002B01D0FEF764FB2B68DD
:102FF000019A1C121340044A9B009B580435FEF7AB
:103000003CFBC046AC020020A4D70000A300FE1A7F
:1030100031002000049303F06FFF049B3060FF1A1F
:10302000984B04371B78002B01D0FEF744FB2B682C
:10303000019A1C121340944A9B009B580435FEF7DA
:103040001CFBA300FE1A31002000049303F05CFF78
:10305000049B3060FF1A8B4B04371B78002B01D088
:10306000FEF729FB2B68019A1C121340864A9B002D
:103070009B580435FEF701FBA300FF1A390020001E
:1030800001F0ACFA7F4B1B78002B01D0FEF713FB4D
:103090002B68019A1C1213407B4A9B009B580435F5
:1030A000FEF7EBFAA300FF1A3900200001F0D2FB73
:1030B000744B1B78002B01D0FEF7FDFA2B68019AA8
:1030C0001C121340704A9B009B580435FEF7D5FA3A
:1030D000A300FE1A31002000049301F037FB049B8B
:1030E0003060FF1A674B04371B78002B01D0FEF7C6
:1030F000E2FA2B68019A1C121340634A9B009B580A
:103100000435FEF7BAFAA300FF1A3900200001F0D7
:10311000E5FA5C4B1B78002B01D0FEF7CCFA2B684C
:10312000019A1C121340584A9B009B580435FEF725
:10313000A4FA002C55DD3B1F1E68012C0CD1264241
:1031400007D1042E05D90F23326830001340042B19
:1031500011D00120404212E0022CFAD13B00083B82
:10316000186801231842F4D10428F2D902680E33FA
:103170001340042BEDD100F0DDFCFEF71FF9A30096
:10318000FF1A00282DDB0022022C11D1012333402D
:10319000934222D1042E20D931680F320A40092AE5
:1031A0001BD172685210D2B29100994210D17F188F
:1031B0000002104304003A00069B0C32D31AD82BAD
:1031C00001DCFEF7AFFC1A222E4B1A70FEF773FAE1
:1031D000F418A468FC500433E7E73E60012204378A
:1031E000E6E700233B60274B3A1D1B78002B02D0FB
:1031F0001700FEF760FA2B6801991C120B40224958
:103200009B005B5817000435FEF737FA069B029ABD
:10321000FB1A9B101361A300FF1A3900200002F073
:10322000D1FE184B1B78002B01D0FEF744FA2B6817
:10323000019A1C121340144A9B009B580435FEF758
:103240001CFA069B029AFB1A9B101361A300FE1A3C
:1032500031002000049302F0B5FE049B3060FF1A99
:10326000084B04371B78002B01D0FEF724FA2B689B
:10327000019A1C121340044A9B009B580435FEF728
:10328000FCF9C046AC020020A4D700000023F7B52B
:103290005A1E0192002B07DA01F06AFB02F0AAFF26
:1032A00003F020F91923019300263000194B196807
:1032B000B14212DD184B1A6801328A420FDAF0244B
:1032C0001A601D68154F6C43E35D002B1FD0E41995
:1032D000022B06D12000FEF7AFF9019BD8E70022B0
:1032E000EDE7012B0DD1002801D100F05BF9F022B0
:1032F0006A43BB185B680A49C31A8B4201D8022390
:10330000BB54F0235D43054BEB5C022BE2D001364E
:10331000CCE7C046D405002000000020441C00205B
:103320003F420F0080220B4B52001A600121A8225D
:10333000A920094BD20019649A58C00005321A50CE
:1033400006481A50C122C020920000039850044B36
:103350001970704700E100E0008000404C0500005B
:10336000FD05002004207047F8B550C90123220054
:103370001A40101E2DD03340181E2AD06410002091
:103380001A2C26D81D4B761035009E4200DD1D00FC
:103390001B4F3B5D012B05D00121200005F014F8E7
:1033A00001233B55174B1B78002B01D1FFF7BAFFC8
:1033B0000023154A9E420DDCFF2514491448D65CB3
:1033C000B44202D15E007052D5540133042BF6D1C1
:1033D0000420F8BDD15C8C4203D10C4A5B009D52A5
:1033E000F6E70133042BF5D10023D15CFF2901D18D
:1033F000D454F2E70133042BF7D1E9E78813000036
:10340000E0050020FD0500201C0000200E0000202B
:10341000DC05000070B530C9012322001A40101EDF
:103420001BD02B40181E18D064101A2C00D9192458
:10343000154E335D012B05D00121200004F0C4FF9F
:103440000123335569100800104A1038104B904280
:1034500004D9012252421A60042070BD1C600D483C
:1034600006F056FC0C4B040018800C4B1B78002B0C
:1034700001D1FFF757FF0122094B9A64A922D2001C
:10348000995864189C50E7E7E005002090860100F9
:103490001800002020A107000C000020FD050020DE
:1034A00000800040F8B501260D683400B04200DD10
:1034B0004C682B003340181E0BD023003340181EDD
:1034C00007D06D10002D05DCA12300201E4ADB0073
:1034D000D650F8BD641000201A2CFAD81B4F3B5D63
:1034E000012B04D00121200004F06EFF3E5529007D
:1034F000174806F00DFC0A21053006F009FC154BB3
:10350000A400E258144B12021343A2221349D20022
:103510008B50134C0C4B9C50124C195101241249E6
:103520005C50124B196900219950114A904200DDFC
:103530001000A8228021D2009850012289005A5000
:1035400004201A60C5E7C04600F00140E0050020F5
:1035500000B4C404A8EA00000300030000600040B7
:1035600040A10040140500000405000000A0004038
:10357000FFFF0000030010B50120002B02DC1B3010
:10358000FEF73CF810BD0420704710B5002803DC9E
:103590001C20FEF733F810BD0B680020DB07FAD4BF
:1035A0000D30F6E70122034B1A64A822D200985886
:1035B0007047C046008000400122054B10B51A64D8
:1035C000A822FA21D2009858890006F017FB10BDF6
:1035D00000800040012070470048704768DA000012
:1035E0001B20704770B5054E0400335C0D008B4204
:1035F00002D004F0E9FE355570BDC046E00500205C
:1036000070B50024084D635D012B09D10021200015
:1036100004F0F8FE0021200004F0D6FE00236355DC
:1036200001341B2CEED170BDE00500207047112045
:103630007047372070470000F8B501240B6806007A
:103640000D00234204D10D20FDF7D8FF2000F8BD66
:103650005B1004D103F09EFA40002043F7E72000FE
:10366000072BF4D80D4A9B009C580D4F3B5D002B57
:1036700005D00021200004F0A7FE00233B55012EB9
:1036800006DD6B68042B03D10221200004F09CFEB0
:10369000200004F047FD01244000DEE748DA000086
:1036A000E0050020F8B501260568354202D04468DF
:1036B000344203D10D20FDF7A1FFF8BD6D101A2D86
:1036C000FBD80A4F7B5D012B04D03100280004F0A9
:1036D0007BFE7E55064964108C4202DCE143C9172B
:1036E0002140280004F0A4FDE7E7C046E0050020E3
:1036F000FF03000070B501240D68254204D10D20A0
:10370000FDF77CFF200070BD6D101A2D17D8002426
:10371000012804DD4C68043C63425C416400094EAE
:10372000735DA34204D02100280004F04DFE7455BF
:10373000280004F07DFE03000420012BE3D00020CC
:10374000E1E7C046E005002070B504000D001A282E
:103750000ED8084E335C012B04D0012104F034FE56
:1037600001233355290020004D1EA94104F04AFED3
:1037700070BDC046E0050020036810B5DA0703D429
:103780000D20FDF73BFF10BD4168581004394A4237
:103790005141FFF7D9FFF6E737B569460A00064BF6
:1037A00030CB30C203680220042B02D101F002F8B2
:1037B00037BD01F027F8FBE708DA000010B5084C28
:1037C000237D002B05D00021142004F0FDFD0023F3
:1037D0002375142004F02CFE43425841800010BD94
:1037E000E005002010B5084CA37D002B05D000217A
:1037F000162004F0E9FD0023A375162004F018FE3E
:1038000043425841800010BDE0050020A022002363
:103810000349D2008B50034910328B507047C04689
:1038200000F0014000600040F7B52F4D2F4EEB6CCB
:10383000002B14D0A9240023E4003759EB642C4B4F
:10384000186800280BDB2B4B19784A425141C9B24A
:10385000197004F0D7FD284B1B88DF1937512B6DE9
:10386000002B38D00021254B254FF45829653A7894
:103870000193244D8A4206D02B68032B03D8224A99
:10388000D05C04F0BFFD2B68204A0133134004D5FF
:103890000422013B5242134301331B4900228C4650
:1038A0002B60042B18D06046C05C591CFF2802D145
:1038B0000B000122F5E7002A00D02B60012104F063
:1038C000A1FD01233B702B68114A5B009B5A0C340D
:1038D000E418019BF450F7BD01235B422B600023E9
:1038E0003B700C4BF4E7C046FC8000400080004079
:1038F00018000020FC0500200C0000204C050000F2
:10390000FB050020DC0500201C00002003000080D7
:103910000E0000205C460000084B094AFF201A8078
:103920005A809A80DA800023064A07491370074AB2
:10393000087048708870C870136070470E000020CF
:10394000DC050000FB0500201C000020DC05002039
:103950000122024B52421A607047C04618000020F4
:1039600010B5034A0721034802F0D2F810BDC04643
:1039700010DA000016E20000E12170B54902194892
:1039800004F046F9002401220320174B17491A615D
:103990005C50043158508018083158501A60063075
:1039A00004F0BAFBFF21124AA15401341B2CFBD1B5
:1039B000012200200F4B01001A6004230E4A0F4D14
:1039C0001468002CFCD02C680002013B20431160DD
:1039D000002BF5D101220A4B1A6004F0D5FA01F050
:1039E00013F970BDCC1B00200080004004050000CE
:1039F000E005002000D0004000D1004008D5004084
:103A000004D00040F8B50B4E070030000D0004F064
:103A100047F90400A84200DD2C003D00EB1B9C424E
:103A200005DD300004F046F928700135F6E7200086
:103A3000F8BDC046CC1B002010B50100014804F0C1
:103A4000EFF810BDCC1B002010B5054C200004F091
:103A5000F5F8E1212000490204F0DAF810BDC04673
:103A6000CC1B0020C3070CD4064B1B68834208D82C
:103A7000054B1B68984204D8031F1B68002B00D01D
:103A800018007047080600200406002000230122C9
:103A900010B50A48990001334250642BFAD1084C02
:103AA000084B00211A602000074A08F075FA074BFE
:103AB000074A6360074B1A6010BDC0469C2D00206A
:103AC0000C06002008000020D40900003027000068
:103AD000100600200006002010B5044B044A1A60AE
:103AE000044B054A1A60FFF7D1FF10BD08060020FD
:103AF0000C06002004060020E00F0020044B1B6889
:103B00001868000980B20238C343DB1718407047B9
:103B10000006002000B59BB00200054901A808F08E
:103B20007FFD01A802F02CFA02F0DCFCFCE7C046A5
:103B3000F6DA00000B4BC20704D4042804D80A4B61
:103B400000D00A4B180070470F2203681A40031D6B
:103B5000042AF7D0064B092AF4D0064B032AF1D0E9
:103B6000054BEFE7D0DA00004AD6000044D600004B
:103B7000DADA0000EADA0000E1DA00000020064AA2
:103B80000649131F186013681B099BB202339B0080
:103B9000D2188A42F5D3704710060020E00F0020AB
:103BA000F7B50F240126314B314A1968314B324D9C
:103BB000186813681F002740072F26D813681B09B1
:103BC0009BB202339B00D218AA42F2D300242B4EA0
:103BD000A500AD192868FFF745FF01342860642C63
:103BE000F6D1274C2068FFF73DFF2060254C206868
:103BF000002802D0FFF736FF20600025224B1B680B
:103C00000093009B9D4214DBF7BD1B099BB29B00F8
:103C1000D3189A42D2D01F68374208D1B94206D28F
:103C2000B84204D3043F3F68002F00D01F60043B1C
:103C3000EFE7F0236B43154A9B181A78002A01D14D
:103C40000135DEE71F693C2300266B43DB199B002F
:103C500001930136BB1BF3D4019BB4001C1B0B4B1F
:103C60001C19A069FFF7FEFEA061F2E7080600201C
:103C70001006002004060020E00F00209C2D0020EC
:103C800008000020E00F0020D4050020441C002084
:103C9000F7B50124204246D1234B1B689C4698422D
:103CA00041D3224B1B68019398423CD8031F1B68E9
:103CB000002B38D10200036800941B099BB2002B33
:103CC0000FD10099131F196090422CD015682B1F3B
:103CD0001B68990069180C68013B14600A602A008F
:103CE000EDE79D0055192968009C214219D18C45AA
:103CF00017D8019C8C4214D30E1F3468002C10D1AD
:103D00000F680F343C40072C08D92F60151F2B601B
:103D10000B680A601B099BB20A00D0E7009931606A
:103D2000CDE7013BCBE7F7BD0806002004060020E5
:103D30000D4970B50A000D4D1368141F1B09266844
:103D40009BB2981C002E0BD000238A4200D00B009F
:103D500023608300C91880001218AA42ECD370BDFA
:103D60001B011360F7E7C04610060020E00F00209B
:103D7000F8B5124C27000F223B681D09ADB2134263
:103D80000DD06E1CB600A74204D0320039002000CE
:103D900008F0EFF80022A3190436A4191A600235BE
:103DA000AD00074B7F199F42E5D31B1B9B10013BC6
:103DB0001B012360034B1C60F8BDC04610060020A9
:103DC000E00F002000060020F0B59BB0FFF7EAFBF3
:103DD00000240700214AA300D0580134FFF758FF00
:103DE000642CF7D11E4B1868FFF752FF1D4B186863
:103DF000002801D0FFF74CFF00261B4B1B689E429A
:103E000017DBFFF795FFFFF7CBFEFFF7B1FFFFF7DB
:103E1000C9FB164BC21B1B6815491B6801A81B096F
:103E20009BB2023B08F0FCFB01A802F0A9F81BB012
:103E3000F0BDF02575430F4BED182B78002B01D109
:103E40000136DAE72B695C1E002CF9DBA300EB18C6
:103E50009869FFF71DFF013CF6E7C0469C2D002046
:103E600008000020E00F0020D405002000060020FC
:103E7000B0DA0000441C0020F7B5174D4F1C2B682A
:103E800006001B680C001B099BB201929F420BDBD2
:103E9000FFF79AFF2B681B681B099BB29F4203DB4D
:103EA0000A20FDF7ABFBFEBD2868A71CBA00DB1B90
:103EB00081181B010B6029600021031F19600F236B
:103EC0001E4003002401264340C3083A9A189A4230
:103ED000E9D9019902C3FAE700060020F7B503000B
:103EE0000122134004000D000193002B2BD1174B2E
:103EF0001B68834227D8164B1B68834223D90F23A4
:103F0000144F386000681840FFF7B6FF019B3C680B
:103F1000061E3B6017D0236804301B099BB29D42EC
:103F200000DD1D00AA00211D251F08F019F8FFF76C
:103F300025FE2E60FFF734FE00232B602268064B1F
:103F40001340236034002000FEBDC0460806002058
:103F500004060020E00F0020F0FF0F0003230430D0
:103F600010B5C11719400918891000220420FFF765
:103F700083FF10BD70B5050008000C00FFF7EEFFD1
:103F80000023002804D170BDE95CC218117101330F
:103F9000A342F9DBE343DB171C4000230419237120
:103FA000F1E7F0B50C009BB0022804DC1C20FDF703
:103FB00025FB1BB0F0BD01230868184206D1042878
:103FC00004D90F2601683140042901D00E20EEE704
:103FD00061680D001D40F9D10429F7D90A68324003
:103FE000042AF3D1A2681A4201D10D20DFE7FFF7BE
:103FF000A1FD06006068FFF79DFDA768010001AC08
:104000007F103000257003F02DFA39006423220060
:1040100003F08DFA200008F049FB01002000FFF7B3
:10402000A9FFC6E710B51C4CA544041E02D1FFF73A
:1040300095FF0BE003F02EF90138062828D805F08B
:10404000D3FD090911182904240000208023DB0076
:104050009D4410BD200003F099F9011B2000FFF7DB
:1040600089FFF3E7200003F03FF9430001201843E4
:10407000ECE780226946D200200003F04CF9684644
:1040800008F014FB01006846E9E704210348E6E76D
:104090000020CCE70420D9E700FCFFFF3CDB000058
:1040A00070B50C00022803DC1C20FDF7A7FA70BDD8
:1040B00001230868184206D1042804D90F25016895
:1040C0002940042901D00E20EFE761681942FAD196
:1040D0000429F8D90A682A40042AF4D1A2681A42AD
:1040E00001D10D20E1E7FFF725FD05006068FFF72E
:1040F00021FDA46801006410280003F0B3F9210039
:1041000003F0F0F9FFF78EFFD1E770B50D0001283D
:1041100003DC1C20FDF772FA70BD01240868204200
:1041200006D1042804D90F2102680A40042A01D0CC
:104130000E20EFE76A682242FAD1042AF8D9136800
:104140000B40042BF4D1FFF7F5FC06006868FFF77D
:10415000F1FC0100300003F085F903F007FA40009C
:104160002043D9E7F8B507000C001C20012F0BDD18
:1041700001250868284206D1042804D90F210268C5
:104180000A40042A03D00E20FDF738FAF8BD626811
:104190002A42F8D1042AF6D913680B40042BF2D135
:1041A000FFF7C8FC06006068FFF7C4FC0100022F9F
:1041B00014D0A4682C4211D06410300003F052F9DE
:1041C000050003F067F8012811D1002C02DD01354C
:1041D000012C06D12800FFF725FFD7E70124644210
:1041E000EBE7280003F0DFF8013C0500F0E70228C8
:1041F000F0D1002CEEDD0135012CEBD0002228009F
:10420000110003F002F903F0CEF8013C0500F3E7DA
:1042100010B501240868044016D04410200006F0B0
:104220000BF8154905F0D6FE07F0BCFD04F00EFAB8
:104230000022124B06F070FF04F0B0F907F042FDC7
:1042400043000120184310BD042810D90F23026831
:104250001340042B07D1FFF76DFC21000A2208F060
:10426000EDFA0400DAE7032B01D10430F5E70D2065
:10427000FDF7C4F9D2E7C046D30237390000D04079
:10428000086870B501240500254006D1042804D92A
:104290000F2302681340042B03D00E20FDF7AEF964
:1042A00070BDFFF747FC03782900233B5A42534176
:1042B0001022C01808F0C2FA80239B05C218044BD4
:1042C0009A4201D91420E9E740002043E8E7C046BC
:1042D000FFFFFF3F10B5034A0621034801F018FC19
:1042E00010BDC0460CDB000007DB0000002070475B
:1042F00010B51E20FDF782F910BD10B51E20FDF788
:104300007DF910BD10B51E20FDF778F910BD10B570
:104310001E20FDF773F910BD10B51E20FDF76EF9D4
:1043200010BD10B51E20FDF769F910BD10B51E2097
:10433000FDF764F910BD10B51E20FDF75FF910BD43
:1043400010B51E20FDF75AF910BD10B51E20FDF75F
:1043500055F910BD10B51E20FDF750F910BD10B570
:104360001E20FDF74BF910BD10B51E20FDF746F9D4
:1043700010BD10B51E20FDF741F910BD10B51E206F
:10438000FDF73CF910BD10B51E20FDF737F910BD43
:1043900010B5034A1121034801F0BAFB10BDC04615
:1043A00078DB000000DC00000120034B1860034BA9
:1043B0001B6883401843704704100020E40F00205E
:1043C000F0B5EFF310810123194083F31088134CEB
:1043D000134AA4461268134E013A9340124F134AEF
:1043E000002B17D0146803420FD03D682C60C046E4
:1043F000C046C046C046C046C046C046C0460C4C3B
:104400001568246825605B08EAE765462C60146837
:104410003460F8E781F31088F0BDC046080500500D
:10442000200000200C050050F00F0020F80F0020A5
:10443000EC0F002030B585B001AD0C2206492800F4
:1044400007F08EFD0024285D01210134FFF7CAF832
:104450000C2CF8D105B030BDE9DC0000F7B56A4698
:104460003B4B01AE1380062393703A4B33800F23EE
:10447000B370FFF797F8384B384DC0182B68984247
:1044800001D200232B602C68002C41D1375D012123
:104490003800FFF7A7F801340021380003F0B2FF1D
:1044A000032CF3D1002401276B461E5D3900300038
:1044B000FFF798F801343900300003F0A3FF032C14
:1044C000F2D1C8200138C046C046C046C046C046EA
:1044D000C046C046C046C046C046C046C046F1D1F0
:1044E0006B4600211878FFF77DF86B46002158785D
:1044F000FFF778F86B4600219878FFF773F8FFF71D
:1045000051F8FA2300241B01C01828602000FEBDCA
:10451000FFF748F82B6800249842F7D3042003F0F3
:1045200001FE0600052003F0FDFD3618062003F00D
:10453000F9FD0B4B9B1B181A0A4BA04206DB1860B7
:104540000023094A2B6013600124DFE71C60F7E7B2
:10455000040500000D0E000010270000FC0F0020D5
:1045600043030000E40F0020041000200022054B4C
:1045700010B51A60044B1B68934201D002F02AFE6A
:10458000002010BD00100020F01A002010B5041EFD
:1045900010DA1A240A4BA400E25801239340094A76
:1045A00009491360094A1160094A0A4911600A4A17
:1045B000136010BDFFF714F8A042EADDEAE7C04639
:1045C000A8EA0000F80F002008050050F00F0020B6
:1045D000EC0F00200C05005018050050F0B53B4BC7
:1045E00085B01B680C00002B03D101204042FFF76F
:1045F000CDFF246801222700174028D0FF23601236
:10460000184033496714661040431F401E4005F0B0
:104610007FFB050438002E49784305F079FB000242
:10462000054330002A49704305F072FB294B2843AB
:104630001B68202B06D16400A40E274BA400E3586E
:1046400000021843FFF7BCFE002005B0F0BD042CAB
:10465000FAD90F2321680B40092BF5D16368039227
:104660005B100193019B9F42EEDABB00E3189E684A
:10467000039B1E4228D0FF237012184072101A406C
:104680001349751440431D40009205F041FB03049B
:1046900028000F496843029305F03AFB029D00028F
:1046A000054300980A49404305F032FB094B284373
:1046B0001B68202B06D17600B60E074BB600F558C6
:1046C00000022843FFF77CFE0137CBE7F80F0020FC
:1046D0005906000020000020D0DE0000020008681B
:1046E00010B5C3070FD540101823012A03DD4A680F
:1046F000042A00D10833054A1360FEF797FFFFF73D
:1047000045FF002010BD01204042EDE720000020C1
:1047100010B50124044002D04410200010BD04282C
:1047200010D90F2302681340042B07D1FFF702FAB8
:1047300021000A2208F082F80400EEE7032B01D1E1
:104740000430F5E70D20FCF759FFE6E70868F8B5F7
:10475000C3071AD5FFF7DCFF0300203B5E2B25D8EB
:104760000520434301221D180020114E9D4219D0FF
:1047700005211024F75C3C4200D08018013952001A
:1047800064100029F7D10133F0E704280ED90F2275
:1047900003681A40042A09D11B099BB2002B05D0DB
:1047A0000379DAE7012340001843F8BD0120FCE754
:1047B000F5DC000070B508680D00FFF7A9FF0400E4
:1047C0006868FFF7A5FF621E0100042A14D8451E81
:1047D000042D11D805236B439B18012215009D4021
:1047E0002B00064805682B430360054B1B68002B14
:1047F00002D0200002F0EFFC002070BD001000206D
:10480000F01A002070B508680D00FFF781FF040062
:104810006868FFF77DFF621E0100042A13D8451E59
:10482000042D10D805236B439B1801229A4007489A
:10483000036893430360064B1B68002B03D00022E0
:10484000200002F0C8FC002070BDC046001000200F
:10485000F01A0020F0B5050089B008680C00FFF7D9
:1048600057FF0690022D36DD6068FFF751FF01907B
:10487000A068FFF74DFF04000127231D661E079364
:10488000731C0293079B9E4235D005237343059307
:10489000019B019D05330493049BAB421ED0042E63
:1048A00016D86B1E042B13D80122059B2349013B0C
:1048B0005B199A409446224A0B681068069A3A405F
:1048C00003920DD062461A430A60012200280DD1DE
:1048D0007F000135E0E701240194CDE7029ECFE798
:1048E000624693430B600028F2D0039A0299280095
:1048F00002F071FCECE7019B1E1D042E1AD8012C5E
:1049000018D1002505273B0021006B439B199940D6
:104910000B000A4A013511689943094B11601B6865
:10492000002B05D0019B0022581D290002F053FCEA
:10493000052DE8D1002009B0F0BDC04600100020D0
:10494000F01A0020086810B5C30703D5FFF7E0FE92
:10495000054B1860054B1B68002B03D0024B1868F1
:1049600002F03AFC002010BD00100020F01A0020D8
:104970007FB5A04C2368002B0AD19F4A1268002AF9
:1049800006D19E4B1B68002B01D0FFF767FD7FBD52
:104990009B4D2A68002A26D1984A1268002A1BD00B
:1049A000FFF75CFD0028F2D0FFF744FD924B24682E
:1049B0001A681C60002A16D0002C14D101AD0C22FC
:1049C0009049280007F0CCFA285D00210134FEF759
:1049D00009FE0C2CF8D1DAE7874A1268002AE5D1E3
:1049E000002BE3D0E0E700210D2003F00BFD0021B8
:1049F0000E2003F007FD00210F2003F003FD2E68B9
:104A0000012E5DD0022E00D1A2E0002E51D1013640
:104A10003100794C04202368994303F0F3FC04210E
:104A20002368052019404B42594103F0EBFC10214B
:104A30002368062019404B42594103F0E3FC8021D2
:104A40002368090119404B4259410C2003F0DAFC5C
:104A500080212368090219404B4259410B2003F081
:104A6000D1FC80212368490219404B4259410A2058
:104A700003F0C8FC80212368890219404B42594148
:104A8000092003F0BFFC80212368C90219404B4272
:104A90005941082003F0B6FC802321681B0319400C
:104AA0004B425941072003F0ADFC31000D2003F0CB
:104AB000A9FC2B680321581C05F010FA296066E751
:104AC00002214D4C0720236819404B42594103F005
:104AD00099FC0820216801404B42594103F092FCA7
:104AE00080212368C90019404B425941052003F039
:104AF00089FC80212368490119404B425941062015
:104B000003F080FC80212368C90119404B425941C0
:104B1000042003F077FC80212368890319404B426D
:104B200059410A2003F06EFC802321681B041940C0
:104B30004B425941092003F065FC31000C2003F081
:104B400061FC31000B2003F05DFC31000E20AEE76C
:104B50002021294C0720236819404B42594103F07A
:104B600051FC40212368082019404B42594103F071
:104B700049FC80212368092019404B42594103F028
:104B800041FC80212368490019404B4259410A20C9
:104B900003F038FC80212368890019404B425941B9
:104BA0000B2003F02FFC80212368890119404B4220
:104BB00059410C2003F026FC802123684903194049
:104BC0004B425941062003F01DFC80212368C90394
:104BD00019404B425941042003F014FC8023216802
:104BE0005B0419404B425941052003F00BFC0121A5
:104BF0000F205CE700100020F40F002004100020BC
:104C0000E80F0020E9DC0000012010B54042FFF76A
:104C1000BDFC0020FFF7D4FB10BD000010B5034A17
:104C20000921034800F074FF10BDC046D0DF00002A
:104C300018E000008023F0B502255B051A690A4CD4
:104C40000A4BA1261D5103278025F600ED00BA432B
:104C5000884202D300221A51F0BD5F59002FFCD0C8
:104C600098518018F4E7C0460405000000E00140B8
:104C700010B5002806D1C020B02140028902FFF7FC
:104C8000D9FF10BDB02080218002C902F7E70000E3
:104C900043425841064B40421840B0239B02C01883
:104CA000036800201A0E532A01D11B02180A70470C
:104CB00000C0FEFF30B501248025054B054AED00FC
:104CC0009C505C59002CFCD001600021995030BDF3
:104CD00000E001400405000043425841074B4042B8
:104CE0001840B0239B02C018A62310B50902DB05AB
:104CF000090A1943FFF7DEFF10BDC04600C0FEFFE2
:104D0000F0B5012480260D4B0D4DF6005C510029B5
:104D100002DC00225A51F0BD577814783F02274335
:104D2000947824042743D478043224063C439F59C2
:104D3000002FFCD010C00139E9E7C04600E0014077
:104D40000405000070B505004B680A009C1C21009A
:104D5000A400FFF7D5FF281970BD0000134B1B6896
:104D6000002B0CD08022B023D2029B0200280BD152
:104D70001A1D5B681B0E522B00D110007047B02229
:104D8000C02392025B02F1E782420DD903681B0E39
:104D9000522B09D1436802339B00C018824203D9C9
:104DA00003681B0E522BE9D00020E7E70811002012
:104DB000F0B50020B7B00024FFF7D0FF27000500B2
:104DC0002600002D2ED1284D2868FFF761FF320004
:104DD0003B0001900094254904A807F021FC04A899
:104DE00001F0CEF8224B64201C682B68A0215A42A7
:104DF0005341204A5B421340B02292029B18E41AAE
:104E00006043490204F084FFA02252020300009292
:104E10001949220004A807F003FC04A801F0B0F827
:104E200037B0F0BDFF226B6829689C460233FF183B
:104E30000B12013613409C4200DA1C00FF200A14BA
:104E4000024003926246014001920091039A0B498D
:104E500004A807F0E5FB04A801F092F82800FFF78A
:104E60007DFF0500ADE7C0460811002022E10000EB
:104E70000C11002000C0FEFFCCE000000EE100009D
:104E800070B50020FFF704FF04000120FFF700FFCA
:104E9000844200DA04000A4B1D686A42554128002A
:104EA0001D60FFF7E5FEA0226B4252021340054A47
:104EB00028009B18044A611C1360FFF70DFF70BDAA
:104EC00008110020048001000C110020F8B500201A
:104ED000FFF7DEFE07000120FFF7DAFE3E00204D5F
:104EE0000643204C0DD18021C020C9024002FFF7AB
:104EF000A1FE01213000FFF7EFFE1B4B2E60236067
:104F00001DE0874209DD0023B0212B60164B89028A
:104F1000236023680020012517E0012380212B60F6
:104F2000124BC9022360F4E7120E522A08D000285F
:104F300000D023600E4801F023F8FFF7A1FFF8BD71
:104F400028005A68023292009B188B4205D21A68D8
:104F5000561CE9D10028F2D0D1E72160EFE7C04626
:104F6000081100200C1100200480010004C0020080
:104F7000E7E0000070B50020FFF7F0FEFF26050017
:104F8000002801D1280070BD03681C143440FFF7CD
:104F9000E5FEDA2CF4D10500F2E700008022F0B53E
:104FA0005200A1B00021674806F0F6FF80220021E0
:104FB0005200654806F0F0FF644BFF271B681A009B
:104FC000049353425A4110000592FFF751FE049C8E
:104FD0000020631E9C415E4B64421C405D4BE41804
:104FE000FFF7C8FF0600002E2DD10498FFF750FEF2
:104FF000411C0598FFF770FE059A574D534B2C60E6
:105000001A60FEF721FD514B64201B68A0215A4213
:1050100053414F4A5B421340B0222C6892029B18C6
:10502000E41A6043490204F073FEA0225202030016
:1050300000924A49220007A807F0F2FA07A800F0F8
:105040009FFF21B0F0BD3268131412123A403B406A
:1050500003921A000A3A092A49D83A4B039A995CF2
:10506000002931D110223E4806F096FF35002B680A
:1050700003991A123A40914209D11A143A400B2A64
:1050800027D0132A2DD00A2A01D1354B1D602800C4
:10509000FFF764FE051EEAD1314B196800290FD0D5
:1050A0002000FFF74FFE04002D4B5B1959680029C3
:1050B00003D02000FFF746FE040004350C2DF3D189
:1050C000204B0121039A99543000FFF747FE060058
:1050D00089E73B40022BDADC214A9B00D3185D6054
:1050E000D5E7102200211E4806F056FFCFE71A0030
:1050F000153A082AE8D8144A0399525C002AE3D1E9
:105100003500152B00D01500300003681A143A4002
:10511000152A0FD01D2A00D10025FFF71FFE0028F9
:10512000F3D1002D04D020002900FFF70BFE04006E
:10513000054BC6E7039A1B123B409A42EDD105008E
:10514000EBE7C046081000201011002008110020D5
:1051500000C0FEFF04C002000C110020B1E00000FE
:105160002C2F002010B5FFF719FF10BDF0B585B04A
:10517000039203220333DC17294D1440E4182B68F3
:10518000284F5A42534180225B42D202A4103B4036
:105190009B18A21C0291244E91000091019031684D
:1051A00000980A18934215D2FFF7F8FE2B685A426E
:1051B000534180225B421F40D202BF183368009ADD
:1051C0009B189F4206D2194800F0DAFE00252800FD
:1051D00005B0F0BD029B356819066B461A7BA42307
:1051E000DB051343FF222F00090C1943019B120416
:1051F0001B04134019432800FFF75CFD0837281DE6
:1052000021003760FFF756FD002C04D00A9A2100D8
:105210003800FFF775FD009B083BFF183760D6E7A5
:105220000811002000C0FEFF0C1100208BE00000E0
:1052300070B59AB0FFF74AFEFF221E4CD200002143
:10524000200006F0A9FEFF25FFF794FE00260028A7
:1052500014D10200C300E3580130591E8B41D2180B
:10526000FF28F7D1144901A807F0DAF901A800F0E6
:1052700087FE124800F084FE1AB070BD03681A144D
:105280002A400A2A0AD11A122A40FF2A03D0D20041
:10529000A1180B71A050FFF761FDD8E7132AFAD1CE
:1052A0001B122B40FF2BF6D0DB00E2181671E650E4
:1052B000F1E7C046A425002057E100006BE10000A3
:1052C0000021094B094A5960013151605968002990
:1052D000FCD000211961012393600222044B81312B
:1052E000FF315A501A607047FC1000400010004017
:1052F00000E100E00222064B0121DA670022054BA3
:105300005A61054A11615A69002AFCD07047C046AB
:1053100004E100E0FC1000400010004010B5044C17
:105320002378002B01D0FFF7E5FF0020207010BD8F
:1053300011120020802301205B055B6E5B00184387
:10534000704700000120024B1B685B001843704748
:10535000941200200120024B1B685B001843704729
:10536000240000200120024B1B685B00184370479B
:105370009812002070B504000D001600FEF71CF90D
:10538000802301215B055A6E267000265300617050
:10539000E1706272010A5A0A6071A171A272010C75
:1053A0005A0C000E5B0EA6702571E1712072E2723C
:1053B000237370BD10B5044C200007F077F901008D
:1053C0002000FEF7D7FD10BD9D1200200E4B10B53A
:1053D0001B680E4C5A1C0FD00D4C002B0CD00D4CE2
:1053E000012B09D00C4C022B06D0094C042B03D006
:1053F0000A4C052B00D1074C200007F057F901009B
:105400002000FEF7B7FD10BD28000020FCE10000E1
:10541000E8D9000007E20000EFD9000001E2000037
:1054200070B5214C2278002A3DD1204B01215A60D1
:105430008022D20511605A68002AFCD00022072081
:105440001B4B1C4901255A500439585008315A50F9
:1054500019481A4958501A491A485A501A495A5064
:10546000A622D2009D50082218495A5004315850A3
:1054700002201749585017491748585017480439FF
:105480005850182016495850C12189005A500539E2
:10549000FF395858921802435A501249124A9950EB
:1054A000FFF70EFF257070BD11120020FC000040B8
:1054B000001000400C050000746962751C050000B6
:1054C00024050000200004022C0500001405000043
:1054D000340500003C050000FFFF00002110010022
:1054E00054050000121200200405000070B50E4B98
:1054F00006001B78002B01D1FFF792FF00200B4D17
:105500002C7884420ED00A4B202219780323091BE1
:105510001940084B4901C918300006F021FD01204F
:10552000013C2C7070BDC046111200209C1200205E
:105530001012002012120020002370B588B098428B
:1055400035DD0D6801262C0034409C422FD123000C
:10555000042D2CD90F222B681A402300092A26D1AA
:105560006A683F2A23DD6846FFF7C0FF2300002852
:105570001DD06B4619783300A14203DB6B461B5DDF
:105580005B003343A200AA1801349360202CF2D1AF
:10559000092169444A780B7812021A438B781B045C
:1055A0001A43CB781B061343024A136004231800E6
:1055B00008B070BD9812002070B5454B8AB01B78BA
:1055C000002B01D1FFF72CFF02AC2000FFF78EFF6C
:1055D000002802D100200AB070BD23780B2BF9D926
:1055E0006378012BF6D1E378012BF3D1002311204E
:1055F000384E394D33602B7068442379374A4178EF
:105600001360027809021143827812041143C278B0
:1056100012060A4332490A60002B0ED11521694453
:105620004A780B7812021A438B781B041A43CB7802
:105630001B0613433360002318E0012B1AD11521F8
:1056400069444A780B7812021A438B781B041A4378
:10565000CB781A211B06134333600E23627C694406
:10566000934200DD130000229A422CD10022042034
:10567000EA54B0E7022B03D1627B10331621EEE728
:10568000042B0DD1152108226944684606F068FCF8
:105690000098019902F0F2FE06F014FB3060CAE7B0
:1056A000052BC8D1152108226944684606F058FC2C
:1056B0000098019902F0E2FE06F004FB3060627D82
:1056C0000A231E21CBE7885CA8540132CCE7C046F0
:1056D00011120020941200209D12002028000020AA
:1056E0009812002010B5134B04001B78002B01D139
:1056F000FFF796FEFFF7FEFD00200F4A0F49104B03
:10570000545058600130106058680028FCD00020C8
:1057100018610130906018690028FCD0094B0A48D4
:105720001B785B011B185350FFF7E4FDFFF7C8FD22
:1057300010BDC046111200200010004004050000FA
:10574000FC100040101200201212002010B588B08A
:1057500000281DDD0A68012113000B4018D1042A1E
:1057600016D90F2014682040092811D150683F280D
:105770000EDD9800101880680024084201D0401007
:10578000C4B26846C4540133202BF2D1FFF7AAFFFC
:10579000002008B010BD000010B5002813DD0C6813
:1057A000E30710D56410532C0DD8084B1B78002B41
:1057B00001D1FFF735FEFFF79DFDA123044ADB0071
:1057C000D450FFF77DFD002010BDC046111200200F
:1057D0000010004010B500280EDD0C68E3070BD563
:1057E0006410FF2C08D8054B1B78002B01D1FFF764
:1057F00017FE034A034BD450002010BD11120020A5
:10580000001000402405000013B5002814DD0C68CA
:10581000E30711D5094B64100093094B0193072C42
:105820000AD8084B1B78002B01D1FFF7F9FD6B4616
:10583000054A1957054BD150002016BDE2ECF0F493
:10584000F8FC000411120020001000400C050000BC
:1058500070B588B0002820DD0124086804401CD100
:1058600004281AD90F2302681340042B15D1FEF720
:1058700061F9060006F01AFF0500122800D912256A
:105880002A0002210D326846FFF774FD6B465D73F6
:10589000A54205DC6846FFF725FF002008B070BD73
:1058A0002300325D6B449A730134F1E7F0B50D00CB
:1058B0008BB0012832DD08680122040014402DD18C
:1058C00004282BD90F2301680B40042B26D16B68C9
:1058D000134223D0FEF72EF96E6807007310019370
:1058E00006F0E4FE05000E2800D90E252A0001214D
:1058F000113202A8FFF73EFD6A46127902AB5A73D5
:1059000002AA73129373019B76141B0ED673137441
:105910005574A54205DC02A8FFF7E4FE00200BB099
:10592000F0BD3A5D02A963189A740134F1E730B50D
:1059300089B0002814DD0C68E30711D510226846F1
:105940000021FFF717FD6B466A4665105D736846D8
:1059500063122D0E64149373D4731574FFF7C2FE93
:10596000002009B030BD0000174B184A59680029C3
:1059700003D00021596001319160196900291FD0BD
:10598000002018618023DB00D3581149012B18D166
:10599000A923DB00D3585B420B600E490B78032B25
:1059A00001D801330B7003200B490B7801330340FE
:1059B0000B700A495B015B1809495350012393603E
:1059C00070470860FAE7C046FC1000400010004035
:1059D000240000209C12002010120020121200202F
:1059E0000405000010B5034A1021034800F090F8A8
:1059F00010BDC0467CE1000073E10000044A054987
:105A00001368C85401339B059B0D13607047C04653
:105A1000CC160020CC12002070B5114C114A23681E
:105A2000834202DC0023236016E0155C411C2E003B
:105A3000FA3E012E05D899420FDA555C013D1F2D23
:105A400001D90800ECE70100151A565C6E540131CB
:105A50008B42FADC181A206070BD1570FAE7C04658
:105A6000D81A0020D816002010B5FDF79BFD064B74
:105A70001A68824201D900221A601B68C31A0348BF
:105A800098428041404210BDC8120020204E0000C4
:105A900010B5094C094A23681268934200D110BD21
:105AA000074AD05CFDF7C8FF0028F8D0236801330F
:105AB0009B059B0D2360ECE7D0160020CC16002040
:105AC000CC12002010B50400064B074A1B68126870
:105AD0009B1ADB439B059B0DA34200DB10BDFFF728
:105AE000D7FFF1E7CC160020D016002070B5FFF7E5
:105AF00041FAFF250400002801D1200070BD036891
:105B00001B142B401D2B00D10400FFF727F9F2E7EF
:105B100070B5074E33680B2B08DC0C255D43054C34
:105B20000133285164196160A260336070BDC046C2
:105B3000D41600203C2F002010B5FBF79DFBFFF78B
:105B40006DF8FBF7C1FBFDF70BFFFEF7C3FBFEF79C
:105B50001FFCFFF747FF01F049F801F011FB01F0CE
:105B60003DFB01F087FD10BD962210B5120100210A
:105B7000034806F011FA0022024B1A6010BDC0461D
:105B8000441C0020D405002070B514007F22174B60
:105B9000C000C0580D00836813401C2B01D00020AA
:105BA00070BDC368190011400429F8D101690A4089
:105BB000192AF4D11B0A01339B000C30C018FDF7E1
:105BC000B9FF037806000120002BE9D0300006F071
:105BD0006DFD0023A042E2D1A34201DB0120DFE7FB
:105BE000F15CEA5C9142DAD10133F5E7A4250020AB
:105BF000064B074A1B6812689B1ADB439B059B0DEB
:105C00000122834200DC002210007047CC160020E5
:105C1000D0160020F8B505000C0016001F1E0ED18E
:105C20000320FFF7E5FF002808D0FA20FFF7E6FE83
:105C3000E8B2FFF7E3FEE0B2FFF7E0FEF8BD501D6B
:105C4000FFF7D6FF0028F9D0FB20FFF7D7FEE8B218
:105C5000FFF7D4FEE0B2FFF7D1FEF0B2FFF7CEFEC1
:105C60003012C0B2FFF7CAFE3C00E31B9E42E5DDE6
:105C70002078FFF7C3FE0134F7E7000070B5002479
:105C8000F0250B4B1B68A34202DCFFF76DFF70BDD4
:105C90002B006343074A9B181A78002A05D05978CD
:105CA000002311201A00FFF7B5FF0134E9E7C046D1
:105CB000D4050020441C0020F8B507000024F0257E
:105CC0002B0063430C4A01349E18B74211D031783F
:105CD00000290BD00133D15C002311201A00FFF7FB
:105CE00099FF2A000021300006F056F90A2CE7D16E
:105CF000F8BD024B1C60F9E7441C0020D4050020CD
:105D0000F0B5150001222F007A4C1740A5440190F0
:105D10000291002F11D005AB1A706A105A70120E42
:105D20001A710522691299706D140299DD70FFF7DE
:105D300071FFCF239B009D44F0BD042D2AD90F2471
:105D400028680440042C32D1022304AA28001371CD
:105D5000FDF7F0FE050006F0A9FCC82302009B0039
:105D6000984200DD1A007C1C97420DD1984206D95A
:105D7000614804AB03226149C01806F0F1F8220023
:105D800005AB02990198D2E72700611E695C05AC5A
:105D9000E155E8E7042D00D0A7E0032304AA043D61
:105DA00013716B425D4105AB55710222E9E7092C85
:105DB0007ED1042205AB1A706A68511000916946C1
:105DC000521209789A70009A59701F2A01DD202218
:105DD00000926A46127806ACDA70009BBB4202DC85
:105DE00005ABE21ACDE70126BB00EB189868064028
:105DF00006D1042837D90F210368194002290CD194
:105E0000012323704310637042121B0E4014A270D2
:105E1000E070237105340137DFE7042921D1022323
:105E20002370FDF787FE039006F040FCA31C0C28AE
:105E300009D86070864201D19C19ECE7039A925D03
:105E40009A550136F6E70C226270039A925D9A55D4
:105E50000136092EF9D12E23E372237363730E34B6
:105E6000D9E7012907D1032304382370434258415D
:105E700060700234CFE7092909D1042323704368F5
:105E80005A1062705B12A370E6700434C3E70329F2
:105E90000BD1052323700068020992B2430F9200D0
:105EA0000B40D31A63701B12EDE726700134B2E782
:105EB000032C00D03DE7052205AB01091A7089B219
:105EC000420F890022408A1A11125A709970642A6E
:105ED00000DD64220421DA70081F824201DC0432F2
:105EE0004FE7685C58540131F6E7002D00D020E7F9
:105EF00053E7C046C4FCFFFF2203000054D6000055
:105F000070B502000024F0210D4E08006043801996
:105F10004578954203D001340A2CF6D170BDF022A9
:105F2000002106F039F8074A1368013BA34200D16B
:105F30001460002329001A001120FFF76BFEEDE723
:105F4000441C0020D405002010B5B2B002236A46DC
:105F50000400137006F0AAFBC72800D9C72000234D
:105F6000984207DC421C6B46FE211420FFF752FECC
:105F700032B010BD694601335A1EA25CCA54EFE725
:105F800030B5B3B002236A460500137006F08EFBED
:105F90000400C72800D9C72400239C420BDC200042
:105FA0003230FFF78FFD621C6B46FF211420FFF794
:105FB00031FE33B030BD694601335A1EAA5CCA5463
:105FC000EBE70000F0B5BDB005900C00012803DC44
:105FD0001B20FBF713FB55E02C4B08680393C3070A
:105FE00009D4042807D90F2302681340042B02D1D7
:105FF000FDF7A0FD0390254B60680493C30709D407
:10600000042807D90F2302681340042B02D1FDF79F
:1060100091FD049000261E4B1B680893089BB34219
:106020000BDC049B1B4A0093C821039B0AA806F0C3
:10603000C5FA0AA8FFF7A4FFCAE70C257543164B5B
:106040000399ED18286806F027FB071E05D16B6839
:10605000AD680993099B9F4201DB0136DEE72868A2
:106060000499079506F018FB0835069000280BD117
:1060700021000598079B08315B6802389847074B59
:10608000069A1A603DB0F0BD0137E3E706DB000079
:10609000D4160020D8E200003C2F0020E00F0020A2
:1060A000F7B5234B06001B68F02100930023009AEC
:1060B0009A4211DC0024F0231A00624301920199F4
:1060C0001C4A55182F78002F12D001340A2CF3D116
:1060D0001948FFF755FF29E00A005A43154882186E
:1060E0005078B04202D11278002A1FD10133DEE786
:1060F000F0223900280005F04FFF02230D4A0199D4
:10610000EB6053540D4AF1008A58009B6E70AE70DC
:10611000AA602F616F61A34202DC054B01341C6051
:10612000002331001A001020FFF774FDF7BDC046B0
:10613000D4050020441C002021E70000A4250020F5
:1061400010B5FFF79BFDFF24084AE3005B429B1854
:10615000074AD35C043B012B03D8E043C0B2FFF7EE
:106160009FFF013C002CEFD110BDC046FC07000092
:10617000A4250020F8B505000E00FDF7FBFEFF2466
:106180000D4B18600D4AE3005B429B180C4AD35C30
:10619000062B01D0032B0BD1E743FFB232002900BD
:1061A0003800FFF7F1FC002802D03800FFF778FF35
:1061B000013C002CE6D1F8BD08000020FC070000DF
:1061C000A425002070B50500FF24084AE3005B42C7
:1061D0009B18074AD35CAB4203D1E043C0B2FFF740
:1061E0005FFF013C002CF0D170BDC046FC070000F1
:1061F000A4250020F7B5FDF7D5F9574B1A68824260
:1062000001D900221A601A685449821A8A420DD9AB
:10621000FF2253491860D3005248CB1A1B181B7831
:10622000073B022B0CD9013A002AF4D1F7BD072015
:10623000FFF7C8FF4C4B27E00820FFF7C3FF38E00B
:10624000FDF7BAF9071E00D101270020FDF7B6FAC5
:1062500001900020FDF7C6FA019B0090434C444D8D
:10626000002B12D02368002B6ED12B682760002BE7
:106270006ED0404B01261B78002BD8D10920FFF7A8
:10628000A1FF394B1E703B4B1E70009B002B12D0A0
:106290002B68002B0FD123682F60002B1ED0324BB0
:1062A00001261B78002BC7D10920FFF78BFF2E4B4F
:1062B0001E70304B1E702368002B0FD02A4E327890
:1062C000002A0BD19F4200D227602368FB1A312B92
:1062D00004D90720FFF776FF012333702B68002BCA
:1062E0000FD0244E3278002A0BD1BB4200D92F6048
:1062F0002B68FF1A312F04D90820FFF763FF012311
:1063000033702368002B0CD0019B002B09D1164E53
:106310003378002B02D10720FFF754FF00232360BE
:1063200033702B68002B00D180E7009B002B00D03E
:106330007CE7104C2378002B02D10820FFF742FFA6
:1063400000232B60237071E7009A002AA0D1B5E7E3
:10635000009B002B9FD1AEE7C41200200F27000046
:10636000A4250020FC070000B8120020B412002071
:10637000BC120020C012002037B500240500FFF732
:106380007DFC01A80194FDF707FA21002000FEF72B
:10639000EDF8FEF7EDFAFDF739FAFDF7BDFAFDF776
:1063A000D7FAFEF731FCFDF72BF9A54204D0FDF733
:1063B0006DFB0248FFF7E4FD37BDC04612E7000061
:1063C000002310B501001A001120FFF723FC10BDB7
:1063D00007B56B46197069465A7013128B70131407
:1063E000120ECB700A716B46010005221320FFF7D5
:1063F00011FC07BD10B50A0001001220FFF780FC58
:1064000010BD70B505000C00FDF7E4F8002809D0B8
:1064100020003230FFF756FB2B00220000211B200A
:10642000FFF7F8FB70BD10B50C000300110014203D
:106430002200FFF7EFFB10BD012370B5FF24084ACF
:1064400041185B42884201D3D84370BD06781D0ACB
:10645000234073409B009B5801306B40F2E7C046DD
:10646000F4E2000013B50400FE2813D80A4BC20062
:10647000D05800280ED0436808309900FFF7DCFFA1
:1064800001900920FFF71EFB01AB04222100172019
:10649000FFF7C0FB13BDC046A4250020F7B501904F
:1064A000FFF724FB01250400FF276D42002C01D1DA
:1064B0002800FEBD266833143B40152B0DD121006A
:1064C0000198083106F0E8F8002801D135123D4066
:1064D0002000FEF743FC0400E8E71D2BF8D101255E
:1064E0006D42F5E7F0B580279FB0FFF7D1FAB54CC4
:1064F000B54D2068FF00391A4019FDF783FA23686B
:106500000600C3182360002B0ED11FB0F0BD206819
:10651000391A2818FDF776FA236806001B1823603D
:10652000FDF740F8A94B1860002EF0DC2B78FA2B11
:1065300000D00EE12368022B07DCFFF795FA002854
:10654000E3D00120FFF768FADFE76B78AC78981E9C
:10655000182800D9F2E003F047FB0D2024282B3443
:10656000F13E707A7E94CDDEF1F1F1F1F1F1F1F1CD
:10657000F1F1EC00FF2C0ED02000FFF7C1FC00224F
:10658000934BE100CA505B181A712100009213006E
:106590001320FEF7EBFD0320D4E72000FFF780FD7A
:1065A000F9E72000FFF7ACFCF5E7FFF7C9FDF2E7DC
:1065B000FFF764FB0020FFF7DFFE8648FFF7E0FCF3
:1065C000E9E7632CE7D8844BA200D25821001520BC
:1065D000FFF796FBDFE7FFF789FAFF270400002C9F
:1065E000D9D025682B143B40152B04D02000FEF792
:1065F000B5FB0400F3E72000083006F057F806006A
:106600000530FFF75FFAFB20FFF7F8F92D121D2088
:10661000FFF7F4F9E8B2FFF7F1F9F0B2FFF7EEF99E
:106620003012C0B2FFF7EAF925002B1B9E42DDDDD8
:10663000287AFFF7E3F90135F7E700211D200091E3
:106640000B000A00FEF792FDFDF720FAA3E72000F9
:10665000FFF708FF9FE7FCF7BFFF05AC5F4A642127
:1066600000905F4B200005F0A9FF0223200023705B
:1066700006F01CF82300020000211620FFF7CAFADA
:1066800089E70026524AF3009B181C68002C28D08A
:106690001B790393636808349F00B81D0293FFF7CA
:1066A00011FAFB20FFF7AAF901207D1CFFF7A6F9DC
:1066B000F0B2FFF7A3F9E8B22D12FFF79FF9E8B2A5
:1066C000FFF79CF90398FFF799F9E719A7420CD84F
:1066D000FFF7DEF905230298584301F073FCFFF73A
:1066E000D7F90136FF2ECDD155E72078FFF786F98F
:1066F0000134EBE70024FFF7C1FA220021000094E7
:106700002300DA20FEF732FDFF222100D2003048BC
:1067100005F042FC98E7012C02D1FEF749FB3AE76D
:10672000022C02D1FEF71EFD35E70120FFF724FE03
:1067300031E7002321001A001A209FE71A00C83A07
:10674000052A00D927E7002218001100FAF7C8FD32
:1067500021E7FB2B00D0F4E62268042A00DCECE6FB
:106760002E79E8781F4B360206439E4200DDE8E6AC
:10677000331D9A4200DCE0E6EB5CFE2B00D0E0E645
:106780006878AC78771E1B2800D17DE02ED80728CA
:1067900063D0082838D001282DD1FF2C10D020003C
:1067A000FFF7AEFB6D79104AB31E009221002A005C
:1067B0000A20FEF7DBFC064BE400E0501B191D71BC
:1067C000701DBFE6D81A0020D8160020C81200207D
:1067D000A4250020F4E600009C2D00200BE700001B
:1067E00006E70000F6030000DE1600201D285DD03D
:1067F0004FD31E2871D00300C83B052BE0D8404A78
:106800003900FAF76DFDDBE7632CD9D86A79022AE3
:1068100013D0032A1BD0012AD2D1E979AB7909021E
:1068200019432B7AA4001B0419436B7A1B060B43F4
:106830005B001343334AA350C2E7002FC0DDB11EF3
:106840003148FDF797FB2F4BA400E050B8E7AB7938
:10685000A4005A1E93419B00ECE7632FB0DC05AD0A
:106860003A002749280005F07BFB00232800EB5560
:10687000FFF714FE0028A3DB224B8000C258210042
:106880001520FFF73DFA9BE739001D48FFF772FC22
:1068900096E7FF2C94D06A79022A91D81A490B20E6
:1068A00000912100B31EFEF761FC89E7632F00DD34
:1068B0006327002305A9BB420ADBFB430022DB1749
:1068C0003B40CB181A70152000917B1C2100EAE791
:1068D000EA185279CA540133EDE7012C00D06FE772
:1068E000002F00DC6CE76B79002B03D01C00322BEF
:1068F00000DD322464235C43044B1C6060E7C04627
:10690000DD1600209C2D0020DE1600200400002053
:106910000120704710B5064C200000F0BFFF05496C
:10692000200000F0EFFF0122034B1A6010BDC046AB
:10693000141B0020801A0600DC1A00201FB500215D
:106940001020FCF74FFE01211120FCF74BFE012126
:106950001620FCF747FE1C4C200000F0FDFE1B4BF0
:106960001B4A1B6812681B49D2B28B420BD880238A
:106970009B04019301AB1A710199029A0023200034
:1069800000F006FF1FBD14498B4202D88023DB04B0
:10699000EFE712498B4202D880231B05E9E7104933
:1069A0008B4202D880235B05E3E70E498B4202D875
:1069B00080239B05DDE70C498B4202D88023DB0551
:1069C000D7E780231B06D4E7F41A0020300000200C
:1069D0002C00002048E8010090D0030020A107000F
:1069E00040420F0080841E0000093D0010B50028C1
:1069F00015DD01240B68234211D023410C4A13609A
:106A00000C4AA04209D04B68234206D02341022BF6
:106A100009D0032B09D0A34203D002231360002026
:106A200010BD0023FAE70323F8E71460F7E7C04638
:106A3000300000202C000020F8B501250C682C4205
:106A400003D10D20FAF7DAFDF8BD64102DD4FCF760
:106A5000C7FDA04229DB00212000FCF7C3FDFA227C
:106A60002900D200200001F0DFFA00281DD0002507
:106A700000270726FA2201219200200001F0D4FA13
:106A8000002812D0282802DD0123B3401F43013E15
:106A9000F0D20E4EAF550135052DE9D10122062168
:106AA0000920FDF7E9F9002801D10020CCE70B23EC
:106AB000012443600023F25C9900520041182243F4
:106AC00001338A60052BF6D1BEE7C046E01A0020EC
:106AD000F0B50E0085B000282BDD01230A681340B5
:106AE00027D1042A25D917680F221740032F20D158
:106AF000802101AA104D13718904029A2800039382
:106B0000019100F045FE366833681C095B0F3B407D
:106B10003700A4B2A400E41ABB1B9C4206DD3979FD
:106B2000280000F03BFE0137F870F5E7280000F080
:106B300034FE002005B0F0BDF41A002010B5046842
:106B40000D20E30703D56410FF2C03D91720FAF7B3
:106B500055FD10BDFFF7F2FEE1B2044C200000F03D
:106B60001DFE200000F019FE0020F2E7F41A0020BC
:106B700070B5FFF7E3FE064D0021280000F00EFE81
:106B80000400280000F009FE01206400204370BDCD
:106B9000F41A0020A02101220B4BC9005A500B48C7
:106BA0000B4958500B491A604A68002AFCD0002251
:106BB0004A60A121C900585801215960A021C9008B
:106BC0005A50054BC0187047007000406A10000012
:106BD00004050000FC700040FBFDFFFF10B5FFF74F
:106BE000D9FF43000120184310BD000010B5034A2F
:106BF0000D210348FEF78CFF10BDC04638E70000AA
:106C0000A0E700000D4B70B51B6804000E001500D6
:106C1000002B01D1FFF77EFEE1B2094C200000F00D
:106C200008FFF1B2200000F005FEE9B2200000F0FC
:106C300001FE200000F068FF70BDC046DC1A002095
:106C4000141B002010B501240368234205D04168BD
:106C5000214202D08268224203D10D20FAF7CEFCF5
:106C600010BD5810802801D91520F7E74910FF29D9
:106C700001D91620F2E75210FF2A01D91720EDE7BB
:106C8000FFF7C0FF0020EBE710B5002803DC1C2055
:106C9000FAF7B4FC10BD0B68DA0701D40D20F7E752
:106CA0005B100322012B06DD0522022B03D00C22F0
:106CB000042B00DC08220F211820FFF7A3FF02207D
:106CC00001F080F90020E5E7F7B5012214009042B9
:106CD00026DD0D682A4223D02D4B15411B684C68D8
:106CE000002B01D1FFF716FE2A4EE9B2300000F06A
:106CF000A0FE27000122174014D01441FF2C02D916
:106D00001720FAF77BFCE1B2300000F093FD300071
:106D100000F0FAFE0024A04202D02320FAF76EFC15
:106D20002000FEBD042CF2D90F2523681D40092D3B
:106D30001CD1636801925B100093009BBB42E6DDAF
:106D4000BB00E3189D68019B1D420BD06D10FF2D09
:106D500002D91720FAF752FCE9B2300000F06AFDC0
:106D60000137EAE71720FAF749FCF9E7032DCED1FE
:106D700027001A0992B25B0F92001D40551B3B1B66
:106D80009D42C4DD3979300000F054FD0137F6E74B
:106D9000DC1A0020141B0020154B70B51B68050081
:106DA0000E00002B01D1FFF7B5FD124CEDB229000A
:106DB000200000F03EFEF1B2200000F03BFD00217B
:106DC000200000F041FE002801D0404270BD72B6A4
:106DD00001222900200000F027FE62B6200000F00A
:106DE0001AFD0028F2D0200000F01AFDEEE7C046A0
:106DF000DC1A0020141B002010B501240368234274
:106E000002D04168214203D10D20FAF7F7FB10BDF3
:106E10005810802801D91520F7E74910FF2901D91A
:106E20001620F2E7FFF7B8FF40002043EFE700002D
:106E300070B5284D04002B68002B08D105211820BF
:106E4000FFF7AAFF022001F0BDF801232B60012CFF
:106E500014D105211820FFF79FFF7F282BDC0300AA
:106E60007F3301DA7F204042C8235B4258437F21B1
:106E700002F04EFF052C00D1404270BD032C11D111
:106E800021001820FFF788FF7F2814DC03007F33E0
:106E900001DA7F204042C8235B4258437F2102F041
:106EA00037FFEAE70020052CF5D107211830FFF75E
:106EB00073FF7F2802DD0138FF38D0E703007F33FE
:106EC00001DA7F204042C8235B4258437F2102F011
:106ED0001FFFD1E7E81A002010B50120FFF7A8FF37
:106EE00043000120184310BD10B50320FFF7A0FF99
:106EF00043000120184310BD10B50520FFF798FF8F
:106F000043000120184310BD10B508211820FFF7D9
:106F100043FF0300C00FC01801234010153040008C
:106F2000184310BDF8B501231C0098422BDD0F68F3
:106F30003B4228D04E6835001D4024D1042E22D972
:106F40000F2231680A40092A1DD173685C10202C79
:106F500000DD2024144B1B68002B01D1FFF7DAFC65
:106F600072B67F10F9B2114F2200380000F05CFDBC
:106F700062B6A54214DA380000F04DFC002804D1B6
:106F800001246D002C432000F8BD380000F048FCBF
:106F90000122AB004000F31810439860AD18E8E7F9
:106FA00064000125EEE7C046DC1A0020141B002017
:106FB00070B52B4B86B01B68002B02D10120FFF768
:106FC00037FF01AD14220021280004F0E5FF254E13
:106FD0001821300000F02DFD0321300000F02AFCC4
:106FE0000021300000F030FD041E13D172B60522DE
:106FF0001821300000F018FD62B6300000F00BFCE4
:10700000002802D0300000F00BFCA3000134E8504F
:10701000052CF2D1019B7F2B01DD013BFF3BAA68D0
:107020007F2A01DD013AFF3A29697F2901DD013913
:10703000FF39C820434342434843DB11D211524336
:10704000C0115B4340439B18181804F071FE01F017
:1070500045FB04F037FE43000120184306B070BD25
:10706000E81A0020141B002010B5054C2368002BE3
:1070700002D01B20FAF7C2FA0020206010BDC046E3
:10708000EC1A002010B5002803DC1C20FAF7B6FA31
:1070900010BD0B68DA0706D4042B04D90F221B6835
:1070A0001340032B01D02420F0E7034B25201B685D
:1070B000002BEBD01B20E9E7EC1A002010B50028CC
:1070C00003DC1C20FAF79AFA10BD0B68DB0701D429
:1070D0000D20F7E71B20FAF791FA0020F4E710B52E
:1070E0000400802803DD2620FAF788FA10BD002C62
:1070F000FCDD1B20FAF782FA012000F063FFF6E7BF
:1071000010B5002805DC1C20FAF778FA04002000EE
:1071100010BD144B1B68002B01D12520F4E701247E
:107120000868044006D01B20FAF768FA012000F036
:1071300049FFF8E70428EAD90F2102681140042921
:1071400006D1FCF7F7FC05F0B1FAFFF7C8FFDEE760
:107150000329DCD1100980B2520F80000A40801A46
:10716000F3E7C046EC1A0020044B10B51B6825203D
:10717000002B00D01B20FAF741FA10BDEC1A0020BA
:1071800010B5034A05210348FEF7C2FC10BDC046F6
:107190002CE8000054E800000020704701207047F0
:1071A0000020704700207047002070470120704782
:1071B0000020704700207047002070470020704773
:1071C0000020704700207047002070470020704763
:1071D00000207047704770477047000010B5034AA1
:1071E0000F210348FEF794FC10BDC04670E8000074
:1071F000E8E800000378013B1F2B00D970470130FD
:10720000F8E710B5FFF7F6FF0378002B0BD001303D
:10721000222B11D10378002B03D0421C222B03D147
:107220001000FFF7E7FF10BD5C2B03D14378002B64
:1072300000D0821C1000EDE73A2BF2D02C2BF0D0BE
:107240007B2B0BD1FFF7D6FF0378002BE9D07D2BEA
:1072500001D10130E5E7FFF7D4FFF5E720225B2BF2
:1072600014D1FFF7C7FF0378002BDAD05D2BF0D0E5
:10727000FFF7C7FFF7E7202BD3DD2C2BD3D0190066
:1072800091435D29CFD0222BCDD001300378002B44
:10729000F1D1C6E7002210B5904216D0FFF7AAFF41
:1072A00003780422222B10D0023A7B2B0DD0013A16
:1072B0005B2B0AD0190030390232092905D92D2B50
:1072C00005D14178303909290AD8100010BD0522AE
:1072D000742BFAD00132662BF7D001326E2BF4D02A
:1072E000581E83415A42F0E770B5FFF783FF0378D9
:1072F00001222D2B01D18018023A00230A2502E039
:107300006B430130CB1801783039CCB2092CF7D956
:107310005A43100070BDF8B50C001500FFF76AFF66
:107320000378222B02D000232370F8BD0D236A1EA0
:10733000210008250C260A279C4601300378222BC1
:1073400002D100230B70F0E7002BFAD0441C5C2B19
:107350000BD14378841C622B0ED0662B0ED06E2B83
:107360000ED0722B0ED0742B0ED0002AE9DD0B70DC
:10737000013A01312000E1E72B00F6E73300F4E7A2
:107380003B00F2E76346F0E70923EEE710B504009F
:10739000FFF737FFA04203D90378013B1F2B00D929
:1073A00010BD0138F6E710B5002815D00378002B82
:1073B00013D0FFF71FFF2021037802008B4300202A
:1073C0005D2B09D01000FFF71CFF03782C3B5A42BD
:1073D0005341C018FFF70EFF10BD1800FCE7030073
:1073E000002070B50C0081420EDD1A785B2A0BD1AB
:1073F000581CFFF7FFFE0125AC4205D0FFF7D3FF75
:10740000002801D00135F7E770BD70B50C001500FC
:10741000002901D000230B70002820D00378002B16
:107420001ED0FFF7E7FE037806002C2B03D10130B6
:10743000FFF7E0FE0600337800207D2B0FD084425A
:1074400004D02A0021003000FFF765FF3000FFF76D
:10745000D8FE03783A2B02D10130FFF7CBFE70BD86
:107460001800FCE7F0B50D0004009DB02E78002E4A
:1074700035D02E21280005F001F9071E14D0431B3A
:107480000193303E092E14D82800FFF72DFF01008C
:107490002000FFF7A4FF0400002C20D0002F1ED0F6
:1074A000019B0133ED18E1E7280005F0FFF801909A
:1074B000E7E723787B2B11D1601C642203A9FFF737
:1074C000A4FF041E0BD0019A290003A805F0F5F8CB
:1074D0000028E1D02000FFF794FEEEE70024200012
:1074E0001DB0F0BD70B5050000200C0081421DDD0F
:1074F0002800FFF7CFFE0300681C012B14D00020EA
:10750000022B13D10022681C1100FFF77EFF012C13
:107510000CD0FFF748FF00221100FFF776FF013C77
:10752000F5E7FFF740FF013C012CFAD170BDF8B53B
:10753000050000200C0016001F0081420DDD280010
:10754000FFF7A8FE03000020022B06D1681C3A00BA
:107550003100FFF75AFF012C00D1F8BDFFF723FFE0
:107560003A003100FFF751FF013CF4E710B5002469
:10757000A04218D0FFF73EFE03787B2B0AD10130E2
:1075800000221100FFF741FF00280CD0FFF739FE61
:107590000134F5E75B2B06D10130FFF704FF00282B
:1075A00001D00134F9E7200010BDF8B5002816DD40
:1075B0000D68EB0713D56D10013D0124FDF7DAFCD2
:1075C0000026FF27644200280CD1002E21D0300075
:1075D00005F06CF801003000FCF7CCFCF8BD01258B
:1075E0006D42EAE703681A143A40152A0BD11B12C0
:1075F0003B409C4200DA1C009D4201D10600083647
:10760000FDF7ACFBDFE71D2AFAD101240026644216
:10761000F6E70120013464002043DFE710B5086875
:107620000C00FCF787FAFEF739FF002803DB6268DD
:10763000024B8000C250002010BDC0469C2D00208F
:1076400010B50868FCF776FAFEF728FF012300283A
:1076500002DB024B8000C358180010BD9C2D002097
:1076600010B50868FCF766FAFEF718FFC043C00FB4
:10767000800010BD10B5034A04210348FEF748FA04
:1076800010BDC04684E900007EE9000010B5FCF79B
:1076900073F9FCF721FAFEF74FFA0448FEF770FC85
:1076A000FDF7C6FDFEF74CFD10BDC046D3E9000056
:1076B00010B5FBF7EBFD10BD70B5002504AC2478C8
:1076C0000573A94205D10A4B0A4A25210A4804F04C
:1076D000D9FB01600949920052589B0002715B5826
:1076E000A40083716358856043710223C37170BD28
:1076F000EBE900004AEA0000F9E90000A8EA00000E
:10770000037B002B04D14373837303610133037341
:10771000704700001FB50191A02100240068C90036
:10772000D2B24450012A10D0A24209D0032A0AD072
:10773000074A8350074B019AC250012343501FBD93
:1077400002221343F4E70422FBE70622F9E7C046CE
:10775000540500002405000010B50400FFF7D0FF19
:10776000A1222368A179D20099506179064A2000AC
:107770009950217904329950044B19685A689B68D2
:10778000FFF7C8FF10BDC0460C050000081B002015
:107790001FB5FFF7BFFF05B000BD70470368074A7C
:1077A00099501A00FC32D1680029FCD0A321C900ED
:1077B00058580023C0B2D3607047C0461C05000073
:1077C00007B58022074BD2051A6000229A60023268
:1077D0001A7111230E320093034905330348FFF752
:1077E0006BFF07BD081B002000300040F41A00208A
:1077F000F8B505000E0017000024BC4208D02B6825
:10780000315D1B6828009847002801D00134F4E757
:107810002000F8BD704710B51C3000F0AFF910BD66
:1078200010B51C3000F09CF910BD10B51C3000F0F4
:10783000ABF910BD70B5437E0D00002B01D10020C7
:1078400070BD6430040000F0A8F90028F7D12000D2
:10785000290000F076F90120F2E70000F7B5019366
:10786000FA23002504009B0083600B4B456008331E
:1078700003601C300F00160000F058F9200064303F
:1078800000F054F96B461B79276166756576A5761D
:107890002000A375FEBDC04688EA0000012330B574
:1078A000A024C375837D13499B005A58437DC13280
:1078B000114DFF32E40592009B005B581551CC221C
:1078C000C133FF339B001D5104690C4B5204E2503D
:1078D00005220469243BE250837D04699B005A58C9
:1078E000A123DB00E250437D02699B005958044B01
:1078F000D15030BDA8EA00000C06000024050000AD
:107900000C050000A022002310B50469D200A3508A
:107910000A4CA1420FD90A4C8C425B4109495B4297
:107920000B40CD21C9045B18046907496350052148
:107930000369995010BDCC235B04F5E7A0860100D4
:1079400090D00300000098FD24050000F7B5040066
:1079500000200D000193824265D01600402A00D914
:10796000402627001C37380000F0F6F8B1232269C2
:10797000DB00D55080220123216992008B50A27E2A
:10798000002A03D122691362226913600025731E45
:10799000AB4207D1019B002B04D080220221236936
:1079A00092009950012223691A622369FC33DA6834
:1079B000002A02D19A6A002AF9D09A6A002A0BD1C9
:1079C000DA60A3232269DB00D1583800C9B201353F
:1079D00000F0B7F8B542DAD3019B2269002B0FD132
:1079E0001300FC339B6A002B0AD10133A376D361C9
:1079F0002369FC33DA6C002AFCD00022DA640AE046
:107A000000230121A37651611A002369FC33996890
:107A10000029FCD09A602369FC339A6A002A01D0BD
:107A200000229A62E8B2FEBD10B50123FFF78EFF77
:107A300010BD0300AC3310B504001970643000F0C1
:107A40008BF80123637610BD0023020070B5AC32C1
:107A500043760D001178B12204000069D2008150F4
:107A60008022216992008B502269013313622269BE
:107A7000936026006436300000F080F8002812D0B1
:107A8000300000F06DF81E4B2269D0502369FC33A2
:107A90001A6A002A02D19A6A002AF9D09A6A002A40
:107AA00001D11A62E5E723690122002D0DD11900E9
:107AB000FC31896A002908D1DA612369FC33DA6C68
:107AC000002AFCD00022DA6407E05A612369FC3303
:107AD0009A68002AFCD000229A6000202369FC33B7
:107AE0009A6A82420BD098622169064A8B588B5061
:107AF0001800022B03D0181F431E9841033070BD9D
:107B00001C050000C404000010B50121FFF79CFF14
:107B100010BD000010B51323122202490248FFF7DE
:107B20009DFE10BD00400040141B002010B54022F7
:107B30000021040004F030FA002320002364636471
:107B400010BD10B53F24026C531C2340446C9C4272
:107B500001D08154036410BD002303644364704763
:107B6000436C026C934206D03F21C25C01330B4050
:107B700043641000704701204042FBE7036C406CF7
:107B8000181A00D540307047436C026C934201D004
:107B9000C05C704701204042FBE73F22036C406C11
:107BA00001331340181A43425841C0B270470000D5
:107BB00003210A4802680A430260094802680A432E
:107BC00002600849084A094B9B1A03DD043BC85868
:107BD000D050FBDC00F012F8F8F796FA24050040CC
:107BE00054050040F0EF0000000000206C0200206F
:107BF000FEE7FEE7FEE7FEE7FEE7FEE7014B024A8F
:107C00001A607047340000200024F40001207047FF
:107C100010B503681322DB69984710BD7047000058
:107C2000054B0269D1500369FC331A6A002AFCD063
:107C3000002201201A6270471C050000030010B5E5
:107C40005C331A781F231A401E3B19009140114AD9
:107C5000D167C222042104699200A15002695360D5
:107C60000269D360A02300220169DB00CA5001230E
:107C70000169094A5B428B500169084A8B500169CE
:107C80000C3A8B50016908328B501430FFF764FFB7
:107C900010BDC04604E100E00C0500001405000022
:107CA00010B51430FFF76AFF10BD10B51430FFF7A0
:107CB0006BFF10BD10B51430FFF752FF10BD000070
:107CC000030070B55E331A780469724BE25003000A
:107CD0005D331A780469704BE250030061331C78FD
:107CE00002696E4B012C00D09EE005005F352E78B6
:107CF000A225ED005651020060321578A1220669D6
:107D0000D200B5500269D4509623DB00994200D8C6
:107D10008CE096231B01994200D88AE096235B01F0
:107D2000994200D888E096239B01994200D885E0CB
:107D3000E1239B01994200D882E09623DB0199421E
:107D400000D880E0E123DB01994200D87DE0962352
:107D50001B02994200D87AE0E1231B02994200D825
:107D600077E096235B02994200D874E0E1235B023E
:107D7000994200D871E0E1239B02994200D86EE05D
:107D8000474B994200D86CE0E123DB02994200D8CE
:107D90006AE0E122002312038A425B41414A5B42CE
:107DA0001340802252059B1801693F4A8B50A02343
:107DB00004220169DB00CA5000210369FC33D96049
:107DC0000369FC331962012301690B6001698B604F
:107DD000C1210469890062501F215C3002780A4089
:107DE00093406231314AFF315350002141560029FE
:107DF0003CDA0F230B40083B2D4C9B089B001B19C2
:107E000003242140A140FC348C40DD69A5432C00B3
:107E1000C0258D4029002143D9611F2301781940D5
:107E20001E3B8B40136070BD00246CE79E23DB0279
:107E3000BAE79D231B03B7E71E4BB5E71E4BB3E71D
:107E4000EC239B03B0E71D4BAEE71D4BACE71D4B8E
:107E5000AAE71D4BA8E71D4BA6E71D4BA4E71D4B4A
:107E6000A2E78023DB049FE71B4B9DE78C080F4BA9
:107E7000A400E41803230B40FF21C025DB00994038
:107E8000AD0066598E433100C0269E4033000B433F
:107E90006351C2E70C050000140500006C050000EA
:107EA00090D0030000D0BEFE2405000000E100E0F9
:107EB00000ED00E000B013000050270000A04E00CD
:107EC00000F0750000509D0000F0EB0000903A01BA
:107ED00000E0D70100B0AF0300705F07F7B5009373
:107EE00008AB1B7800250193FA2304009B008360F4
:107EF0000E4B45600833036014300F001600FFF787
:107F000015FE23005C3327611E70009B084A9B000E
:107F1000995823005D331970019B20009B009A58EB
:107F200023005E33DD701A70FEBDC04624EB0000F6
:107F3000A8EA0000036910B51A00FC32D2680400F8
:107F4000002A0AD0A322D20099581430C9B2FFF7F0
:107F5000F8FD00222369FC33DA6010BD10B5024839
:107F6000FFF7E8FF10BDC046CC1B00201D2307B55E
:107F700002220093024901330248FFF7AFFF07BD19
:107F800000200040CC1B002010B5002801D004F0D8
:107F9000BFFA10BD0849094A094B10B51B6888583B
:107FA000FA22190A1B0618439200002301F0E8FF89
:107FB0004904C00B084310BD001001400405000037
:107FC000301C002070B5041E09D0FFF7E3FF050048
:107FD00000F014F8FFF7DEFF401BA042F8D370BD9D
:107FE0000022044B9A60044A13680133DBB2136029
:107FF0007047C046FC100140301C0020704770479D
:1080000010B500F05FF8FFF7FAFF0120FFF7DAFF85
:10801000FFF73CFBFFF74CFB024B002BFAD000E0D4
:1080200000BFF7E700000000F8B54C1EA141012594
:10803000104B114F8000C3584C4238680F499D4087
:10804000160001F0DBFD0A21704301F0D7FD2C4042
:108050000300220029000A4800F016F8FA21094C12
:1080600089004443386801F0C9FD0100200001F097
:10807000C5FDF8BDA8EA00003400002040420F0012
:10808000100500501027000030B504680C409442E1
:1080900006D1013B002BF8D112E0013B002B0FD0A1
:1080A00004680C409442F8D1002405680D409542C4
:1080B00004D101349C42F8D1002002E0201C00E0F1
:1080C000181C30BDC420114B80001A5810491140B3
:1080D000C02212020A431A50C02180224900920293
:1080E0005A501A608023A3220021DB05D200995048
:1080F0000122F9309A60074BFF301950C12002313C
:1081000080001950403019501A60704700E100E0BB
:10811000FF00FFFF00100140014B18607047C04690
:1081200080000020F7B500231E285AD8384B800065
:10813000C258042A5BD007D8022A54D055D8042349
:10814000012A09D000234CE0062A54D051D31A2A20
:1081500053D002231B2AF5D12E4A116808294ED983
:1081600009294FD00A240226A02001252A4AC0004E
:1081700015502A482A4D07681C20BF00074029488F
:10818000019700685759009027481B0207401F437A
:10819000C02300989B020340FF205751575900020B
:1081A00007401F43019B1F43009B58016023184059
:1081B00007433E43565101251C4B15605868002863
:1081C000FCD000205860A1230125DB00D358556066
:1081D000A025ED0050511BB2A14202D015D2611A68
:1081E000CB401800FEBD0823B6E71023B4E72023D8
:1081F000B2E74023B0E78023AEE70123ACE70824D1
:108200000026B1E70C000126AEE7091B8B40E8E72A
:10821000A8EA00007C000020007000403800002028
:10822000040500003C000020FF00FFFFFC70004040
:10823000F0B51E285BD8364B8000C258354B1E68FF
:10824000002E30D1C227344BBF00D859334C032500
:108250000440C02000022043D851C0248020640084
:10826000800018512E4F18602E4B803CD859FF3C8F
:10827000A043D8510437D859A8432043D8510837D0
:10828000D8590C35A8438446072065462843D85161
:10829000A820C0001E50C1208026800076021E50FB
:1082A0001C601C4B1C60142500202B001E4C2E0053
:1082B00046433659771C1BD14343E250A023032584
:1082C000C132FF329200DB05D550184B1A68082ADC
:1082D00014D114234343E3189A6812485132FF32F1
:1082E000920059601150DA68C1239B00C250F0BD62
:1082F0009642E1D001300328D9D1F8E7082A02D903
:10830000083AD140E5E708239A1A9140E1E7C046D0
:10831000A8EA0000341C002000E100E0FF00FFFF9D
:108320000405000000900040400000208000002074
:108330002149F0B54A6C2148002A14D0A025A12675
:1083400000230124ED05F600C258571C06D0C718BB
:108350007F68002F02D027009740AF5114333C2B89
:10836000F2D100234B64A0230121DB0500260F007E
:108370009C4614234B43C3181A1F1268104C0E4D11
:10838000920014195219526C002A10D01A00143A93
:108390001268551C09D0103B1B68FF2B05D03B0011
:1083A000934065461A00074BEA50FC34666401317D
:1083B0000429DED1F0BDC046FC9000404000002002
:1083C000009000400C05000000B51E2810D80C4A93
:1083D0008000835803290BD8A0220800C133FF3343
:1083E000D2059B0001F000FC020905070021D150D5
:1083F00000BD0C21FBE70421F9E70321F7E7C046A4
:10840000A8EA00001E280AD8074B8000C2580123A2
:108410009340A022D205002902D10449535070474D
:10842000A121C900FAE7C046A8EA00000C05000037
:10843000030000201E2B0AD8A021A222C905D200C9
:108440008858034A9B009B58D84001231840704726
:10845000A8EA0000F7B506000D000C008B18019388
:10846000019B671B9C4207D0336821781B68300052
:10847000984701340028F3D13800FEBDF0B5C64658
:1084800000B5CB0F9846404A4B005B0D9A1882B05E
:108490000D000400132A2FDC002A49DB3B4F174153
:1084A0003E000E40064323D07F08390029400C438C
:1084B0000AD03749BD438C4663445C425C4180230B
:1084C000DB021341E4071D434146CE0031492B0036
:1084D0008E192200346875682000290001F0F6FE2C
:1084E000009001910098019922002B0003F086F87A
:1084F00002B004BC9046F0BD332A08DD8023DB00C7
:108500009A42F5D102000B0001F0E0FEF0E7224AAA
:108510009446012263445242DA400242E8D05208B3
:108520000242D1D094438022D2051A411443CBE7B2
:108530004B005B080343DBD00B031B0B1C43634264
:10854000234380244D0C24031B0B23406D042B4339
:1085500019004346DA000F4B9B181C685D68020047
:108560000B002000290001F0B1FE0090019100985D
:10857000019922002B0003F041F842464B005B08B2
:10858000D60733431900B3E701FCFFFFFFFF0F00DD
:10859000EEFBFFFF58EB0000EDFBFFFFF8B5274AAD
:1085A0004B005B0D9A180C000700132A10DC002A00
:1085B00036DB234B13410B423AD080242403144171
:1085C000002064189C430600250030002900F8BDF7
:1085D000332A0EDD80230600DB000D009A42F4D121
:1085E00002000B003800210001F070FE06000D00B3
:1085F000EBE7144D0600AC46012563446D42DD40B7
:10860000AC4663460D000342DFD033239A1A323B57
:1086100093401818874200D94C1C63469843D2E710
:10862000C90FCC070020531CCDD1074B1C43CAE710
:1086300006000D000028C0D1C7E7C04601FCFFFFBF
:10864000FFFF0F00EDFBFFFF0000F03F30B5214AB8
:108650004B0087B05B0893421EDD1F4A934205DD45
:1086600002000B0002F0CAFF07B030BD02AA00F002
:1086700095F803231840049A059B012813D002287B
:108680001DD0002814D00298039900F06FFB8023BE
:108690001B069C466144E7E7002300220093002369
:1086A00001F0DEF8E0E70298039900F05FFBDBE7FA
:1086B000012402980399009401F0D2F8D4E7012430
:1086C00002980399009401F0CBF880231B069C4686
:1086D0006144C9E7FB21E93FFFFFEF7FF0B5474663
:1086E000CE4680B58DB004000D0000F067FA294B2E
:1086F00006001B780F005BB29846013310D02200B1
:108700002B002000290003F0C1FA8146002807D180
:10871000002200232000290001F00AFC002806D1D5
:10872000300039000DB00CBC90469946F0BD0123D5
:108730000293194B0694079503934B460A934346BD
:1087400004940595002B15D0002300221900100079
:1087500002F0D8F8434608900991022B0ED103F09D
:10876000AFFB212303600A9B0193002B0CD1089ED1
:10877000099FD5E7002300240893099402A801F07B
:10878000C1F90028EFD1EAE703F09AFB0A9B0193B5
:108790000360ECE78400002068EB0000F0B54E4673
:1087A0004546DE465746E0B5E14B4C008FB090465B
:1087B000894664089C4200DC87E0DE4B9C4222DC58
:1087C000DD4A002900DC92E0DC4B02F017FFDB4BB6
:1087D00006000F009C4200D17EE1D94AD94B02F03D
:1087E0000DFF02000B00414630000A604B6039006B
:1087F00002F004FFD34BD24A02F000FF43460125AA
:108800009860D9606BE0D04B9C4200DC8FE0CF4B8E
:108810009C4200DD55E1CE4A231592469A445146CA
:108820000905631A19001D00040003F04BFA03F058
:108830007FFA02000B00200029000892099302F041
:10884000DDFE0022C34B02F067FC0F00060003F0C0
:1088500039FA03F06DFA04000D0002000B0030003D
:1088600039000A940B9502F0C9FE0022B94B02F0C0
:1088700053FC002200230C900D9101F053FB0028C3
:1088800000D192E1002300222000290001F04AFBE0
:10889000434243410133B04A41460192022208A8B3
:1088A0000092524600F07CFB4B460500002B16DA86
:1088B000802243461206944642465B684542634422
:1088C0005360D3686344D36009E00B000200414663
:1088D0000A604B600022002300258A60CB602800DC
:1088E0000FB03CBC90469946A246AB46F0BD934BB8
:1088F00001F0ECFC914B06000F009C4200D13DE1E1
:108900008F4A904B01F0E2FC02000B004146300020
:108910000A604B60390002F071FE894A894B01F010
:10892000D5FC012543466D429860D960D7E701F038
:1089300049F88A4A8A4B06000F0002F0EDFB00223C
:10894000884B01F0C3FC03F0BDF9050003F0F0F91A
:10895000794A7A4B0490059102F0DEFB02000B008D
:108960003000390002F04AFE754A06000F000498F4
:108970000599744B02F0D0FB029003911F2D00DC8F
:10898000C7E0029A039B3000390002F037FE8346AD
:108990008A4653465B0024155B0DE31A102B6CDDF1
:1089A00004980599D322674B520502F0B5FB0200EB
:1089B0000B00300039000292039302F01FFE0A0000
:1089C000010013000691079202003900300002F006
:1089D00015FE029A039B02F011FE06000F00049898
:1089E0000599614A614B02F097FB32003B0002F0AF
:1089F00005FE069E079F0B00020039003000029220
:108A0000039302F0FBFD4B005B0D83468A46E41A9C
:108A1000312C32DD04980599B822544B920502F0AE
:108A20007BFB03000C000200029303940B000698EA
:108A3000079902F0E3FD02000B0006000F00069804
:108A4000079902F0DBFD029A039B02F0D7FD484A2A
:108A50000290039104980599464B02F05DFB029A3F
:108A6000039B02F0CBFD02000B00300039000292A4
:108A7000039302F0C3FD83468A465A465346414655
:108A800030000A604B60390002F0B8FD029A039B87
:108A900002F0B4FD44460B000200A260E3604B46C6
:108AA000002B00DB1BE75B46236080231B0653443F
:108AB000636080231B069C466144A060E1606D42B8
:108AC0000DE70B00020002F099FD43460025986077
:108AD000D9601860596002E7D3221A4B520502F0A0
:108AE0008DFD214A214B0D00040002F087FD02009C
:108AF0000B00414620000A604B60290002F07EFD19
:108B00001A4B194A02F07AFD434601259860D96054
:108B1000E5E602000B003000390002F06FFD6B1E2D
:108B2000154A9B009B5883468A46A342A5D130E74D
:108B3000FB21E93F7BD9024000004054FB21F93F73
:108B40003163621A61B4D03DFB213941FFFFEF7FF1
:108B5000EAFBFFFF00007041F0EB000083C8C96D25
:108B6000305FE43F0000E03F7370032E8A19A33B9F
:108B7000C14920259A837B3970EB0000D3220C4B2E
:108B8000520501F0A3FB0B4A0B4B04000D0001F052
:108B90009DFB02000B00414620000A604B6029004B
:108BA00002F02CFD034A044BB9E6032373E6C046EA
:108BB00061B4D03D7370032E8A19A33BF8B54746C4
:108BC000CE46674B80B50A000F00190005003940FA
:108BD000994200D19BE004000100002F69DD3F15A0
:108BE00000D1B4E05F4B12039C468023120B5B0361
:108BF00013435B00CA0F67449B184A00F80703D56C
:108C0000D20F5B009B188A0079108C4600218020CF
:108C10001624894680030D189D4202DC29185B1B2F
:108C20008144D50F5B00013C5B1952004008002CC9
:108C3000F1D100208046802020250027000609E091
:108C40008B425CD0D40F5B00013DE318520040081A
:108C5000002D16D0C4198B42F2DD27180E00002C0F
:108C600049DB5B1AA242894149425B1A121BD40FAD
:108C70005B00013D80443100E31852004008002DA4
:108C8000E8D113434ED143465B0837494A468846EC
:108C9000494652104244C90702D5802109060B43B8
:108CA00061460F05BD18180029000CBC9046994676
:108CB000F8BD7B005B0803433900002BF5D0002F83
:108CC0003CD1E30A153A6405002BFAD0802040031A
:108CD00003423FD1002700E00F005B00791C0342F4
:108CE000FAD0250020208D40401A2900D71B2200F1
:108CF000C2401A4376E7FE43F60F8E19B1E794425D
:108D0000A0D82718002CF6DB1E000023AEE70200D7
:108D10003B002800390002F0FFF92A003B0001F077
:108D2000D5FAC2E74346013303D0434601335B081B
:108D3000ABE7012398460023C144A6E73B000200AD
:108D400002F05CFC02000B0001F0DCFDADE713005B
:108D50000022BBE70127210020207F42C6E7C04652
:108D60000000F07F01FCFFFF0000E03FF0B5474648
:108D7000CE4680B587B000920193754B4F00814677
:108D800088467F089F4263DC02F09CFF002800D1E8
:108D9000D4E04A4643464846414602F0BDF9040045
:108DA0000D006C4A6C4B02F0B7F96C4A6C4B01F049
:108DB0008DFA22002B0002F0AFF96A4A6A4B02F0EA
:108DC0001DFC22002B0002F0A7F9684A684B01F055
:108DD0007DFA22002B0002F09FF9664A664B02F0F2
:108DE0000DFC22002B0002F097F9644A644B01F05D
:108DF0006DFA22002B0002F08FF9029003910022FD
:108E0000604B2000290002F087F9029A039B0600BC
:108E10000F002000290002F07FF9009A019B040056
:108E20000D004846414602F077F902000B00200091
:108E3000290002F0E3FB02000B003000390002F0D1
:108E4000DDFB02000B0000204F4902F0D7FB70E071
:108E500002000B0002F060F904000D003D4A3E4B99
:108E600002F05AF93D4A3E4B01F030FA22002B0045
:108E700002F052F93B4A3C4B02F0C0FB22002B00AF
:108E800002F04AF9394A3A4B01F020FA22002B004D
:108E900002F042F9374A384B02F0B0FB22002B00B7
:108EA00002F03AF9354A364B01F010FA2B00220055
:108EB00002F032F9354B029003919F429FDD344B13
:108EC00000229F423DDC334900207B182E491600CA
:108ED0001F0002F093FB049005910022294B200013
:108EE000290002F019F932003B0002F087FB029AD8
:108EF000039B06000F002000290002F00DF9009AE4
:108F0000019B04000D004846414602F005F90200AD
:108F10000B002000290002F071FB02000B00300062
:108F2000390002F06BFB02000B000498059902F077
:108F300065FB07B00CBC90469946F0BD0020124975
:108F4000F7E7154B002604920593144FC5E7C0467A
:108F5000FFFF3F3ED43888BEE9FAA8BDC4B1B4BD16
:108F60009EEE213EAD529C804F7E923E9015CB19D5
:108F7000A001FA3E7751C1166CC1563F4C5555556C
:108F80005555A53F0000E03F0000F03F3233D33F8E
:108F90000000E93F0000E0FF0000E73F0000D23F93
:108FA000F0B5DE464E4645465746E0B5DC4CA54496
:108FB0000D9114001900A49A0993DA4B9200D65827
:108FC0004D1E03901821E01E0696029500F0A0FEAB
:108FD000C3430100DB1719404B1C9A009B1ADB00AE
:108FE0001B190B9105934C1B771918D4A59BA50051
:108FF0009C463F1922AE6544013707E0286802F01D
:1090000097FE013403C60435BC4208D0002CF5DAC3
:1090100000200021013403C60435BC42F6D1069B72
:10902000002B01DA00F0FDFB069B03990133DB0006
:109030009A46099BDA00944600920022914672AA51
:109040000492B94A6144934688469AAB63449B4470
:10905000029B002B00DABCE15D4600260027039C42
:109060004D442A686B6803CC02F056F802000B00EE
:109070003000390001F02AF9083D06000F00444590
:10908000EFD1049B4B441E605F6008239C46E14483
:10909000D145DDD10EA804218446494261448C4665
:1090A000069A93009C44614684460A910399083BC2
:1090B00063448C460C93009B009263449B46009A49
:1090C0000498D10003008C46634408911E685F68D1
:1090D000002A33DD954980468C466244D30098448B
:1090E00070AB9A460EAB99460022914B3000390086
:1090F00002F012F802F0E6FD02F01AFE00228D4B9B
:1091000004000D0002F008F802000B0030003900E6
:1091100002F074FA02F0D6FD4B4601C3994643466D
:1091200020001A685B68290001F0D0F808235B4230
:109130009C46E04406000F00D045D5D1059B300089
:109140001A003900984600F0DFFCFF2300229B053F
:1091500004000D0001F0E0FF00F038FC0022764B27
:1091600001F0DAFF02000B002000290002F046FAAD
:109170000D00040002F0A6FD814602F0D9FD0200B8
:109180000B002000290002F039FA060040460F00CB
:10919000002800DCEEE0009B18215A1E92000EAB66
:1091A0009B58091A1D000D41A9448D405D1B0EAB53
:1091B0009D5017231B1A1D41002D2DDD01239C46B8
:1091C000009BE144002B00DC1CE20E9C0123002CE0
:1091D00000D0B5E0009A012A09D099000EAA54588F
:1091E0000133002C00D0ACE0009A9A42F5D1059BE7
:1091F000002B0EDD012B00D1A8E1022B09D1009B31
:109200000EA95A1E92000EAB9B5807939B029B0A15
:109210008B50022D00D1C1E0002300223000390024
:1092200000F080FE009B002800D194E2069A591EAF
:109230008A4210DC414A0A9894460EAA6344944636
:1092400000229B0063441C68043B22438342FAD102
:10925000002A00D0C0E0069B0EAA013B9B00D35819
:10926000002B00D0B3E001220C9B043B5968013273
:109270000029FAD0009B9C466244110007921A0014
:1092800001338B4246DC0B9863468046A59C4344E1
:10929000A046099C9B00A1464A449844D30022AAB8
:1092A0009146049A99449446089BA59A634484463F
:1092B000614494469A468B00634400934346586841
:1092C00002F036FD4B4618605960029B002B24DBF0
:1092D0004D46039C0026002701E0286869680CCCF5
:1092E00001F01AFF02000B003000390000F0EEFF21
:1092F000083D06000F005C45EFD153469E60DF60DD
:1093000004239C460433E0449C46009BE144E24431
:109310009845D3D1079B0093D1E600260027ECE7C0
:1093200094FDFFFF38ED000018FEFFFFFFFFFF1F59
:109330000000703E0000704100002040FFFFFF3F32
:10934000002180225204141B0EAA54500099994205
:109350000EDD0EA884469B000EAA8900D2586144F7
:109360006344CF4800E01A68821A04C38B42FAD1E2
:1093700001243CE7059B002B06D1009B0EAA013B74
:109380009B00D558ED1517E70022C64B300000F0C2
:10939000EDFD002800D024E100253DE732003B0030
:1093A0000020C14902F02AF906000F00002C00D16C
:1093B00032E7059A0020BC4900F0A6FB02000B0032
:1093C0003000390002F01AF906000F0024E70122EC
:1093D00050E70026002754E64B46059A0793884637
:1093E0008B000EA9CB58183A08950592002B0DD189
:1093F0008C464146AD4B43449B006344043B586854
:109400000139183A0028F9D088460592059A0020BB
:10941000A54900F079FB434604000D00002B00DA5B
:1094200005E29E000EAB9C464346DB0066449C462C
:10943000059370AB9946049F67440097306802F02B
:1094400077FC22002B0001F067FE00223860796073
:10945000974B2000290001F05FFE083F04000D003B
:10946000043EB945EAD14AAB03939B4600239A4692
:10947000069B4246994643460132029204934B466C
:10948000002B00DAAAE080208A4B009D9846C00598
:10949000894900260027002408E008239C46083557
:1094A000E044544511DC4346186859682A686B68E3
:1094B00001F032FE02000B003000390000F006FF20
:1094C000013406000F00A145E7DA5B46C0C39B46A6
:1094D00001239C46009BE244083B0093029B9A4573
:1094E000CDD1049B9846A49B022B00DD8EE0002B7F
:1094F00037DC1FD1059B00271D00039B00249C46E1
:109500001E006544083E2A686B683800210000F0A0
:10951000DDFE083D07000C00AE42F4D1089B002B95
:1095200003D080231B069C4664443A0023000D9917
:109530000A604B600720079B18409B239B009D44BB
:109540003CBC90469946A246AB46F0BD009B0EA996
:109550005A1E92000EAB9B5807935B025B0A8B501E
:1095600057E64346002B00DA70E100200021DB00C3
:109570004AAAD61848AF32687368083E00F0A6FEC3
:10958000B742F8D1089B002B00D025E10B00020068
:109590004A984B990D9C2260636002F02FF8434675
:1095A00007000C00002B13DD01254CAEB14638003E
:1095B0002E0021004C4601360CCC00F087FEA1465F
:1095C000B045F7DA089B07000C00002B00D015E12E
:1095D0003A0023000D998A60CB60ABE70026002794
:1095E00073E701239C46009BE1440225002B00DD2C
:1095F000EBE532003B0000202B4901F0FFFF0600A5
:109600000F0009E60024F2E54AAB0393A49B032B69
:1096100000D08FE74346002B00DC14E1039ADB0007
:109620009B46130091465B441E685F68234B43448E
:109630000293DB00994448AB9A464B465C681B6832
:109640001800210032003B000090019100F03EFE26
:1096500004000D0002000B000098019901F0CEFFFC
:109660003B00320000F032FE4B469860D9601C602F
:109670005D6008235B429C46E14426002F00CA45FA
:10968000DBD14346012B00DCE3E0039A13005B448B
:109690001E685F68029BDB0099464A44904610E0D2
:1096A000FFFFFF000000E03F0000F03FFFFFFF3F33
:1096B0000000703EF8EC0000FB21F93FFFFFFF1FA8
:1096C000984643465C681B681800210032003B0046
:1096D0000090019100F0FAFD04000D0002000B0063
:1096E0000098019901F08AFF32003B0000F0EEFD86
:1096F0004346039A9860D9601C605D60083B260071
:109700002F009A42DCD14D4694460026002447465D
:10971000083565442A686B683000210000F0D6FDEA
:10972000083D06000C00AF42F4D1039B4A9F5D68E0
:109730009968D868089B002B65D080221206944651
:109740000D9B6544604464441F605D609960D8600F
:109750001E615C61EEE69A464B460793059B30001E
:109760005A423900089500F0CFF900223A4B060022
:109770000F0000F0FBFB002824D0384B0022300003
:10978000390001F0C9FC02F09DFA52460400950030
:1097900002F0CEFA0022304B01F0BEFC02000B00BA
:1097A0003000390001F02AFF02F08CFA0EAA505165
:1097B0000122059B524418339046059393000EAA4C
:1097C000D45023E65346300039009C0002F07AFA68
:1097D0000EAB1851D04619E680230D9A1B06CB1804
:1097E000106053600B0002004A984B9901F006FF8D
:1097F000434607000C00002B00DDD5E680231B0646
:109800009C466444E4E62B003A000D9D2A606B60A0
:109810000A000300AA60EB60320023002A616B613A
:1098200088E6099BDB00009372AB049332E4A49BAF
:10983000022B00DDE8E6002B00DD92E600D079E6A1
:10984000002700246AE6002600246EE7002000219D
:1098500098E60026340068E7000070410000703E82
:10986000F0B5CE46474680B587B000920193474A8F
:109870004B00814688465B08934207DC41464846D8
:1098800002F020FA4146031E484666D04A46434647
:109890004846414601F040FC04000D0002000B0068
:1098A0004846414601F038FC394A3A4B06000F0061
:1098B0002000290001F030FC374A384B01F09EFEB1
:1098C00022002B0001F028FC354A364B00F0FEFC4C
:1098D00022002B0001F020FC334A344B01F08EFEB5
:1098E00022002B0001F018FC314B324A00F0EEFC54
:1098F0000E9B02900391002B34D000980199002216
:109900002D4B01F009FC029A039B04900591300055
:10991000390001F001FC02000B000498059901F0E8
:109920006DFE22002B0001F0F7FB009A019B01F075
:1099300065FE224A04000D00214B3000390001F081
:10994000EBFB02000B002000290000F0BFFC02002E
:109950000B004846414601F051FE07B00CBC904652
:109960009946F0BD02000B002000290001F0D4FB55
:10997000124A134B01F042FE32003B0001F0CCFBD7
:109980004A46434600F0A2FCE7E7C046FFFF3F3EE1
:109990007CD5CF5A3AD9E53DEB9C2B8AE6E55A3E79
:1099A0007DFEB157E31DC73ED561C119A0012A3F15
:1099B0001111813FA6F810110000E03F495555559F
:1099C0005555C53F49004B0819007047474AF0B547
:1099D0004F4691464B005B0D99444646D6464A4653
:1099E000C0B505000C000E0088460700132A27DCCE
:1099F000002A4BDB3E4B13419A460B005246134064
:109A0000034318D03B4A3C4B2800210000F05EFC89
:109A10000022002300F0A0FA002847D0002C04DA2E
:109A200080234A465B031341984446465346002729
:109A30009E43380031001CBC90469946A246F0BDBA
:109A4000332A08DD8023DB009945F4D102000B00A6
:109A500000F03CFCEFE7294A94460122634452425D
:109A6000DA4092460242E6D0224A234B28002100E7
:109A700000F02CFC0022002300F06EFA002815D024
:109A8000002C1EDB534646469F430FE0194A1A4BF3
:109A90002800210000F01AFC0022002300F05CFAEC
:109AA000002803D0002C04DB0027002638003100FA
:109AB000C1E76400640825430027002DF6D0104E4E
:109AC000F4E74B46142B0BD03422D21A01239340D7
:109AD0005D19BD4208D201239C462F00E044D1E726
:109AE000133B9C46E044CDE72F00CBE701FCFFFF92
:109AF000FFFF0F009C7500883CE4377EEDFBFFFF05
:109B00000000F0BF002070474B0070B55B0D1400E3
:109B10000A00002B1AD14B005B08034315D0234BDE
:109B2000002201F0F9FA224B9C422DDB0A004B0087
:109B30005B0D363B1F4DE318AB422ADC002B0DDDDD
:109B40001D4C1B0522401A43110070BD1B4DAB423A
:109B5000F0D102000B0000F0B9FBF6E71D0035352F
:109B600019DA174B02009C4209DD0B001548164913
:109B700000F032F8134A144B01F0CEFAE5E70B007F
:109B80001248134900F028F8104A114B01F0C4FAAA
:109B9000DBE70200E9E7084C363322401B0513439C
:109BA000190000220B4B01F0B7FACEE7000050433A
:109BB000B03CFFFFFE070000FFFF0F80FF07000023
:109BC00050C300009C7500883CE4377E59F3F8C20E
:109BD0001F6EA5010000903C30B54A00DB0FDB078B
:109BE00052081A43110030BD02B4714649084900B9
:109BF000095C49008E4402BC7047C04600224308FD
:109C00008B4274D303098B425FD3030A8B4244D344
:109C1000030B8B4228D3030C8B420DD3FF22090286
:109C200012BA030C8B4202D31212090265D0030B45
:109C30008B4219D300E0090AC30B8B4201D3CB033B
:109C4000C01A5241830B8B4201D38B03C01A52417D
:109C5000430B8B4201D34B03C01A5241030B8B427F
:109C600001D30B03C01A5241C30A8B4201D3CB026A
:109C7000C01A5241830A8B4201D38B02C01A52414F
:109C8000430A8B4201D34B02C01A5241030A8B4252
:109C900001D30B02C01A5241CDD2C3098B4201D36A
:109CA000CB01C01A524183098B4201D38B01C01AE8
:109CB000524143098B4201D34B01C01A524103095F
:109CC0008B4201D30B01C01A5241C3088B4201D30E
:109CD000CB00C01A524183088B4201D38B00C01ABB
:109CE000524143088B4201D34B00C01A5241411AE2
:109CF00000D20146524110467047FFE701B50020EF
:109D000000F0F0F802BDC0460029F7D076E77047B2
:109D100003460B437FD4002243088B4274D30309CC
:109D20008B425FD3030A8B4244D3030B8B4228D36D
:109D3000030C8B420DD3FF22090212BA030C8B4293
:109D400002D31212090265D0030B8B4219D300E033
:109D5000090AC30B8B4201D3CB03C01A5241830BB8
:109D60008B4201D38B03C01A5241430B8B4201D368
:109D70004B03C01A5241030B8B4201D30B03C01A91
:109D80005241C30A8B4201D3CB02C01A5241830A0B
:109D90008B4201D38B02C01A5241430A8B4201D33A
:109DA0004B02C01A5241030A8B4201D30B02C01A64
:109DB0005241CDD2C3098B4201D3CB01C01A5241CB
:109DC00083098B4201D38B01C01A524143098B4254
:109DD00001D34B01C01A524103098B4201D30B013D
:109DE000C01A5241C3088B4201D3CB00C01A524162
:109DF00083088B4201D38B00C01A524143088B4227
:109E000001D34B00C01A5241411A00D201465241BF
:109E1000104670475DE0CA0F00D04942031000D3DE
:109E20004042534000229C4603098B422DD3030A33
:109E30008B4212D3FC22890112BA030A8B420CD343
:109E4000890192118B4208D3890192118B4204D36C
:109E500089013AD0921100E08909C3098B4201D3EC
:109E6000CB01C01A524183098B4201D38B01C01A26
:109E7000524143098B4201D34B01C01A524103099D
:109E80008B4201D30B01C01A5241C3088B4201D34C
:109E9000CB00C01A524183088B4201D38B00C01AF9
:109EA0005241D9D243088B4201D34B00C01A5241D0
:109EB000411A00D20146634652415B10104601D35D
:109EC0004042002B00D54942704763465B1000D3E7
:109ED000404201B5002000F005F802BD0029F8D08D
:109EE00016E770477047C046D0400B1C1141203A1E
:109EF00003D49C461341184363465242934018438F
:109F00007047C0468446101C62468C46191C634646
:109F100000E0C0461FB501F097F8002801D40021E9
:109F2000C8421FBD10B500F0EFFF4042013010BD28
:109F300010B501F089F8002801DB002010BD0120D8
:109F400010BDC04610B501F07FF8002801DD0020EB
:109F500010BD012010BDC04610B501F011F8002859
:109F600001DC002010BD012010BDC04610B501F07D
:109F700007F8002801DA002010BD012010BDC046FE
:109F8000F0B5CE46474615042D0C2E0080B50704CB
:109F9000140C3F0C9946030C7E435D4367436343B7
:109FA0007F19340CE4199C46A54203D980235B0237
:109FB0009846C4444B4643435143250C36046544FC
:109FC000360C2404A4195B19591820000CBC9046C7
:109FD0009946F0BDF0B54E4657464546DE46E0B5DB
:109FE00043025B0A450083B00F1C99462D0EC60F35
:109FF000002D57D0FF2D24D08020DB00C004184353
:10A00000002381469A469B467F3D7C027A00FB0FE7
:10A01000640A120E984623D0FF2A4BD0E300802416
:10A020000020E4047F3A1C43AD186B1C47460193A3
:10A03000534677403A000F2B48D87D499B00CB58B8
:10A040009F46002B00D085E008339A46063B9B468E
:10A050007C027A00FB0FFF25640A120E9846DBD1C2
:10A06000002C00D090E0524601231A439246012072
:10A07000DBE74C4658461700022824D0032800D1BD
:10A08000CFE00022002301284DD15802D205400A1A
:10A09000FF071043384303B03CBC90469946A246A4
:10A0A000AB46F0BD002B5BD104239A46033B002551
:10A0B0009B46AAE7FF35002C60D1524602231A4383
:10A0C00092460220B1E7FF220023DEE74B461B0C3D
:10A0D0009C464B462604360C180461463300220C7D
:10A0E0006446000C43434E435043544380191A0CBA
:10A0F0001218964203D9802149028C4664441B04FD
:10A100001B0C1004C01883015E1EB341800E18435F
:10A11000130C1B199B0103431C00230179D5012358
:10A1200062081C401443019A7F32002A4DDD630708
:10A1300004D00F232340042B00D00434230103D583
:10A140003C4B019A1C408032FE2ABCDCA3015B0A16
:10A15000D2B29AE70C239A46093BFF259B4654E767
:10A16000180001F071FE4A46431F76259A400023ED
:10A170006D4291462D1A9A469B4646E75246032366
:10A180001A439246032050E7200001F05DFE431F72
:10A190002D1A9C40763D002047E780230027DB03F3
:10A1A000FF2272E7424666E74C463200584662E7B5
:10A1B00080234A46DB031A4222D01C4220D123438B
:10A1C0005B025B0A4746FF225FE701239A1A1B2ABC
:10A1D00021DC23000199D3409E318C401A002300DA
:10A1E0005C1EA34113435A0704D00F221A40042ACD
:10A1F00000D004335A0111D49B015B0A002244E7CA
:10A2000080234A46DB0313435B025B0A3700FF22CD
:10A210003BE7019587E70022002336E70122002370
:10A2200033E78023DB0323435B025B0AFF222CE737
:10A2300048ED0000FFFFFFF770B500283DD0C317C1
:10A24000C5185D40C40F280001F0FEFD9E22121AC1
:10A25000962A07DCD2B2082833DD08388540680228
:10A26000400A23E0992A0BDD052329001B1AD94057
:10A2700003001B339D402B005D1EAB4119430D00B5
:10A28000052801DD431F9D402B000F490B406E0741
:10A2900009D00F263540042D05D004335D0102D5C9
:10A2A0009F220B40121A9B01580AD2B24002D205DB
:10A2B000400AE4071043204370BD00240022002020
:10A2C000F4E76802400AF1E7FFFFFFFBF0B54F46F5
:10A2D0004646D6460C000903C0B5490A470F5E0042
:10A2E00039431F03DB0F9C4665007B0A570F1F4352
:10A2F0006D0DE40F760DA146C000B846D200AB1B31
:10A3000064457BD0002B5FDD002E00D0A4E03E0032
:10A31000164300D112E15E1E002E00D09EE1871A86
:10A320004346B84280410125C91A4042091A0B022E
:10A3300000D431E149024E0A002E00D16EE1300016
:10A3400001F082FD0300083B1F2B00DD61E12022AC
:10A350003900D21A9E40D1409F400E439D4200DDFD
:10A3600051E15D1B6B1C1F2B00DD7CE12021C91A14
:10A370003D0030008F408840DD40791E8F41310024
:10A3800007222843D940002507433A40002A09D034
:10A390000F233B40042B05D03B1DBB42BF417F42F6
:10A3A000C9191F000B0200D426E26A1CC64B5505D2
:10A3B0006D0D9A4200D106E1C44AFF080A405307D6
:10A3C00052023B43120B8EE0002B00D0B8E06B1C16
:10A3D0005B055B0D012B00DC30E1871A4346B84278
:10A3E000B641CB1A76429E1B330200D54CE13B00AE
:10A3F0003343A1D100220024002570E0002B00DCB3
:10A40000E5E0002E00D183E0AF4EB54260D080265B
:10A4100036043743B846382B00DC3EE1434613434D
:10A420001F007A1E97413F18874280414042091819
:10A430000B0200D4B0E0A44B01359D4200D1C3E033
:10A44000A24A7B080A4001210F401F435108D3074D
:10A4500007221F433A4099E79B4EB54238D08026E9
:10A4600036043743B846382B00DDDCE01F2B00DC18
:10A4700030E11E004746203EF740BC46202B04D06A
:10A480004026F31A46469E403243170063467A1E22
:10A4900097411F43CCE0002B00D104E24346134315
:10A4A00000D159E14B07C00818438023C9081B039A
:10A4B000194208D04546ED081D4204D14346D00854
:10A4C000590708432900420FC9007F4D1143C000BE
:10A4D0004B07CA087C49C00803438D4268D0120369
:10A4E0006D05120B6D0D002112031800130B0A0DE0
:10A4F00012051A43764B2D0513402B435B00E407EE
:10A500005B08234319001CBC90469946A246F0BD47
:10A510003E00164312D05E1E002E00D000E18718C8
:10A520008742804141444042091801250B0233D53E
:10A53000022585E764463300414610001D00C7E749
:10A54000002D00D0DAE00C000443F3D05C1C00D1F5
:10A550009FE15D4CA64200D12FE1DB43382B00DDAB
:10A5600066E11F2B00DD83E120240500E41A0F00C3
:10A57000DD40D940A0404346A7405B1A441EA0419D
:10A5800098462F433843171ABA42924143465242E3
:10A59000991A64463500CAE607223A40002A00D0DC
:10A5A000F6E64B07CA084849FF083B438D4296D15F
:10A5B0001900114300D19EE1802109030A431203CF
:10A5C000120B414D8FE71500002200238BE7002B73
:10A5D00000D0C7E06B1C5F057F0D012F00DCF1E0B0
:10A5E000394DAB4200D1B9E085180A008542894156
:10A5F0004244494251180722CF076D082F434908AA
:10A600003A401D00C2E607223049ED1A31403A4077
:10A61000BCE63E002838864000279FE6380001F05F
:10A6200013FC20308EE6434613431F007A1E9741E9
:10A63000C71BB84280414042091A78E60E003B0031
:10A6400006431343002D61D1002E00D0F4E0002B0F
:10A6500000D11BE164463900100039E71A4FBB42B4
:10A660007AD03300FFE630001F3DE840202B03D0B6
:10A670004021CB1A9E4037437B1E9F410722074350
:10A680003A400021002589E7171A4346BA42B641ED
:10A69000591A76428E1B64464EE61F2B00DDADE054
:10A6A00020264746F61AB740B9461700B246DF40A3
:10A6B0004E463E4337005646B240561EB2411743FF
:10A6C0004246DA408918AEE6FF070000FFFF7FFF31
:10A6D000FFFF0F8020264746F61AB740B9461700FD
:10A6E000B246DF404E463E4337005646B240561E05
:10A6F000B24117434246DA40891A99E77F4CA64295
:10A700005BD0802424045B42214327E7002E0CD138
:10A71000002B00D1CBE0644639001000774DD7E61E
:10A72000764FBB4218D0330075E6002B14D04B0790
:10A73000C00818438023C9081B03194207D0FC082E
:10A740001C4204D17907D0080843E14621004C4659
:10A75000420FC9001143C000684DB9E61D00002238
:10A760000023C0E6002D5BD10D00054300D1E2E6D9
:10A770005D1C00D1B0E0614DAE421FD0DB43382BF1
:10A7800071DC1F2B00DD96E020250F00ED1AAF4095
:10A79000B9460700AA46DF404D463D432F005546C7
:10A7A000A840D940451EA84188440743BF18974296
:10A7B00092415142414435003AE6644635004146F3
:10A7C000100085E60B000343002D00D063E6002B4C
:10A7D000F5D04346134300D17AE68718874280417B
:10A7E00007224144404209183A400B0200D4D5E602
:10A7F000434B01351940C9E5380069E61E0047465C
:10A80000203EF740BC46202B04D04026F31A464693
:10A810009E403243170063467A1E97411F4302E66B
:10A82000364DAE42CAD080252D045B422943A6E7AF
:10A830000843411E8841A6E6002B00D148E6871A4E
:10A840004346B842B641CB1A76429E1B33024BD5E3
:10A85000171A4346BA429241591A5242891A07229C
:10A8600064463A4092E501430F00791E8F419DE70F
:10A870001C000F00203CE740202B03D04024E31AAB
:10A8800099400843411E884138437CE60022002459
:10A8900025E6171A4346BA429241591A5242891A7A
:10A8A0006446350043E541461000144D10E6802211
:10A8B0000024120380E61D000F00203DEF40BC463F
:10A8C000202B03D04025EB1A99400843070063462C
:10A8D000781E87411F4369E7871897429B4141448F
:10A8E0005B42C9183500A3E53B003343CED00722B5
:10A8F00031003A4052E600231A00F4E5FF07000059
:10A90000FFFF7FFFF0B55746DE464E464546E0B5B1
:10A91000834607000E03480085B092461C00360BA4
:10A92000400DCD0F002800D19DE0954B984239D0C5
:10A930008023F6001B041E43924A7B0F3343994643
:10A94000944603006344009300230026FF00029313
:10A9500023031B0B98466300E40F52465B0D0194E2
:10A9600000D1B3E086498B4200D19EE04246D1003F
:10A97000802212040A435146490F11438B468149F4
:10A9800052468C4600996344CB1A0021D2000093B2
:10A990002B0063409A460F2E00D905E17A4BB60092
:10A9A0009B599F465B463343994600D0B8E002234B
:10A9B0000826002700900293CAE7CB463A00029986
:10A9C0000195019B9A46022927D0032900D180E2F4
:10A9D000012944D06D49009B8C4663441C00002C27
:10A9E00038DD530700D013E2D2085B46DB0109D5FE
:10A9F0005946674B19408B468021C9008C46009B05
:10AA000063441C00634B9C4207DC5B4664055F07A4
:10AA10005B0217431B0B620D02E000230027584A1C
:10AA200000211B031C0B0B0D1B05234314055A4A65
:10AA3000380013401C4353466400DB0764081C4382
:10AA4000210005B03CBC90469946A246AB46F0BDFD
:10AA50000122524201231B1B382B00DCADE10022F6
:10AA600000230027DCE75B46334399465ED0002E87
:10AA700000D18AE1300001F0E7F903000B3B1C2B09
:10AA800000DD7BE11D22D31A5A460100DA40083965
:10AA90008E4013005F46334399468F403F4B00265C
:10AAA0001B1A00930023029352E7414653460B437F
:10AAB0003B499B468C46009B634400935B46002BBE
:10AAC0003BD1022300221E43022161E74346134388
:10AAD0009B4637D04346002B00D162E1404601F04F
:10AAE000B3F903000B3B1C2B00DD53E10200414690
:10AAF000083A914088461D21CB1A5146D9400B0097
:10AB000041460B439B46534693401A00009B254900
:10AB10009C46604403008C4663440093002137E761
:10AB20000323B14600900C26029311E70023009303
:10AB300001330426002702930AE70323C3461E437A
:10AB4000032125E701331E430022012120E70023D2
:10AB50009A46802300271B03094A61E78023494660
:10AB60001B03194200D1E2E05946194200D0DEE051
:10AB70000B431B0317001B0BA246014A50E7C046BC
:10AB8000FF07000001FCFFFF88ED0000FF0300004D
:10AB9000FFFFFFFEFE070000FFFF0F800DFCFFFF21
:10ABA00001F8FFFFF3030000D94500D9CBE000D145
:10ABB000C6E03C0048460027009B013B00935B46F3
:10ABC000160E1B021E431302984633041B0C9946B3
:10ABD000310C0191FFF798F84A4642430B04210CCF
:10ABE000050019438A4207D98919013D8E4203D8CD
:10ABF0008A4201D9851E8919881A0199FFF784F8BC
:10AC000009048C464A46210464464243090C030069
:10AC100021438A4204D98919013B8E4200D8F1E0D0
:10AC20002D041D43AB464346891A4246280C1204A4
:10AC30001D0C5B46140C22001B041B0C5A4303948E
:10AC40006B434443029568431B19150CEB189C4257
:10AC500003D980246402A44660441C0C15041B0420
:10AC60002D0C20185D19814277D373D00C1AA24A9B
:10AC70007D1BAF42BF419446009B7F426344E01B73
:10AC80001C00864200D1DBE00199FFF73DF84A46FF
:10AC900042430B04290C070019438A4207D989193A
:10ACA000013F8E4203D88A4201D9871E8919881A2A
:10ACB0000199FFF729F809044A46894629044D46B7
:10ACC0004243090C030029438A4207D98919013BF1
:10ACD0008E4203D88A4201D9831E89193F04891AFA
:10ACE0003A00039F1A43380013041B0C5843814653
:10ACF0000298150C6F43434345434846000C844675
:10AD0000DB1963449F4203D9802040028446654496
:10AD100048461F0C00041B04000C7D191818A9429A
:10AD200000D284E000D17FE001231A4357E680235C
:10AD30004A461B0313431B031B0BAA466F4A6FE6CD
:10AD4000BA4200D935E74B46DC0758087B081C435C
:10AD5000FF0734E70024AF4289D247444745A44166
:10AD60005B466442A4196418013BA6421ED2A0426D
:10AD70006DD800D1B6E0241A9B4678E703005A4606
:10AD8000283B9A400027914688E6584601F05CF837
:10AD9000203072E603005246283B9A409346002238
:10ADA000B4E6504601F050F820309AE6A642E2D1CF
:10ADB000B845DCD9341A9B4659E71F2B65DC504C4B
:10ADC0000099A4465C46614408008C401100824012
:10ADD000D940501E82410C4314435A46DA401300B6
:10ADE000620709D00F222240042A05D02200141D38
:10ADF0009442894149425B181A0262D5012200231C
:10AE000000270DE68A4200D80AE7831E891907E762
:10AE10000F231340042B00D1E6E5171D9742924102
:10AE200053429B44FA08E0E5002800D1D7E57118A9
:10AE3000531EB14227D3A94215D358D01A0073E745
:10AE4000002B00DC04E6012300229B44CDE5022315
:10AE50004744474589415B429C46494289190C1940
:10AE6000E344241A03E743465F0047459B41B84645
:10AE70005B429E19023A8919A94200D054E7404525
:10AE800000D051E7ABE51A00F6E71F215F464942C3
:10AE90000C1BE740202B07D01A49009B8C466344CB
:10AEA00018005B4683401A43501E82413A430727ED
:10AEB0000023174009D00F2100231140140004295A
:10AEC00095D122005F075B021B0BD20817430022BB
:10AED000A6E5802359461B030B431B0317001B0BDE
:10AEE000064A9DE5BD42B2D89B460024BFE6804598
:10AEF000B9D31A00C3E7C046FF030000FF070000F4
:10AF00001E0400003E040000F0B54F464646D646FB
:10AF10008446C0B58046194E18030F034D00000B40
:10AF20005C0082463F0B6D0DC90F9146640DDB0F2F
:10AF30000120B5420AD0B44203D0A54201D1574501
:10AF40000CD01CBC90469946A246F0BD66463E43D6
:10AF5000F7D1AC42F5D154461443F2D10120C84593
:10AF6000EFD1994207D0002DEBD163461F43380043
:10AF7000471EB841E5E70020E3E7C046FF070000B1
:10AF8000F0B54F464646D6464D00C0B50E03C90F34
:10AF90008A462C491F035C008046360B6D0D914696
:10AFA0003F0B640DDB0F8D421ED08C4216D0002D5E
:10AFB0001ED130438446002C01D13A4323D062464F
:10AFC000002A1AD09A4529D051460220013908405A
:10AFD00001381CBC90469946A246F0BD3900114389
:10AFE000E5D002204042F4E73043FAD1AC420FD022
:10AFF000002C0FD13A43E7D00CE00122013B9343F0
:10B0000018000130E5E763460020002BE1D0DBE7C4
:10B010003A43E6D19A45D7D1A542D5DCA54205DB16
:10B02000BE42D1D808D00020BE42D2D25046012321
:10B03000013898430130CCE7C845C5D80020C84541
:10B04000F4D3C6E7FF070000F0B54F464646D646A4
:10B050004D00C0B50E03C90F8A462E491F035C0080
:10B060008046360B6D0D91463F0B640DDB0F8D4214
:10B0700018D08C4211D0002D18D130438446002CBA
:10B080001ED13A431CD163460020002B30D05146DC
:10B0900002200139084001382AE039001143EAD082
:10B0A000022025E03043FBD1AC4226D0002C26D133
:10B0B0003A4324D15146022001390840013817E0B3
:10B0C0006246002A0FD09A45E1D1A54205DBBE4277
:10B0D000DDD819D00020BE420AD2504601230138E3
:10B0E0009843013004E00122013B934318000130F2
:10B0F0001CBC90469946A246F0BD3A43D0D19A4531
:10B10000C5D1A542C3DCE0E7C845C0D80020C8458A
:10B11000E3D3EDE7FF070000F0B55746DE464E46A5
:10B120004546E0B5834606000F03480087B09246C7
:10B130001D003F0B400DCC0F002800D16FE0DE4B0F
:10B14000984238D08023FF001B041F43730F3B43FA
:10B150000193DA4B0027994600239B46F600814471
:10B160002B0369001B0B52469846490DED0F002931
:10B1700000D185E0D04B994200D173E04346DA001C
:10B1800080231B0413435246CC48520F844613437A
:10B19000524600206144D200894421006940009158
:10B1A0008C46012149448A460F2F00D990E0C449BA
:10B1B000BF00CF59BF465B463B43019300D06AE1D5
:10B1C00002230827002681469B46C9E732005846DD
:10B1D000019B61460091022800D175E0032800D14F
:10B1E000FEE1012800D02CE10023002700260025E5
:10B1F0003F032A0D3F0BB34812053A4302401B059B
:10B200001343009A5B00D1075B080B433000190021
:10B2100007B03CBC90469946A246AB46F0BD5B46A3
:10B220003B43019300D12FE1002F00D1A5E138006D
:10B2300000F00AFE03000B3B1C2B00DD96E11D22F3
:10B24000D31A5A460100DA405E4608398F4013008F
:10B250008E403B4301939C4B00271B1A99460023C9
:10B260009B467DE7414653460B4393498C46E14458
:10B27000002B00D01AE102220220174300228CE7A3
:10B28000134300D10DE14346002B00D181E140463C
:10B2900000F0DAFD02000B3A1C2A00DD72E1010029
:10B2A000434608398B4098461D239A1A5346D3408B
:10B2B0001A004346134352468A404946081A8249B7
:10B2C00089468144002068E77B4B002700268EE7F3
:10B2D000140C1204120C1100370C3604350C79438F
:10B2E00028008C462E00604360448346564321006C
:10B2F000300C80465846794340440291844506D933
:10B300008846802149028C46E04441460291360439
:10B31000010C360C00048B4681191E0C1B041B0CFF
:10B320000391190079438C46280075436544A8466B
:10B330005843050C45447743A94203D9802149026B
:10B340008C466744290C8C4639000004000C2D04FF
:10B350002D186144AB4405915946049101990F049D
:10B360003F0C080C390051434243904602008C4682
:10B37000090C8B4662437C4344445C44A04503D99A
:10B380008021490288464244210C884661460904CE
:10B39000090C8C4639005943434370437E430F0CDC
:10B3A000F6182404BE19644442448C46B34203D9BF
:10B3B00080235B0298464044029B61469846049B6A
:10B3C000370443449B46AB45AD416B420D040599A0
:10B3D0002D0C8C467F196744FD18A8465D462D1933
:10B3E000A542A44193466442A446C344DC448F4230
:10B3F000BF4198459B4193459241A445A4415B427E
:10B400007F421F43360C52426442BF192243BF1889
:10B41000624638184302D20D039913436A020A4365
:10B42000501E82416146ED0D2A434E023243D9013E
:10B4300000D4B3E00126500832400243DE07324315
:10B440005B08224C5444002C62DD510709D00F20C8
:10B450001040042805D0101D9042924152429B1882
:10B460000200D90104D580241948E4000340544463
:10B470001848844200DD27E75E075B02D2081F0BF5
:10B48000630516435B0DB2E600239946013304279A
:10B4900000269B4664E60323019781460C279B46C2
:10B4A0005EE6012201201743002276E603230320F3
:10B4B0001F43434671E6C046FF07000001FCFFFF43
:10B4C000C8ED0000FFFF0F800DFCFFFFFF03000031
:10B4D000FFFFFFFEFE0700000023802700933F03CD
:10B4E0000026434B83E6019B3200A446584670E693
:10B4F000AC466EE6802701993F0339422DD03B428E
:10B500002BD11F433F033F0B00951600384B6EE6CF
:10B5100001252D1B382D00DD66E61F2D40DC35484A
:10B520001C005044160082408440EE40501E824170
:10B5300034431443EB40620709D00F222240042A0F
:10B5400005D02200141D9442804140421B181A026B
:10B550003ED501230027002649E68027019B3F03B3
:10B560001F433F033F0B0094214B40E603005A4624
:10B57000283B9A40002601926DE6584600F064FC94
:10B58000203057E603005246283B9A401300002221
:10B5900093E6504600F058FC20307BE6CA4650E760
:10B5A0001F201E004042041BE640202D03D0124CF9
:10B5B0005444A3401A43501E8241324307260027B9
:10B5C000164009D00F200023104014000428B9D1E0
:10B5D00022005E075B021F0BD2081643002306E61B
:10B5E00080273F031F433F033F0B1600004BFEE540
:10B5F000FF0700001E0400003E040000F8B5574697
:10B600004E464546DE460C000903E0B5490A460FA2
:10B610005F0031431E03DB0F760A9B46530F334313
:10B62000C84E6500C000E40FD2006D0DA2468146F1
:10B630007F0D9C469046B74200D1B9E05B4601269B
:10B6400073409B46EE1BA34500D183E0002E63DDD3
:10B65000002F00D0B1E06346134300D123E1731EF5
:10B66000002B00D0BAE1861A6346B0428041012522
:10B67000C91A4042091A0B0200D447E149024B0A99
:10B6800098464346002B00D189E1404600F0DCFBA0
:10B690000300083B1F2B00DD7CE120223000D21A82
:10B6A0004146D040994002009E400A439D4200DD41
:10B6B0006AE15D1B6B1C1F2B00DD94E12021100053
:10B6C0003500C91A8E40DA408840DD40711E8E4137
:10B6D000110007222843002506433240002A09D0E2
:10B6E0000F233340042B05D0331DB342B6417642BD
:10B6F00089191E000B0200D43DE26A1C914B5505CE
:10B700006D0D9A4200D119E18F4AF6080A40570799
:10B7100052023743120B9BE0002E00D0C5E06E1C96
:10B720007605760D012E00DC48E16746861ACB1BB4
:10B73000B042BF417F42B8461F004346FF1A3B005C
:10B74000B8461B0200D55FE137439AD1002200249E
:10B75000002579E0002E00DCFAE0002F00D18DE01A
:10B76000784B9D4267D0802367461B041F43BC462D
:10B77000382E00DC52E1634613435A1E93411E18D3
:10B7800086428041404209180B0200D4BEE06D4B56
:10B7900001359D4200D1D2E06B4A73080A40012175
:10B7A0000E401E435108D30707221E43324095E73F
:10B7B0001E00164300D045E740E7624B9D423AD059
:10B7C000802367461B041F43BC46382E00DDEBE098
:10B7D0001F2E00DC3AE133006746203BDF403B0090
:10B7E000202E05D04027BF1B6646BE403243904600
:10B7F0004646721E96413343DAE0002B00D114E234
:10B800006346134300D168E180234E07C008C9088E
:10B810001B030643194208D06046C008184204D1F1
:10B8200063460100D2085E071643F3009946C9003B
:10B83000720F444D11434B46DE08424B4F073743CE
:10B84000CA089D4200D16EE012036D05120B6D0D0A
:10B8500000211203130B0A0D12051A433B4B2D0551
:10B8600013402B435B00E4075B08234338001900B7
:10B870003CBC90469946A246AB46F8BD634613438E
:10B8800011D0731E002B00D007E18618864280413C
:10B8900061444042091801250B0237D502257BE798
:10B8A0003E00614691463500C5E75C46002D00D05C
:10B8B000E1E00B000343F3D0731C00D1ACE1214B5A
:10B8C0009F4200D13AE1F343382B00DD6FE11F2B9B
:10B8D00000DD8CE120250E00ED1AAE40B0460600DA
:10B8E000AA46DE40454635432E005546D940A8407D
:10B8F0006346451EA8415B1A9C463043161AB24265
:10B90000924163465242991A3D00B4E60722324002
:10B91000002A00D0E4E60B4BF6084F073743CA086D
:10B920009D4200D090E73B00134300D1A6E1802365
:10B930001B031A431203120B024D89E71500002264
:10B94000002785E7FF070000FFFF7FFFFFFF0F8055
:10B95000002E00D0C7E06B1C5E05760D012E00DCCA
:10B96000F0E0C84DAB4200D1B9E085180A0085422D
:10B9700089416244494251180722CE076D082E437F
:10B98000490832401D00A9E6BF49ED1A11400722BF
:10B990003240A3E6320028388240002686E6300096
:10B9A00000F052FA203073E6634613435A1E934167
:10B9B000C61AB04280414042091A5CE60E00674652
:10B9C00006431743002D5ED1002E00D0F3E0002F78
:10B9D00000D11EE15C46614691462CE7A94FBE426C
:10B9E0007BD01E00F1E610001F3DE840202B03D065
:10B9F0004021CB1A9A401643731E9E4107220643EC
:10BA000032400021002583E7161A6346B242804186
:10BA1000591A40420B1A98465C4632E61F2E00DD4A
:10BA2000ABE02027BB1B9A4663465746BB4099466E
:10BA300013004F46F3401F433B005746BA40571E82
:10BA4000BA4113436246F240891898E62027BB1B8F
:10BA50009A4663465746BB40994613004F46F3400B
:10BA60001F433B005746BA40571EBA411343624634
:10BA7000F240891A9CE7834B9F425FD080252D04BA
:10BA80007342294320E7002E0CD1002F00D1D0E0D3
:10BA90005C46614691467B4DCDE67A4FBE421CD056
:10BAA0001E0065E6002F18D0C0084E070643802010
:10BAB000C9080003014208D06346DC08044204D1EF
:10BAC0002100DA46D2085E071643F30099460124A6
:10BAD0005346C900720F11431C406A4DABE61D006E
:10BAE00000220027B4E6002D59D10B00034300D1FA
:10BAF000D6E6731C00D1B2E0624B9F421ED0F343E6
:10BB0000382B6FDC1F2B00DD97E020250E00ED1A8F
:10BB1000AE40B0460600AA46DE40454635432E00FC
:10BB20005546A840D940451EA8418C440643B61846
:10BB300096429241514261443D0025E63D006146F6
:10BB4000914678E60B000343002D00D055E6002B0C
:10BB5000F5D06346134300D16DE6861886428041D6
:10BB600061444042091800220B0200D4D0E6464B43
:10BB700001351940B2E5B1465DE633006746203B2A
:10BB8000DF403B00202E05D04027BF1B6646BE404D
:10BB9000324390464646721E96413343EFE5394B99
:10BBA0009F42CBD080252D0473422943A8E7084348
:10BBB000411E8841A2E6002F00D13CE66346861A6A
:10BBC000CF1AB0429B415B42FB1A98461B024ED5EE
:10BBD000161A6346B2429241591A5242891A5C4679
:10BBE00000227BE501430E00711E8E419FE71D0080
:10BBF0000E00203DEE40B046202B04D04025EB1A2D
:10BC000099400843814648464346411E88411843AF
:10BC100074E60022002417E6161A6346B2429241E7
:10BC2000591A5242891A3D0025E561469146154D43
:10BC300001E680220024120379E61D000E00203D5B
:10BC4000EE40B046202B04D04025EB1A9940084323
:10BC500081464E464346711E8E411E4367E7861855
:10BC600096429B4161445B42C9183D008CE54746C2
:10BC70003743CED007224146324049E600273A00FA
:10BC8000E6E5C046FF070000FFFF7FFF70B50C4EE2
:10BC90000D031C0349005B002D0B490D240B5B0DAC
:10BCA000B14208D0064900208B4203D11443200042
:10BCB000441EA04170BD05430120002DFAD1F1E7DB
:10BCC000FF07000030B5144D0A034B00120B5B0D4B
:10BCD000C90F0024AB4211DD104CA34210DC8024BC
:10BCE000640322430E4CE41A1F2C0CDD0D48C31ACA
:10BCF000DA4013005C42002900D11C00200030BD56
:10BD0000094BCC18FAE7094DE040AC4663449A4031
:10BD100013000343EEE7C046FE0300001D040000CD
:10BD20003304000013040000FFFFFF7FEDFBFFFF63
:10BD300070B500282DD0C317C5185D40C40F28006A
:10BD400000F082F8154B1B1A5B055B0D0A2815DD08
:10BD50000B38854000222D032D0B002110002D03F0
:10BD60000A0D2D0B12052A430D4D1B052A401343C6
:10BD70005B00E4075B082343190070BD0200290043
:10BD8000153291400A000B21081AC5402D032D0BD6
:10BD9000E3E70024002300250022DEE71E04000064
:10BDA000FFFF0F804100090E4B1C70B5DBB246024D
:10BDB000750AC40F012B14DDE0239B006D07360BC1
:10BDC000CB1800210A0D280012051C4D32435B05DB
:10BDD0002A405B0813435B00E4075B082343190018
:10BDE00070BD002914D1002D1ED0280000F02CF8C1
:10BDF0000A281CDC0B232A001B1ADA400300153327
:10BE00009D400F4B12031B1A5B05160B5B0DD8E709
:10BE1000002D06D0320B802636036D071643094BE2
:10BE2000CFE7084B0026CCE700230026C9E7030034
:10BE30002A000B3B9A400025E3E7C046FFFF0F8036
:10BE400089030000FF0700001C2101231B04984206
:10BE500001D3000C10391B0A984201D3000A08399B
:10BE60001B09984201D30009043902A2105C401852
:10BE70007047C046040302020101010100000000F6
:10BE80000000000030B51C00094B05001B6885B0A0
:10BE9000D868084B002A01D1074B1A00029201937F
:10BEA00000912B002200054900F026F800F0A6FDC5
:10BEB0008800002008EE000006DB000015EE000000
:10BEC000014B18687047C04688000020084B10B529
:10BED0000400002B02D0002100E000BF054B1868D1
:10BEE000836A002B00D09847200001F05DFBC0461C
:10BEF0000000000044EE00000EB403B5010003ABE7
:10BF0000044804CB0068019300F076F802B008BC46
:10BF100003B018478800002070B500260C4D0D4C6A
:10BF2000641BA410A64209D1002601F03FFB0A4D74
:10BF30000A4C641BA410A64205D170BDB300EB5897
:10BF400098470136EEE7B300EB5898470136F2E721
:10BF500058020020580200205802002068020020E9
:10BF6000002310B59A4200D110BDCC5CC4540133FB
:10BF7000F8E710B5884202D98B18984203D3002302
:10BF800007E08B5C8354013AFBD210BDCC5CC454F7
:10BF900001339A42FAD1F8E703001218934200D114
:10BFA000704719700133F9E7936810B5013B93604E
:10BFB000002B04DA9469A34207DB0A2905D0136831
:10BFC000581C10601970080010BD00F04BFC0100F7
:10BFD000F9E7F8B506000F001400D518AC4201D1FE
:10BFE000002007E021783A003000FFF7DDFF013440
:10BFF000431CF3D1F8BD0000F0B59FB002900F00D4
:10C0000016000593002805D083690493002B01D105
:10C0100000F0F4FD7B4B9F425BD1029B5F68BB89C4
:10C020001B0762D53B69002B5FD0002306AC636120
:10C03000203363761033A37635002B78002B01D0A4
:10C04000252B5CD1AB1B04930CD032003900029835
:10C05000FFF7BFFF431C00D1C4E06269049B944614
:10C06000634463612B78002B00D1BBE001220023E5
:10C070005242626002A9543252186E1C2360E3607F
:10C08000A3601370A365317805225F4800F0D4FEE9
:10C09000751C002835D12268D30604D5532302A984
:10C0A0005B1820211970130704D5532302A95B18CC
:10C0B0002B21197033782A2B2CD0350000210A202F
:10C0C000E3682A786E1C303A092A64D900292ED0F8
:10C0D00026E04E4B9F4202D1029B9F689FE74C4B4C
:10C0E0009F429CD1029BDF6899E73900029800F0DB
:10C0F0000FFC002899D0012040421FB0F0BD01354F
:10C100009BE7414B2268C01A0123834013432360FD
:10C110002E00B8E7059B191D1B680591002B01DB5C
:10C12000099304E05B42E3600223134323602B780E
:10C130002E2B0AD16B782A2B35D1059B02351A1D7F
:10C140001B680592002B2BDB0793324E29780322C4
:10C15000300000F071FE002806D04023801B834091
:10C160002268013513432360297806222A486E1C71
:10C17000217600F061FE00283AD0284B002B25D113
:10C180000722059B07339343083305936369039A9A
:10C190009B18636150E7434301219B18350090E7EA
:10C1A00001235B42D0E700230A201A0001356360B7
:10C1B00029786E1C3039092903D9002BC5D0079284
:10C1C000C3E74243012352183500F1E705AB009362
:10C1D0003A00134B2100029800E000BF0390039B3C
:10C1E0000133D3D1BB895B0600D584E70B9884E784
:10C1F00005AB00933A000A4B2100029800F080F84A
:10C20000ECE7C0469CEE000048EE0000BCEE0000EB
:10C210007CEE00004EEE000052EE00000000000038
:10C22000D3BF0000F7B5150001938A680B69009031
:10C230000C00934200DA130022002B604332127884
:10C24000002A01D001332B6023689B0602D52B689E
:10C2500002332B60062723681F4027D02300433377
:10C260001B785A1E93412268920630D4220001990D
:10C2700043320098089EB047431C25D0062320680F
:10C280002A68E16803400025042B03D18D1AEB4393
:10C29000DB171D40A3682269934201DD9B1AED184C
:10C2A0000027BD4220D1002010E00137E3682A6852
:10C2B0009B1ABB42D2DD220001231932019900985A
:10C2C000089EB047431CF0D101204042FEBD302003
:10C2D000E1184331087021005A1C45310978A21831
:10C2E000433202331170C1E7220001231A3201994F
:10C2F0000098089EB047431CE6D00137D1E7000004
:10C30000F0B589B004920A0043320593039002927B
:10C310000A7E0C000E9B6E2A00D186E01FD8632A8D
:10C3200033D008D8002A00D18CE0582A4DD02500FF
:10C3300042352A7030E0642A01D0692AF7D11968A1
:10C3400025680A1D280629D508681A60002803DA1E
:10C350002D23029A404213706B4E0A274FE0732A36
:10C3600074D008D86F2A1FD0702AE0D12022096823
:10C370000A43226003E0752A16D0782AD7D122001A
:10C38000782145321170614E22E025001A6842354D
:10C39000111D196013682B70012365E008681A608D
:10C3A0006906D3D500B2D1E719682568081D186061
:10C3B00008682E0605D5544E08276F2A1BD00A2779
:10C3C00019E06D06F7D580B2F5E745314E4E0A709B
:10C3D00018682268011D00681960150621D5D30769
:10C3E00002D520231A4322601027002803D12023DE
:10C3F00022689A4322602300002243331A70636844
:10C40000A360002B58DB042221689143216000289F
:10C4100054D1029D002B5AD02500337842352B7021
:10C4200055E05506DBD580B2D9E71A680D68101DB6
:10C430004969186013682E0601D5196002E06D067F
:10C44000FBD519800023029D23614FE01A68111D5E
:10C450001960156800216268280000F0EDFC0028D2
:10C4600001D0401B6060636823610023029A13704F
:10C470003CE023692A0004990398059DA847431CC2
:10C480003ED023689B0715D4079BE068984239DAB1
:10C49000180037E022000123193204990398059E01
:10C4A000B047431C2CD00135E368079A9B1AAB4276
:10C4B000F0DCE9E70025F7E70028ADD0029D390060
:10C4C000FDF722FC735C013D2B700028F7D1082F8B
:10C4D00009D12368DB0706D563682269934202DC31
:10C4E0003023013D2B70029B5B1B2361059B07AA38
:10C4F00000932100049B0398FFF794FE431CB8D1DE
:10C500000120404209B0F0BD59EE00006AEE000083
:10C510000D4B70B51C680500A36B002B0FD11820C4
:10C5200000F06EFC094BA0630360094B01224360DD
:10C53000084B83600B238381002302614361002247
:10C54000A36B1D615A6170BD880000200E33CDAB16
:10C5500034126DE6ECDE0500124B10B51C68A36BBF
:10C56000002B0FD1182000F04BFC0F4BA063036091
:10C570000E4B012243600E4B83600B23838100230B
:10C5800002614361A46B0B4A206961690A4BFDF7A4
:10C59000F7FC0122002380185941206161614800A5
:10C5A000400810BD880000200E33CDAB34126DE67C
:10C5B000ECDE05002D7F954C2DF451580CB430B5B0
:10C5C000164B9DB00C1E1D6808DA8B2301202B60D2
:10C5D00040421DB030BC08BC02B01847822302A9FB
:10C5E0009B008B810023029008619C4200D0631E57
:10C5F0008B604B6101235B42CB81209A21AB2800E9
:10C60000019300F055FD431C01DA8B232B60002CB5
:10C61000DFD00023029A1370DBE7C04688000020B9
:10C620000EB400B50B499CB01DAB0290069007916B
:10C6300004910948094904CB0591006802A90193B6
:10C6400000F036FD0023029A13701CB008BC03B042
:10C650001847C046FFFFFF7F880000200802FFFF49
:10C66000020010B51378541C002B05D1CC5CD454B7
:10C670000133002CFAD110BD2200F3E7C9B20378D0
:10C68000002B04D08B4200D170470130F7E74B42BA
:10C69000594149420840F7E702780B78002A03D055
:10C6A000013001319A42F7D0D01A70470023C25CA2
:10C6B0000133002AFBD1581E7047002330B59A423F
:10C6C0000AD0013AC45CCD5CAC4204D1934202D0A2
:10C6D0000133002CF6D1631B180030BD30B50500C6
:10C6E000002A00D130BD0C78013A6B1C2C7001314E
:10C6F000002C05D19A189A42F4D01C700133FAE745
:10C700001D00EDE710B50378002B0FD10B785A42CE
:10C7100053415B42184010BD0023CA5C002AFAD086
:10C72000C45C944201D10133F7E701300378002B58
:10C73000F2D11800EFE70000F0B51F000E0087B03F
:10C740000590019102920C98347800F0EAFA0822E0
:10C7500000194378751C134036D12D2C36D1B51CE9
:10C7600074780126002F62D0102F09D1302C07D108
:10C7700020222B789343582B54D110276C78023504
:10C780002D4B3900F31818000393FDF7BDFA0491FF
:10C7900001210023494202008C4618002100303953
:10C7A00009291AD80C00A74223DD591C09D0634679
:10C7B000824206D302D10499A14202DB01237843CD
:10C7C00020182C780135E9E72E00BCE72B2C01D08E
:10C7D0001E00C7E7B51C7478FAE721004139192912
:10C7E00001D8373CDFE721006139192901D8573CCE
:10C7F000D9E75A1C08D1059A23331360029B03988A
:10C80000002B09D107B0F0BD002E00D04042029AA3
:10C81000002AF7D0002B01D06B1E0193029B019AD6
:10C820001A60EFE73024002FAAD10827A8E7302CA0
:10C830009ED00A27A4E7C046FFFFFF7F37B513004D
:10C84000064A05001068046A002C00D1044C0A0056
:10C8500000942900FFF770FF3EBDC046880000200D
:10C86000EC000020F8B505000E001400002804D0EC
:10C870008369002B01D100F0C1F9224B9C422DD1DC
:10C880006C68A369A360A3891B0731D52369002BBA
:10C890002ED023682269F7B2981A6369F6B28342F0
:10C8A00005DC2100280000F03BF9002826D1A36810
:10C8B0000130013BA36023685A1C22601F7063692A
:10C8C000834204D0A389DB071AD50A2E18D1210090
:10C8D000280000F025F9002812D00FE00A4B9C42F6
:10C8E00001D1AC68CDE7094B9C42CAD1EC68C8E7DE
:10C8F0002100280000F00CF80028CAD0012676425A
:10C900003000F8BD9CEE0000BCEE00007CEE0000A4
:10C91000364B70B51D6806000C00002D05D0AB69C4
:10C92000002B02D1280000F069F9314B9C420FD155
:10C930006C680C23E25E93B219072DD4D90611D48A
:10C9400009230120336037331343A381404270BD74
:10C95000284B9C4201D1AC68EBE7274B9C42E8D1C5
:10C96000EC68E6E75B0713D5616B002908D023006C
:10C970004433994202D0300000F06AFA0023636326
:10C980002422A3899343A381002363602369236046
:10C990000823A2891343A3812369002B0BD1A02173
:10C9A0008022A389890092000B40934203D021008A
:10C9B000300000F0E1F90123A289134011D00023D7
:10C9C000A36063695B42A361002023698342BED1F7
:10C9D0000C23E25E1306BAD540231343A38101382A
:10C9E000B5E7920700D46369A360EDE788000020F3
:10C9F0009CEE0000BCEE00007CEE000010B50620AE
:10CA000000F090FC012000F0CFFD0000F7B58A890E
:10CA100005000C00130760D44B68002B04DC0B6C82
:10CA2000002B01DC0020FEBDE76A002FFAD00023B6
:10CA30002E682B6080235B01216A1A4034D0606D20
:10CA4000A3895B0706D56368C01A636B002B01D00E
:10CA5000236CC01A0200216A00232800E76AB84745
:10CA6000A189431C06D12B681D2B30D82B4ADA40F4
:10CA7000D3072CD50023636023692360CB0405D53D
:10CA8000431C02D12B68002B00D16065616B2E60C6
:10CA90000029C7D023004433994202D0280000F077
:10CAA000D7F900206063BEE701232800B847431C84
:10CAB000C6D12B68002BC3D01D2B01D0162B01D162
:10CAC0002E60AFE74023A2891343A381ABE7402345
:10CAD0000B430120A3814042A5E70F69002FA1D09D
:10CAE0000B680F60DB1B01930023920700D14B6999
:10CAF000A360019B002B00DC94E7019B3A00216AB4
:10CB00002800A66AB047002803DC4023A28913430B
:10CB1000DFE7019B3F181B1A0193EAE70100402061
:10CB20000B6970B505000C00002B01D1002070BD11
:10CB3000002804D08369002B01D100F05FF80B4B73
:10CB40009C4209D16C680C22A35E002BEED0210020
:10CB50002800FFF75BFFEAE7054B9C4201D1AC6878
:10CB6000F1E7044B9C42EED1EC68ECE79CEE000050
:10CB7000BCEE00007CEE0000002310B50400036052
:10CB80004360836081814366C28103614361836145
:10CB9000190008225C30FFF7FFF9054B246263623D
:10CBA000044BA362044BE362044B236310BDC046F5
:10CBB00065D300008DD30000C5D30000F1D3000081
:10CBC00010B5024900F08CF810BDC04621CB000022
:10CBD00070B568254A1E55430E002900743100F0D7
:10CBE00081F9041E08D000212A00016046600C3043
:10CBF000A0606832FFF7D0F9200070BD836913B5DB
:10CC00000400002B28D18364C3640365134B144ACA
:10CC10001B6882620193984201D101238361200045
:10CC200000F020F86060200000F01CF8A0602000F8
:10CC300000F018F80022E06004216068FFF79CFF14
:10CC400001220921A068FFF797FF02221221E06864
:10CC5000FFF792FF0123A36113BDC04644EE00001D
:10CC6000C1CB0000F8B51C4B07001E68B369002B50
:10CC700002D13000FFF7C2FF4836B4687368013B49
:10CC800004D53368002B07D03668F6E70C22A55E82
:10CC9000002D0DD06834F2E704213800FFF798FF2B
:10CCA00030600028F0D10C2304003B602000F8BD68
:10CCB00020000A4B656625606560A560E36025611C
:10CCC0006561A561082229005C30FFF765F965639D
:10CCD000A563A564E564E9E744EE00000100FFFFF9
:10CCE000F7B504000700002601914834002C01D15B
:10CCF0003000FEBD6368A5680093009B013B009374
:10CD000001D52468F2E7AB89012B08D90E22AB5E6E
:10CD1000013304D029003800019B98470643683549
:10CD2000EBE7EC300068704770B50E001D000E2375
:10CD3000C95E96B01400002907DA00232B60B3897E
:10CD40001B0611D48023DB000FE06A4600F088FB4D
:10CD50000028F2DBF022019B12021340054A9B18C7
:10CD60005A4253412B60EDE740230020236016B068
:10CD700070BDC04600E0FFFFF7B502268B890500B5
:10CD80000C00334206D02300473323602361012384
:10CD90006361F7BD01AB6A46FFF7C6FF0099070064
:10CDA000280000F09FF8002808D10C22A35E9A0505
:10CDB000EFD4032293431E43A681E4E70F4BAB62FB
:10CDC0008023A28920601343A381009B20616361BB
:10CDD000019B002B0DD00E23E15E280000F052FBDA
:10CDE000002806D00322A38993431A00012313438A
:10CDF000A381A0893843A081CBE7C046C1CB000006
:10CE000010B5034B0100186800F06CF810BDC04667
:10CE10008800002082B0002900D101A9101E06D090
:10CE2000002B06D013780B601078431E984102B097
:10CE3000704702204042FAE7C9B28218904201D1FD
:10CE40000020704703788B42FBD00130F6E70000EA
:10CE500070B50500002910D00C1F2368002B00DAE4
:10CE6000E418280000F034FB1D4A1368002B05D19C
:10CE700063601460280000F02CFB70BDA34209D948
:10CE8000216860188342F3D118685B6841182160FB
:10CE9000EEE713005A68002A01D0A242F9D91968B6
:10CEA0005818A0420BD120680918581819608242FE
:10CEB000E0D110685268411819605A60DAE7A04260
:10CEC00002D90C232B60D5E721686018824203D178
:10CED000106852684118216062605C60CAE7C04611
:10CEE000381C0020032370B5CD1C9D430835060077
:10CEF0000C2D1ED20C25A9421DD8300000F0E8FAF6
:10CF0000254A14682100002919D1244C2368002BDC
:10CF100003D1300000F0CAF920602900300000F091
:10CF2000C5F9431C2BD10C233000336000F0D1FA3B
:10CF300003E0002DDFDA0C233360002070BD0B68A6
:10CF40005B1B19D40B2B03D90B60CC18256003E0B5
:10CF50004B688C420DD11360300000F0BAFA20000B
:10CF600007220B30231D9043C31AE7D05A42E250E8
:10CF7000E4E763600C00EFE70C004968C3E70323B4
:10CF8000C41C9C43A042E1D0211A300000F08EF96D
:10CF9000431CDBD1C7E7C046381C00203C1C0020E6
:10CFA000F8B507000D001600002905D11100FFF7A4
:10CFB00099FF04002000F8BD002A03D1FFF748FFC5
:10CFC0003400F7E700F086FA2C00B042F2D23100CC
:10CFD0003800FFF787FF041EECD029003200FEF76F
:10CFE000BFFF29003800FFF733FFE3E7F0B58E6895
:10CFF00085B007000C00039201939E423CD8902319
:10D000008A89DB001A4234D00325096923685B1A38
:10D010000293636902985D43EB0F5D19019B6D10EC
:10D0200001331B18AB4200D91D00530532D529002E
:10D030003800FFF757FF061E09D10C233B60402341
:10D040000120A28940421343A38105B0F0BD029A9A
:10D050002169FEF785FFA389144A1A4080231343F0
:10D06000A381029B2661F61826606561019EED1A78
:10D07000A560019B9E4200D9019E32000399206861
:10D08000FEF777FFA36800209B1BA36023689E190F
:10D090002660DAE72A003800FFF782FF061EE0D19B
:10D0A00021693800FFF7D4FEC7E7C0467FFBFFFFCA
:10D0B000F0B59FB0029005938B890F0016001B06F8
:10D0C00011D50B69002B0ED14021FFF70BFF386003
:10D0D0003861002805D10C23029A013813601FB073
:10D0E000F0BD40237B61002306AC6361203363768F
:10D0F0001033A37635002B78002B01D0252B46D199
:10D10000AB1B04930CD0320039000298FFF76EFF7E
:10D11000431C00D1AEE06269049B944663446361A2
:10D120002B78002B00D1A5E001220023524262603F
:10D1300002A9543252186E1C2360E360A36013707E
:10D14000A365317805225448FFF776FE751C002848
:10D150001FD12268D30604D5532302A95B182021CE
:10D160001970130704D5532302A95B182B211970DA
:10D1700033782A2B16D0350000210A20E3682A785C
:10D180006E1C303A092A4ED9002918D010E001351A
:10D19000B1E7414B2268C01A012383401343236047
:10D1A0002E00CEE7059B191D1B680591002B01DBA6
:10D1B000099304E05B42E3600223134323602B786E
:10D1C0002E2B0AD16B782A2B35D1059B02351A1DDF
:10D1D0001B680592002B2BDB0793304E2978032226
:10D1E0003000FFF729FE002806D04023801B834033
:10D1F00022680135134323602978062228486E1CD3
:10D200002176FFF719FE00283CD0264B002B25D1B4
:10D210000722059B07339343083305936369039AF9
:10D220009B18636166E7434301219B183500A6E71D
:10D2300001235B42D0E700230A201A000135636016
:10D2400029786E1C3039092903D9002BC5D00792E3
:10D25000C3E74243012352183500F1E705AB0093C1
:10D260003A00114B2100029800E000BF0390039B9D
:10D270000133D3D1BB890B985B0600D42FE7012083
:10D2800040422CE705AB00933A00074B210002987F
:10D29000FFF736F8EAE7C04648EE00004EEE000021
:10D2A00052EE000000000000EDCF0000002370B53A
:10D2B000064C05000800236000F060F9431C03D110
:10D2C0002368002B00D02B6070BDC046CC2F0020FF
:10D2D00070B504000D001F2904D916230360012036
:10D2E000404270BD436C002B04D08A009B181A6822
:10D2F000002A08D1200000F031F82A0001002000A7
:10D3000000F01AF8EDE70020012AEAD0511C03D101
:10D31000162301302360E4E7002428001C609047B6
:10D320002000DEE710B5034B01001868FFF7D0FFBF
:10D3300010BDC04688000020002370B5064C0500D3
:10D3400008001100236000F001F9431C03D1236899
:10D35000002B00D02B6070BDCC2F002010B500F04A
:10D36000E5F810BD70B50C000E25495F00F0BAF865
:10D37000002803DB636D1B18636570BDA389024A37
:10D380001340A381F9E7C046FFEFFFFFF8B51F0088
:10D390008B8905000C001600DB0505D50E23C95E40
:10D3A0000022022300F080F8A389054A28001340D8
:10D3B000A38132000E23E15E3B0000F02BF8F8BDA4
:10D3C000FFEFFFFF70B50C000E25495F00F06CF811
:10D3D000A389421C03D1054A1340A38170BD80225A
:10D3E00052011343A3816065F8E7C046FFEFFFFFDA
:10D3F00010B50E23C95E00F021F810BD0B1E04D03D
:10D40000FF2A04D98A2303608B3B180070470A70F7
:10D410000123FAE770B50500080011000022064C50
:10D4200022601A0000F0B8F8431C03D12368002BD7
:10D4300000D02B6070BDC046CC2F0020002370B5FB
:10D44000064C05000800236000F060F8431C03D17F
:10D450002368002B00D02B6070BDC046CC2F00206D
:10D46000002370B5064C050008001100236000F091
:10D4700055F8431C03D12368002B00D02B6070BDEE
:10D48000CC2F0020002370B5064C05000800236057
:10D4900000F054F8431C03D12368002B00D02B600C
:10D4A00070BDC046CC2F002070B5050008001100EB
:10D4B0000022064C22601A0000F050F8431C03D1F1
:10D4C0002368002B00D02B6070BDC046CC2F0020FD
:10D4D000704770470B1F1B68181F002B01DA0B5891
:10D4E000C018704770B50500080011000022064CF6
:10D4F00022601A0000F03AF8431C03D12368002B85
:10D5000000D02B6070BDC046CC2F002058220120D7
:10D51000014B40421A607047CC2F00205822012056
:10D52000014B40421A607047CC2F00205822012046
:10D53000014B40421A607047CC2F00205822024B0A
:10D5400000201A607047C046CC2F002058220120CE
:10D55000014B40421A607047CC2F00205822012016
:10D56000014B40421A607047CC2F00205822012006
:10D57000014B40421A607047CC2F0020044A1368C8
:10D58000002B00D1034B1818106018007047C046DC
:10D59000401C0020D02F002058220120014B404287
:10D5A0001A607047CC2F0020FEE7C046F8B5C04691
:10D5B000F8BC08BC9E467047F8B5C046F8BC08BC2D
:10D5C0009E467047646174610000000058D60000F8
:10D5D000EF01000061D60000E302000069D6000000
:10D5E0009D0A000070D60000AD0B000075D600004B
:10D5F000090500007BD600008906000086D60000E1
:10D60000530300008BD60000050E000097D60000E3
:10D610001F020000A1D6000069090000AFD600007B
:10D62000310A0000BCD6000015080000C8D6000072
:10D630004906000072616E646F6D00616C6C006C75
:10D640006173740066616C736500747275650025A2
:10D650002E3135732E2E2E006D616B654C697374FF
:10D66000006164644C6173740064656C657465008A
:10D670006A6F696E0073706C697400636F707946CD
:10D68000726F6D546F0066696E64006A6F696E53E5
:10D690007472696E677300756E69636F6465417457
:10D6A00000756E69636F6465537472696E67006EAE
:10D6B000657742797465417272617900617342796C
:10D6C0007465417272617900667265654D656D6F52
:10D6D0007279000039D70000911200003ED7000097
:10D6E000AF12000069D60000B312000044D700005A
:10D6F000951200004ED70000B712000057D7000067
:10D70000BB12000061D70000BF1200006CD7000000
:10D71000C312000078D700009912000081D70000E2
:10D72000A71200008BD700009D12000096D70000C2
:10D73000AB12000066696C65006F70656E00636C0B
:10D740006F736500656E644F6646696C650072654F
:10D7500061644C696E6500726561644279746573D9
:10D7600000617070656E644C696E65006170706513
:10D770006E6442797465730066696C6553697A6595
:10D780000073746172744C697374006E65787449C7
:10D790006E4C6973740073797374656D496E666F4E
:10D7A000000000007C1600008C160000A616000089
:10D7B000221700005A1700008E170000C61700003D
:10D7C000EC1700003018000072180000C8180000A4
:10D7D0000C1900006E190000B8190000DE190000D5
:10D7E000161A00005C1A0000821A0000B01A00002D
:10D7F000DE1A0000B6310000961B0000681C000015
:10D80000DE1C00004E1D00009A1D0000BA1D000025
:10D81000DC1D0000341F0000781F0000F01F000016
:10D820001E20000050200000822000000221000085
:10D830006A210000C6210000242200009622000078
:10D840000823000064230000BE230000F42300002E
:10D85000442400008A240000D22400002625000071
:10D860007A250000B8250000242600005A26000072
:10D87000A2260000EA260000322700006C270000E4
:10D88000B42700000428000066290000B01A000038
:10D89000161A00006C2800007C160000A228000068
:10D8A000CE28000004290000302900007C1600006A
:10D8B0007C1600007C1600007C160000E2290000A7
:10D8C000242A00006A2A0000BA2A0000E62A000082
:10D8D0005E2B0000B02B0000142C00007C16000012
:10D8E0007C160000382C0000682C0000982C0000EA
:10D8F000CE2C0000F82C00002E2D0000582D00002A
:10D90000802D0000A82D0000D82D0000082E00005A
:10D91000322E00005C2E00008C2E0000B62E00007F
:10D920007C1600007C1600007C1600007C160000AF
:10D930007C160000E62E0000122F00003E2F000093
:10D940006A2F0000962F0000CC2F00000C30000042
:10D950004230000078300000A4300000D0300000D9
:10D96000063100007C1600007C1600007C160000CA
:10D970007C1600007C1600007C1600007C1600005F
:10D980007C1600007C1600007C1600007C1600004F
:10D990007C16000032310000323100000C320000F1
:10D9A000423200005B2564206974656D206C6973E8
:10D9B000745D002825642062797465732900286FDE
:10D9C000626A65637420747970653A202564290061
:10D9D000537461636B20756E646572666C6F77005B
:10D9E000626F6F6C65616E006E756D62657200735B
:10D9F0007472696E67006C69737400627974652073
:10DA000061727261790000000700000003000000ED
:10DA100071DA00006533000079DA00001534000087
:10DA200082DA0000873500008BDA000069330000DD
:10DA300094DA00008B3500009CDA00007535000098
:10DA4000A5DA0000A53400001C0000000100000061
:10DA500002000000040000000500000006000000B5
:10DA6000100000001100000043616C6C696F70656C
:10DA700000686173546F6E6500706C6179546F6EED
:10DA80006500686173536572766F007365745365E2
:10DA900072766F00646163496E69740064616357F4
:10DAA000726974650073717561726557617665009E
:10DAB000474320746F6F6B20256420757365637313
:10DAC0003B206672656520256420776F7264730061
:10DAD0003C496E74656765723E003C4C6973743EE8
:10DAE000003C4F626A6563743E003C427974654154
:10DAF000727261793E000D0A564D2050616E696365
:10DB00003A2025730D0A006D6973630041DB000044
:10DB1000814200004ADB0000114200004EDB0000A1
:10DB20006541000056DB00000B41000060DB000097
:10DB3000A14000006CDB0000A33F00006E756C6C20
:10DB400000686578546F496E740073696E006A737B
:10DB50006F6E476574006A736F6E436F756E740005
:10DB60006A736F6E56616C75654174006A736F6E8F
:10DB70004B6579417400000004DC0000ED420000B8
:10DB80000CDC0000F142000016DC00000F43000036
:10DB90001FDC0000194300002ADC000023430000C2
:10DBA00036DC00002D43000044DC00003743000059
:10DBB0004CDC00004143000052DC00004B430000FD
:10DBC00067DC0000554300007CDC00005F43000080
:10DBD00088DC00006943000098DC0000734300000B
:10DBE000A4DC00007D430000B1DC0000874300009E
:10DBF000C0DC0000FB420000D3DC00000543000055
:10DC00006E65740068617357694669007374617268
:10DC100074576946690073746F7057694669007775
:10DC2000696669537461747573006D794950416414
:10DC300064726573730073746172745353494473EF
:10DC400063616E0067657453534944006D794D41BB
:10DC500043006874747053657276657247657452D8
:10DC600065717565737400726573706F6E64546F5F
:10DC7000487474705265717565737400687474705B
:10DC8000436F6E6E65637400687474704973436F9C
:10DC90006E6E656374656400687474705265717546
:10DCA0006573740068747470526573706F6E736519
:10DCB00000776562536F636B6574537461727400AF
:10DCC000776562536F636B65744C617374457665F9
:10DCD0006E7400776562536F636B657453656E6431
:10DCE000546F436C69656E74000D0E0F04050C0BC8
:10DCF0000A06070809000000000008080800080AD2
:10DD00004A4000000A5FEA5FEA0ED92ED36E19324C
:10DD10004489330C924C924D080800000004880896
:10DD200008040804848488000A448A4000048EC4DD
:10DD300080000000048800000EC000000000080001
:10DD400001224488100C9252524C048C84848E1C04
:10DD5000824C901E1EC244924C06CA525FE21FF0D3
:10DD60001EC13E02448ED12E1FE24488100ED12ED9
:10DD7000D12E0ED12EC488000800080000048004B3
:10DD8000880244880482000EC00EC00804824488C1
:10DD90000ED126C0040ED135B36C0C925ED2521C4B
:10DDA000925C925C0ED010100E1C9252525C1ED0EF
:10DDB0001C901E1ED01C90100ED013712E12525E9D
:10DDC000D2521C8808081C1FE242524C125498146C
:10DDD00092101010101E113B75B131113935B3710D
:10DDE0000C9252524C1C925C90100C92524C861C1D
:10DDF000925C92510ED00C825C1FE4848484125297
:10DE000052524C1131312A44113135BB7112524CEE
:10DE10009252112A4484841EC488101E0EC8080819
:10DE20000E10080482410EC242424E048A40000095
:10DE3000000000001F0804800000000ED2524F10A6
:10DE4000101C925C000ED0100E02424ED24E0C926C
:10DE50005C900E06C81C88080ED24EC24C10101CD6
:10DE600092520800080808024002424C101498140C
:10DE7000920808080806001B75B131001C92525226
:10DE8000000C92524C001C925C90000ED24EC200CC
:10DE90000ED010100006C8049808080EC80700121B
:10DEA00052524F0011312A4400113135BB00124C3F
:10DEB0008C9200112A4498001EC4881E06C48C84CB
:10DEC00086080808080818080C881800000C8360E9
:10DED000000000000100000002000000030000003C
:10DEE000040000000500000006000000070000001C
:10DEF00008000000090000000A0000000B000000FC
:10DF00000C0000000D0000000E0000000F000000DB
:10DF100010000000120000001400000016000000B5
:10DF2000180000001A0000001C0000001E00000085
:10DF3000200000002300000026000000290000004F
:10DF40002C0000002F00000032000000360000000E
:10DF50003A0000003E0000004200000046000000C1
:10DF60004B00000050000000550000005A00000067
:10DF700061000000680000006F00000076000000F3
:10DF80007D000000840000008B0000009200000073
:10DF900099000000A0000000A7000000AE000000F3
:10DFA000B5000000BC000000C3000000CA00000073
:10DFB000D1000000D8000000DF000000E6000000F3
:10DFC000ED000000F4000000FB000000FF00000076
:10DFD00020E00000A94300002BE0000045490000BC
:10DFE00035E000006D45000042E00000B54700004C
:10DFF00049E000000548000052E0000055480000DC
:10E000005EE000004D4700006FE00000DD450000CD
:10E010007CE00000DD460000646973706C6179008B
:10E020006C696768744C6576656C006D62446973F1
:10E03000706C6179006D62446973706C61794F66D0
:10E0400066006D62506C6F74006D62556E706C6F1F
:10E0500074006D62447261775368617065006D622F
:10E060005368617065466F724C6574746572006EBA
:10E07000656F506978656C53656E64006E656F50AE
:10E080006978656C53657450696E004E6F742065D5
:10E090006E6F75676820726F6F6D206576656E2094
:10E0A000616674657220636F6D70616374696F6E11
:10E0B00000436F6D70616374656420466C617368C2
:10E0C00020636F64652073746F72650A2564206233
:10E0D0007974657320757365642028256425252966
:10E0E000206F6620256400426164207265636F7250
:10E0F0006420666F756E6420647572696E6720694E
:10E100006E697469616C697A6174696F6E00256407
:10E110002025642025642028256420776F7264738D
:10E1200029002564207265636F7264732C20256456
:10E1300020776F7264732C206D61784944202564C8
:10E140002C20636F6D70616374696F6E20637963F7
:10E150006C657320256400526573746F726564206A
:10E1600025642073637269707473005374617274F0
:10E17000656400726164696F000000000CE20000D9
:10E180001D53000019E20000B955000029E200000B
:10E190003955000037E200004D57000042E2000010
:10E1A0004553000052E20000CD53000066E200003B
:10E1B000B553000075E200002F59000081E2000015
:10E1C000AD5800008AE200005158000095E20000BE
:10E1D00099570000A0E20000D5570000A9E2000016
:10E1E00009580000B2E2000055530000C1E20000EF
:10E1F00035530000CAE20000655300006E6F6E6583
:10E20000006F74686572007061697200646973619F
:10E21000626C65526164696F006D657373616765F7
:10E220005265636569766564007061636B657452FD
:10E23000656365697665007061636B657453656ECF
:10E2400064007265636569766564496E74656765C7
:10E25000720072656365697665644D6573736167A5
:10E260006554797065007265636569766564537499
:10E2700072696E670073656E64496E746567657276
:10E280000073656E64506169720073656E645374E7
:10E2900072696E67007365744368616E6E656C00C9
:10E2A00073657447726F757000736574506F77652E
:10E2B00072007369676E616C537472656E6774681F
:10E2C000006465766963654944006C6173744D65EB
:10E2D0007373616765494400556E6B6E6F776E208E
:10E2E0007072696D6974697665205B25733A257370
:10E2F0005D00000000000000963007772C610EEEF4
:10E30000BA51099919C46D078FF46A7035A563E98C
:10E31000A395649E3288DB0EA4B8DC791EE9D5E0B3
:10E3200088D9D2972B4CB609BD7CB17E072DB8E7B2
:10E33000911DBF906410B71DF220B06A4871B9F307
:10E34000DE41BE847DD4DA1AEBE4DD6D51B5D4F440
:10E35000C785D38356986C13C0A86B647AF962FDA5
:10E36000ECC9658A4F5C0114D96C0663633D0FFAF2
:10E37000F50D088DC8206E3B5E10694CE44160D5F8
:10E38000727167A2D1E4033C47D4044BFD850DD2E2
:10E390006BB50AA5FAA8B5356C98B242D6C9BBDBF5
:10E3A00040F9BCACE36CD832755CDF45CF0DD6DCF0
:10E3B000593DD1ABAC30D9263A00DE518051D7C897
:10E3C0001661D0BFB5F4B42123C4B3569995BACF22
:10E3D0000FA5BDB89EB802280888055FB2D90CC643
:10E3E00024E90BB1877C6F2F114C6858AB1D61C1BC
:10E3F0003D2D66B69041DC760671DB01BC20D298DB
:10E400002A10D5EF8985B1711FB5B606A5E4BF9F67
:10E4100033D4B8E8A2C9077834F9000F8EA809965A
:10E4200018980EE1BB0D6A7F2D3D6D08976C6491C5
:10E43000015C63E6F4516B6B62616C1CD8306585DE
:10E440004E0062F2ED95066C7BA5011BC1F40882BB
:10E4500057C40FF5C6D9B06550E9B712EAB8BE8BFC
:10E460007C88B9FCDF1DDD62492DDA15F37CD38C85
:10E47000654CD4FB5861B24DCE51B53A7400BCA383
:10E48000E230BBD441A5DF4AD795D83D6DC4D1A4B5
:10E49000FBF4D6D36AE96943FCD96E34468867AD8C
:10E4A000D0B860DA732D0444E51D03335F4C0AAA2B
:10E4B000C97C0DDD3C710550AA41022710100BBE2E
:10E4C00086200CC925B56857B3856F2009D466B975
:10E4D0009FE461CE0EF9DE5E98C9D9292298D0B0AA
:10E4E000B4A8D7C7173DB359810DB42E3B5CBDB757
:10E4F000AD6CBAC02083B8EDB6B3BF9A0CE2B603D8
:10E500009AD2B1743947D5EAAF77D29D1526DB048C
:10E510008316DC73120B63E3843B64943E6A6D0DD7
:10E52000A85A6A7A0BCF0EE49DFF099327AE000A22
:10E53000B19E077D44930FF0D2A3088768F2011EB5
:10E54000FEC206695D5762F7CB67658071366C194C
:10E55000E7066B6E761BD4FEE02BD3895A7ADA106D
:10E56000CC4ADD676FDFB9F9F9EFBE8E43BEB7174E
:10E57000D58EB060E8A3D6D67E93D1A1C4C2D838D8
:10E5800052F2DF4FF167BBD16757BCA6DD06B53F3E
:10E590004B36B248DA2B0DD84C1B0AAFF64A03367D
:10E5A000607A0441C3EF60DF55DF67A8EF8E6E31FC
:10E5B00079BE69468CB361CB1A8366BCA0D26F2545
:10E5C00036E2685295770CCC03470BBBB916022292
:10E5D0002F260555BE3BBAC5280BBDB2925AB42BA7
:10E5E000046AB35CA7FFD7C231CFD0B58B9ED92CBC
:10E5F0001DAEDE5BB0C2649B26F263EC9CA36A7521
:10E600000A936D02A906099C3F360EEB85670772D7
:10E6100013570005824ABF95147AB8E2AE2BB17B3E
:10E62000381BB60C9B8ED2920DBED5E5B7EFDC7CC5
:10E6300021DFDB0BD4D2D38642E2D4F1F8B3DD681C
:10E640006E83DA1FCD16BE815B26B9F6E177B06F17
:10E650007747B718E65A0888706A0FFFCA3B066604
:10E660005C0B0111FF9E658F69AE62F8D3FF6B6191
:10E6700045CF6C1678E20AA0EED20DD75483044E33
:10E68000C2B30339612667A7F71660D04D476949C1
:10E69000DB776E3E4A6AD1AEDC5AD6D9660BDF40D4
:10E6A000F03BD83753AEBCA9C59EBBDE7FCFB24787
:10E6B000E9FFB5301CF2BDBD8AC2BACA3093B3536C
:10E6C000A6A3B4240536D0BA9306D7CD2957DE5475
:10E6D000BF67D9232E7A66B3B84A61C4021B685D4E
:10E6E000942B6F2A37BE0BB4A18E0CC31BDF055AC7
:10E6F0008DEF022D416C6C207461736B7320737409
:10E700006F707065640076313230002025732025EB
:10E7100073004D656D6F727920636C65617265641D
:10E72000004E6F2066726565207461736B20656EA4
:10E730007472696573000000A8E70000B16F000003
:10E74000B5E70000096F0000C1E70000D96E0000C6
:10E75000C7E70000E96E0000CDE70000F96E000099
:10E76000D3E70000896C0000E9E7000011690000B0
:10E77000F3E70000256F0000FBE70000C96C000014
:10E7800004E80000D16A000010E80000ED69000014
:10E7900019E80000396A000021E80000DD6B000084
:10E7A00073656E736F727300616363656C6572612C
:10E7B00074696F6E0074656D7065726174757265F1
:10E7C0000074696C74580074696C74590074696CD5
:10E7D000745A00736574416363656C65726F6D652F
:10E7E00074657252616E676500746F756368526517
:10E7F0006164006932635265616400693263577213
:10E800006974650073706945786368616E67650057
:10E81000737069536574757000726561644448541F
:10E82000006D6963726F70686F6E650039D70000A4
:10E83000BD7000003ED70000697000005BE800007A
:10E840006971000060E800008570000069E8000060
:10E850000171000073657269616C0072656164002A
:10E8600072656164496E746F007772697465000047
:10E87000ECE8000099710000FAE80000A9710000BE
:10E8800007E900009D71000010E90000AD71000073
:10E890001AE90000B171000023E90000B571000021
:10E8A00028E90000B97100002DE90000BD710000E9
:10E8B00039E90000C171000040E90000C5710000A5
:10E8C00049E90000C97100004EE90000CD71000067
:10E8D00059E90000D171000063E90000A171000056
:10E8E0006DE90000A571000074667400656E6162D8
:10E8F0006C65446973706C6179007365744261631F
:10E900006B6C696768740067657457696474680044
:10E9100067657448656967687400736574506978E1
:10E92000656C006C696E65007265637400726F756A
:10E930006E6465645265637400636972636C65003C
:10E94000747269616E676C650074657874007466D2
:10E9500074546F756368656400746674546F75638E
:10E96000685800746674546F7563685900746674EF
:10E97000546F756368507265737375726500766164
:10E9800072730000A4E9000061760000AEE90000A7
:10E9900041760000B7E900001D760000C3E90000E1
:10E9A000AB750000766172457869737473007661A7
:10E9B000724E616D6564007365745661724E616D6F
:10E9C0006564007661724E616D65466F72496E6472
:10E9D00065780057656C636F6D6520746F204D69B5
:10E9E00063726F426C6F636B732100705F73706949
:10E9F00020213D204E554C4C002F686F6D652F67D0
:10EA000069742F2E706C6174666F726D696F2F70F0
:10EA100061636B616765732F6672616D65776F7295
:10EA20006B2D61726475696E6F6E6F726469636E6F
:10EA30007266352F6C69627261726965732F53500B
:10EA4000492F5350492E63707000535049436C61F5
:10EA500073733A3A535049436C617373284E52466C
:10EA60005F5350495F547970652A2C2075696E7424
:10EA7000385F742C2075696E74385F742C2075694A
:10EA80006E74385F74290000000000000000000070
:10EA900035780000F1770000177800002178000039
:10EAA0002B78000015780000000000000100000035
:10EAB0000200000016000000040000000500000035
:10EAC0000600000007000000080000000900000028
:10EAD0000A0000000B0000000C0000000D00000008
:10EAE0000E0000000F0000001A0000001B000000D4
:10EAF00014000000130000001100000017000000C7
:10EB0000100000001C0000001D0000001E0000009E
:10EB100012000000150000000300000018000000B3
:10EB2000190000000000000000000000217C00002F
:10EB300055840000A17C0000B57C0000AB7C000087
:10EB40001D7C0000117C0000C17C00003D7C0000A9
:10EB50000D7C0000000000000000000000003043B9
:10EB600000000000000030C37371727400000000E8
:10EB7000FB21F93FFB2109407CD91240FB211940C0
:10EB80007A6A1F407CD92240BBFD2540FB212940E9
:10EB90003A462C407A6A2F405C4731407CD932405B
:10EBA0009C6B3440BBFD3540DB8F3740FB21394047
:10EBB0001BB43A403A463C405AD83D407A6A3F40FE
:10EBC0004C7E40405C4741406C1042407CD9424002
:10EBD0008CA243409C6B4440AC344540BBFD454057
:10EBE000CBC64640DB8F4740EB584840FB214940AD
:10EBF00083F9A200444E6E00FC291500D15727006E
:10EC0000DD34F50062DBC0003C9995004190430083
:10EC10006351FE00BBDEAB00B761C5003A6E240055
:10EC2000D24D42004906E00009EA2E001C92D100B4
:10EC3000EB1DFE0029B11C00E83EA700F53582005F
:10EC400044BB2E009CE98400B4267000417E5F0026
:10EC5000D6913900538339009CF439008B5F8400CE
:10EC600028F9BD00F81F3B00DEFF97000F98050054
:10EC7000112FEF000A5A8B006D1F6D00CF7E3600FA
:10EC800009CB2700464FB7009E663F002DEA5F0084
:10EC9000BA277500E5EBC7003D7BF100F7390700A7
:10ECA00092528A00FB6BEA001FB15F00085D8D0085
:10ECB000300356007BFC4600F0AB6B0020BCCF005D
:10ECC00036F49A00E3A91D005E619100081BE6007E
:10ECD00085996500A0145F008D40680080D8FF0012
:10ECE00027734D0006063100CA561500C9A87300E7
:10ECF0007BE260006B8CC00000000040FB21F93F0C
:10ED0000000000002D44743E000000809846F83C4E
:10ED10000000006051CC783B00000080831BF0397C
:10ED20000000004020257A38000000802282E3366F
:10ED3000000000001DF36935020000000300000020
:10ED40000400000006000000CCA0000076A0000037
:10ED500076A00000A4A1000072A0000072A0000034
:10ED60009AA10000A4A1000072A000009AA10000D6
:10ED700072A00000A4A10000A8A10000A8A10000AA
:10ED8000A8A10000B0A10000A8AB00001AAA0000D2
:10ED90005EAA0000C2A900005EAA00004EAB0000FF
:10EDA0005EAA0000C2A900001AAA00001AAA000068
:10EDB0004EAB0000C2A90000BAA90000BAA9000029
:10EDC000BAA900005CAB0000D0B20000D2B10000D4
:10EDD000D2B10000F0B40000CCB10000CCB1000012
:10EDE000D8B40000F0B40000CCB10000D8B40000EA
:10EDF000CCB10000F0B40000E6B40000E6B40000BE
:10EE0000E6B40000F4B400002C2066756E637469EB
:10EE10006F6E3A2000617373657274696F6E2022A1
:10EE2000257322206661696C65643A2066696C65A9
:10EE300020222573222C206C696E652025642573A1
:10EE400025730A008C000020232D302B2000686CD5
:10EE50004C006566674546470030313233343536FD
:10EE60003738394142434445460030313233343536
:10EE7000363738396162636465660000000000005F
:10EE80000000000000000000000000000000000082
:10EE90000000000000000000000000000000000072
:10EEA0000000000000000000000000000000000062
:10EEB0000000000000000000000000000000000052
:10EEC0000000000000000000000000000000000042
:10EED000000000000000000000000000504F5349F7
:10EEE000580000202020202020202020282828280A
:10EEF000282020202020202020202020202020200A
:10EF00002020208810101010101010101010101059
:10EF10001010100404040404040404040410101069
:10EF20001010101041414141414101010101010115
:10EF300001010101010101010101010101011010A3
:10EF400010101010424242424242020202020202E9
:10EF50000202020202020202020202020202101075
:10EF60001010200000000000000000000000000061
:10EF70000000000000000000000000000000000091
:10EF80000000000000000000000000000000000081
:10EF90000000000000000000000000000000000071
:10EFA0000000000000000000000000000000000061
:10EFB0000000000000000000000000000000000051
:10EFC0000000000000000000000000000000000041
:10EFD0000000000000000000000000000000000031
:08EFE000000000000000000029
:08EFE8002011FF7F0100000071
:10EFF000FFFFFFFFE803000001000000E803DC055D
:10F00000DC05DC05DC050000FFFFFFFFFFFFFFFF65
:10F010001800000019FCFFFFFFFFFFFF02000000C7
:10F0200040420F000024F400020000000300000032
:10F03000FFFFFFFF000000000100000000000200D1
:10F0400001000000FFFFFFFF0000000002000000C1
:10F050000000040002000000FFFFFFFF00000000AE
:10F060000300000000000800030000000A00000088
:10F0700008000000010000008C00002000000000DB
:10F080009CEE0000BCEE00007CEE000000000000E2
:10F090000000000000000000000000000000000070
:10F0A0000000000000000000000000000000000060
:10F0B0000000000000000000000000000000000050
:10F0C0000000000000000000000000000000000040
:10F0D00000000000000000000000000043000000ED
:10F0E0000000000000000000000000000000000020
:10F0F00000000000000000000000000043000000CD
:10F1000000000000000000000000000000000000FF
:10F1100000000000000000000000000043000000AC
:10F1200000000000000000000000000000000000DF
:10F13000000000000000000000000000430000008C
:10F1400000000000000000000000000000000000BF
:10F15000000000000000000000000000430000006C
:10F16000000000000000000000000000000000009F
:10F17000000000000000000000000000430000004C
:10F18000000000000000000000000000000000007F
:10F19000000000000000000000000000430000002C
:10F1A000000000000000000000000000000000005F
:10F1B000000000000000000000000000FDD300007F
:10F1C00015CE000000000000E2EE000056D6000060
:10F1D00006DB000006DB000006DB000006DB0000AB
:10F1E00006DB000006DB000006DB000006DB00009B
:10F1F00006DB0000FFFFFFFFFFFFFFFFFFFFFFFF3A
:10F20000FFFF000001004153434949000000000096
:10F2100000000000000000000000000000000000EE
:10F220000000000000004153434949000000000075
:10F2300000000000000000000000000000000000CE
:10F240000000000000000000E9000000C17700009D
:0CF25000157B00006D7F0000C100000075
:0400000300007BB1CD
:00000001FF
